:020000040800F2
:1000000000060020E1020008E3020008E302000805
:10001000E3020008E3020008E3020008E30200082C
:10002000E3020008E3020008E3020008358A000842
:10003000E3020008E3020008E3020008E30200080C
:10004000E3020008E3020008E3020008E3020008FC
:10005000E3020008E3020008E17E00080D7F0008CB
:10006000397F0008657F0008917F0008E3020008DF
:10007000E3020008E3020008E3020008E3020008CC
:10008000E3020008E3020008E3020008E3020008BC
:10009000E3020008E3020008E3020008BD7F000855
:1000A000E3020008E3020008E3020008E30200089C
:1000B000E3020008E3020008E3020008E30200088C
:1000C000E3020008E3020008E3020008E30200087C
:1000D000E3020008E3020008A9800008BD800008D0
:1000E00021800008E3020008E3020008E3020008A0
:1000F000E3020008E3020008E3020008E30200084C
:10010000E302000895800008E5800008E30200088B
:10011000E3020008E3020008E3020008E30200082B
:10012000E3020008E3020008E3020008E30200081B
:10013000E3020008E3020008E3020008E30200080B
:10014000E3020008E3020008E3020008E3020008FB
:10015000E3020008E3020008E3020008E3020008EB
:10016000E3020008E3020008E3020008E3020008DB
:10017000E3020008D97B0008E3020008E30200085C
:10018000E3020008E3020008D1800008E30200084F
:10019000E3020008E3020008E3020008E3020008AB
:1001A000E3020008E3020008E3020008E30200089B
:1001B000E3020008E3020008E3020008E30200088B
:1001C000E3020008E3020008E3020008E30200087B
:1001D000E3020008C57B0008E3020008E302000810
:1001E000E3020008E3020008E3020008E30200085B
:1001F000E3020008E3020008E3020008E30200084B
:10020000E3020008E3020008E3020008E30200083A
:10021000E3020008E3020008E3020008E30200082A
:10022000E3020008E3020008E3020008E30200081A
:10023000E3020008E3020008E3020008E30200080A
:10024000E3020008E3020008E3020008E3020008FA
:10025000E3020008E3020008E3020008E3020008EA
:10026000E3020008E3020008E3020008E3020008DA
:10027000E3020008E3020008E3020008E3020008CA
:10028000E3020008E3020008E3020008E3020008BA
:10029000E3020008E3020008E3020008E3020008AA
:1002A000E3020008E3020008E3020008E30200089A
:1002B000E3020008E3020008E3020008E30200088A
:1002C000E3020008E3020008E3020008E30200087A
:1002D000E3020008E3020008E3020008E30200086A
:1002E00002E000F000F8FEE772B6374880F30888B5
:1002F000364880F3098836483649086040F20000E5
:10030000CCF200004EF63471CEF200010860BFF36B
:100310004F8FBFF36F8F40F20000C0F2F0004EF637
:100320008851CEF200010860BFF34F8FBFF36F8F8B
:100330004FF00000E1EE100A4EF63C71CEF20001E3
:100340000860062080F31488BFF36F8F06F0BAFEB2
:1003500006F0D4F84FF055301F491B4A91423CBF7C
:1003600041F8040BFAE71D49184A91423CBF41F895
:10037000040BFAE71A491B4A1B4B9A423EBF51F83D
:10038000040B42F8040BF8E700201849184A914280
:100390003CBF41F8040BFAE706F0D2FE06F030F954
:1003A000144C154DAC4203DA54F8041B8847F9E7A6
:1003B00000F0C4F9114C124DAC4203DA54F8041B9E
:1003C0008847F9E706F0BABE0006002000220020A8
:1003D0000000000808ED00E00000002000060020FA
:1003E0004896000800220020D8220020D8220020B1
:1003F00020670020E0020008E0020008E002000898
:10040000E00200082DE9F04F2DED108AC1F80CD064
:10041000D0F80CD0BDEC108ABDE8F08F002383F338
:1004200011882846A047002005F05AFEFEE705F097
:1004300099FD00DFFEE7000053B94AB9002908BF63
:1004400000281CBF4FF0FF314FF0FF3000F074B9AF
:10045000ADF1080C6DE904CE00F006F8DDF804E01B
:10046000DDE9022304B070472DE9F047089D0446FA
:100470008E46002B4DD18A42944669D9B2FA82F257
:1004800052B101FA02F3C2F1200120FA01F10CFA93
:1004900002FC41EA030E94404FEA1C48210CBEFBCB
:1004A000F8F61FFA8CF708FB16E341EA034306FB54
:1004B00007F199420AD91CEB030306F1FF3080F0E3
:1004C0001F81994240F21C81023E63445B1AA4B230
:1004D000B3FBF8F008FB103344EA034400FB07F7D2
:1004E000A7420AD91CEB040400F1FF3380F00A8113
:1004F000A74240F207816444023840EA0640E41B08
:1005000000261DB1D4400023C5E900433146BDE8B3
:10051000F0878B4209D9002D00F0EF800026C5E955
:10052000000130463146BDE8F087B3FA83F6002E6D
:100530004AD18B4202D3824200F2F980841A61EBE5
:10054000030301209E46002DE0D0C5E9004EDDE703
:1005500002B9FFDEB2FA82F2002A40F09280A1EBEB
:100560000C014FEA1C471FFA8CFE0126200CB1FB40
:10057000F7F307FB131140EA01410EFB03F0884239
:1005800008D91CEB010103F1FF3802D2884200F2C6
:10059000CB804346091AA4B2B1FBF7F007FB101158
:1005A00044EA01440EFB00FEA64508D91CEB0404F6
:1005B00000F1FF3102D2A64500F2BB800846A4EB51
:1005C0000E0440EA03409CE7C6F12007B34022FA3C
:1005D00007FC4CEA030C20FA07F401FA06F31C436B
:1005E000F9404FEA1C4900FA06F3B1FBF9F8200C78
:1005F0001FFA8CFE09FB181140EA014108FB0EF0BE
:10060000884202FA06F20BD91CEB010108F1FF3A0D
:1006100080F08880884240F28580A8F10208614419
:10062000091AA4B2B1FBF9F009FB101144EA014127
:1006300000FB0EFE8E4508D91CEB010100F1FF34D2
:100640006CD28E456AD90238614440EA0840A0FB6A
:100650000294A1EB0E01A142C846A64656D353D040
:100660005DB1B3EB080261EB0E0101FA07F722FA64
:1006700006F3F1401F43C5E9007100263146BDE88D
:10068000F087C2F12003D8400CFA02FC21FA03F3F0
:10069000914001434FEA1C471FFA8CFEB3FBF7F071
:1006A00007FB10360B0C43EA064300FB0EF69E4296
:1006B00004FA02F408D91CEB030300F1FF382FD22F
:1006C0009E422DD9023863449B1B89B2B3FBF7F6D7
:1006D00007FB163341EA034106FB0EF38B4208D9B0
:1006E0001CEB010106F1FF3816D28B4214D9023EF1
:1006F0006144C91A46EA004638E72E46284605E70F
:100700000646E3E61846F8E64B45A9D2B9EB0208DF
:1007100064EB0C0E0138A3E74646EAE7204694E76F
:100720004046D1E7D0467BE7023B614432E73046A2
:1007300009E76444023842E7704700BF38B500F06B
:10074000D1FB06F0CDFB054606F0B2FC0446E0B94D
:10075000104B9D421BD001339D4241F2883504BFAE
:1007600001240025002006F0C5FB0CB100F07AF84A
:1007700001F02EFB01F0EAF900F01CFD08B100F0D9
:1007800071F8284600F010F9F9E70025EAE7054678
:10079000E8E700BF010007B008B501F0A3F9A0F138
:1007A00020035842584108BD07B541F21203022107
:1007B00001A8ADF8043001F0B3F903B05DF804FB13
:1007C00038B5302383F31188174803680BB105F05F
:1007D0006BFD0023154A4FF47A71134805F05AFD5A
:1007E000002383F31188124C236813B12368013B63
:1007F0002360636813B16368013B63600D4D2B7820
:1008000033B963687BB9022001F05CFA322363607C
:100810002B78032B07D163682BB9022001F052FA21
:100820004FF47A73636038BDD8220020C1070008F6
:10083000F8230020F0220020084B187003280CD861
:10084000DFE800F008050208022001F031BA0220BA
:1008500001F024BA024B00225A607047F0220020B7
:10086000F8230020F8B5494B494A1C461968013164
:1008700000F08A8004339342F8D16268454B9A4273
:1008800040F28280444B9B6803F1006303F5003320
:100890009A4279D2002001F073F90220FFF7CCFFD1
:1008A0003E4B00219A6C99641A6F19671A6FDA6CC3
:1008B000D9645A6F59675A6F1A6D19659A6F99679B
:1008C0009B6F374BD3F8802042F00062C3F8802042
:1008D000D3F8802022F00062C3F88020D3F8802073
:1008E000D3F8802042F00072C3F88020D3F8802033
:1008F00022F00072C3F88020D3F8803072B64FF037
:10090000E023C3F8084DD4E90004BFF34F8FBFF3D1
:100910006F8F244AC2F88410BFF34F8F536923F4BA
:1009200080335361BFF34F8FD2F8803043F6E076C7
:10093000C3F3C905C3F34E335B0103EA060C294632
:100940004CEA81770139C2F87472F9D2203B13F175
:10095000200FF2D1BFF34F8FBFF36F8FBFF34F8FD5
:10096000BFF36F8F536923F4003353610023C2F840
:100970005032BFF34F8FBFF36F8F302383F3118853
:10098000854680F308882047F8BD00BF00000208B4
:1009900020000208FFFF0108002200200045025845
:1009A0000044025800ED00E02DE9F04F93B0B44B45
:1009B0002022FF2100900AA89D6801F0B3F9B14AF6
:1009C0001378A3B90121B04811700360302383F379
:1009D000118803680BB105F067FC0023AB4A4FF4A4
:1009E0007A71A94805F056FC002383F31188009B17
:1009F00013B1A74B009A1A60A64A1378032B03D0B1
:100A000000231370A24A53604FF0000A009CD346A3
:100A10005646D146012001F04BF924B19C4B1B688E
:100A2000002B00F02682002001F05CF80390039B6D
:100A3000002BF2DB012001F031F9039B213B1F2B3E
:100A4000E8D801A252F823F0C90A0008F10A000808
:100A5000850B0008150A0008150A0008150A000889
:100A6000170C0008E70D0008010D0008630D0008D1
:100A70008B0D0008B10D0008150A0008C30D000811
:100A8000150A0008350E0008690B0008150A000851
:100A9000790E0008D50A0008690B0008150A00083D
:100AA000630D0008150A0008150A0008150A000859
:100AB000150A0008150A0008150A0008150A00089A
:100AC000150A0008850B00080220FFF765FE0028C4
:100AD00040F0F981009B022105A8BAF1000F08BF80
:100AE0001C4641F21233ADF8143001F019F891E7C9
:100AF0004FF47A7000F0F6FF071EEBDB0220FFF7E1
:100B00004BFE0028E6D0013F052F00F2DE81DFE832
:100B100007F0030A0D1013360523042105A80593D9
:100B200000F0FEFF17E004215548F9E704215A4878
:100B3000F6E704215948F3E74FF01C08404608F156
:100B4000040801F01FF80421059005A800F0E8FF53
:100B5000B8F12C0FF2D101204FF0000900FA07F78D
:100B600047EA0B0B5FFA8BFB01F028F926B10BF07B
:100B70000B030B2B08BF0024FFF716FE4AE70421E6
:100B80004748CDE7002EA5D00BF00B030B2BA1D1CE
:100B90000220FFF701FE074600289BD00120002617
:100BA00000F0EEFF0220FFF747FE1FFA86F84046EE
:100BB00000F0F6FF0446B0B1039940460136A1F1BA
:100BC00040025142514100F0FBFF0028EDD1BA46EE
:100BD000044641F21213022105A83E46ADF8143036
:100BE00000F09EFF16E725460120FFF725FE244B67
:100BF0009B68AB4207D9284600F0C4FF013040F0A3
:100C000067810435F3E70025224BBA463E461D7046
:100C10001F4B5D60A8E7002E3FF45CAF0BF00B03A9
:100C20000B2B7FF457AF0220FFF706FE322000F0B7
:100C300059FFB0F10008FFF64DAF18F003077FF43D
:100C400049AF0F4A08EB0503926893423FF642AF63
:100C5000B8F5807F3FF73EAF124BB845019323DDD7
:100C60004FF47A7000F03EFF0390039A002AFFF6DB
:100C700031AF039A0137019B03F8012BEDE700BF69
:100C800000220020F4230020D8220020C107000801
:100C9000F8230020F0220020042200200822002057
:100CA0000C220020F4220020C820FFF775FD074623
:100CB00000283FF40FAF1F2D11D8C5F120020AAB59
:100CC00025F0030084494245184428BF424601925A
:100CD00001F002F8019AFF217F4801F023F84FEA62
:100CE000A803C8F387027C492846019301F022F843
:100CF000064600283FF46DAF019B05EB830533E703
:100D00000220FFF749FD00283FF4E4AE00F076FF33
:100D100000283FF4DFAE0027B846704B9B68BB420B
:100D200018D91F2F11D80A9B01330ED027F00303C7
:100D300012AA134453F8203C05934046042205A907
:100D4000043701F0A5F88046E7E7384600F01AFFBF
:100D50000590F2E7CDF81480042105A800F0E0FE2C
:100D600002E70023642104A8049300F0CFFE0028CA
:100D70007FF4B0AE0220FFF70FFD00283FF4AAAECB
:100D8000049800F031FF0590E6E70023642104A8F1
:100D9000049300F0BBFE00287FF49CAE0220FFF716
:100DA000FBFC00283FF496AE049800F01FFFEAE732
:100DB0000220FFF7F1FC00283FF48CAE00F02EFF7C
:100DC000E1E70220FFF7E8FC00283FF483AE05A925
:100DD000142000F029FF07460421049004A800F025
:100DE0009FFE3946B9E7322000F07CFE071EFFF671
:100DF00071AEBB077FF46EAE384A07EB0903926809
:100E000093423FF667AE0220FFF7C6FC00283FF48E
:100E100061AE27F003074F44B9453FF4A5AE4846FD
:100E200009F1040900F0AEFE0421059005A800F0C8
:100E300077FEF1E74FF47A70FFF7AEFC00283FF43D
:100E400049AE00F0DBFE002844D00A9B01330BD0F2
:100E500008220AA9002000F06DFF00283AD02022C5
:100E6000FF210AA800F05EFFFFF79EFC1C4805F07A
:100E70003DF913B0BDE8F08F002E3FF42BAE0BF020
:100E80000B030B2B7FF426AE0023642105A80593EA
:100E900000F03CFE074600287FF41CAE0220FFF75E
:100EA0007BFC804600283FF415AEFFF77DFC41F245
:100EB000883005F01BF9059800F0C8FF46463C460F
:100EC00000F07CFFA6E506464EE64FF0000901E67D
:100ED000BA467EE637467CE6F42200200022002057
:100EE000A0860100704700007047000070470000B6
:100EF000704700002DE9F04100F5803704461646A2
:100F00003B7C5BB9C0681030204400F0E5FEE5682A
:100F10003544B5F5004FE56002D816B1BDE8F08163
:100F2000DEB905F07F0605F110000021C6F180064C
:100F30002044F6B232462E4400F0F4FEA06804F1DC
:100F40001008324600F10060414600F5003005F01F
:100F50008FFD30B901233B74E0E74FF4004635467E
:100F6000ECE7A26805F11001404632442144A2603A
:100F7000E268521BE26000F0AFFE0220BDE8F041E3
:100F800000F0A0BE183000F0E9BC000010B5044627
:100F900007F0FAFD204610BD10B5044607F0F4FD39
:100FA000204610BDC3B280B2A3F14102052A02D887
:100FB000373800B27047613B052B94BF5738303843
:100FC000F7E70000F8B504461546084603220C4929
:100FD00000F08CFE014688B908346F1C15F9110029
:100FE000FFF7E0FF064617F911000131FFF7DAFFBE
:100FF000102940EA061004F8010BEFD1F8BD00BF3C
:10100000008D00082DE9F04FADF53F7D07464168A2
:1010100001222AA802F030FE002840F08780064610
:10102000824681461125DFF80C81DFF80CB101AB57
:101030004FF4805241462AA802F07EFF002875D165
:10104000019AB2F5805F71D8002A65D00446019AF2
:101050009442ECD2282D0FD008DC132D2DD01E2D5C
:1010600039D0112D13D00134A4B2F0E7322D2DD098
:10107000372D2FD02D2DF6D13B68121B08EB040124
:1010800038461B692D259847BDF80440EBE7121B35
:10109000022A09D9594608EB040000F027FE18B9C6
:1010A00002342825A4B2DEE718F804303A2B3DD0EC
:1010B0000A2B1CBFA1461325D5E718F804300A2BCC
:1010C00034D03A2B04BFA2463225CCE718F80430BE
:1010D000202BC8D0264618F804300A2B1AD1AAEBC8
:1010E000090208EB090102A811254F2A28BF4F2247
:1010F00007F0F2FDA21B08EB060116A84F2A28BF35
:101100004F2207F0E9FD3B6816AA02A9DB683846C2
:101110009847A8E71E25A6E73B68384604491B699F
:10112000984701200DF53F7DBDE8F08F0020F9E7DD
:10113000028E000800240020048D000800F1180130
:1011400010B5044686B00846019100F0F1FB204638
:10115000FFF758FF60B1019902A800F049FC102286
:1011600004F1080102A807F033FDB0FA80F040094D
:1011700006B010BD70B504460025EEB2304600F052
:101180000FFD58B100213046013500F019FD08B9B6
:10119000002070BD022000F095FDEEE72046FFF72D
:1011A00031FF0028F4D004F58034207C80F0010069
:1011B000EFE70000F0B5C9B005F0AAFE00F096FE1A
:1011C00018B90025284649B0F0BD69462A4802F002
:1011D00075FF00284BD1294C204602F09FFF28487C
:1011E00002F09CFF274802F099FF2146224803F0B5
:1011F00011F80028E5D1702007F0C8FC064610B1B0
:10120000214B44600360336830469B68984705462D
:1012100000282ED01A4F1948394602F0FBFF054628
:101220000028CED1194807F0B1FC044638B1184B5C
:101230004760036000F58033C0E902551D742368E0
:1012400020469B689847054628B10E490C4802F095
:10125000E1FF0028B5D1336830465B6898471CB180
:10126000236820465B68984700F028FEAAE700251F
:10127000FAE70446EFE700BF088D0008188D000864
:101280002F8D0008458D0008688D000814000100AE
:10129000848D00082DE9F04FD44A8DB00B68D0F84A
:1012A00004A001931A440368D14E1A44D1F81C904B
:1012B000DFF8B4C3DFF8B4B3D0E90234634003EA23
:1012C0000A03634013444A6802920AEB7363029C68
:1012D000C84A2244C468224484688AEA04051D403E
:1012E000654015448A68039203EB3555039CC24A56
:1012F0002244846822448AEA03042C4084EA0A04D3
:101300001444CA6805EBF4340492164483EA0502D7
:10131000224056445A4032440E69059604EBB222EC
:10132000059FB64E3E441E4485EA040313406B40BD
:1013300033444E69069602EB7363069FB04E3E44FB
:101340002E4484EA02051D40654035448E690796A7
:1013500003EB3555079FAB4E3E44264482EA030417
:101360002C4054403444A84E4E4405EBF43416440B
:1013700083EA050222405A4032440E6A089604EB82
:10138000B222089FA14E3E441E4485EA0403134046
:101390006B4033444E6A099602EB7363099F9C4E7F
:1013A000D1F830E03E44D1F83880F3442E4484EA4A
:1013B00002051D40654035448E6AA6F5244703EBBF
:1013C00035550A964F3F274482EA03042C40544087
:1013D0003C44CF6A0B9705EBF4340B9E8D4F37449A
:1013E000029E174483EA050222405A403A448A4F3B
:1013F000774404EBB2221F4485EA040313406B4098
:101400003B444F6BBC4402EB7363654484EA020CBB
:101410000CEA030C8CEA040C6544DFF854C2C444A3
:1014200003EB3555A44482EA03042C405440644441
:10143000D1F83CC0794905EBF4346144114483EAA6
:10144000050222405A400A44754904EBB222314455
:10145000079E194484EA02032B4063400B44714900
:1014600002EBF36331440B9E0D4482EA03012140F9
:10147000514029446C4D03EBF1513544019E254404
:1014800083EA010414405C402C44684D01EBB444F1
:101490003544069E154481EA04021A404A402A4413
:1014A000634D04EB323235440A9E1D4484EA020344
:1014B0000B4063402B445F4D02EBF3633544059EC4
:1014C0000D4482EA03012140514029445A4D03EB67
:1014D000F1516544254483EA010414405C402C44E6
:1014E000564D01EBB4443544099E154481EA04028B
:1014F0001A404A402A44524D04EB32323544049E8D
:101500001D4484EA02030B4063402B444D4D02EB23
:10151000F36345440D4482EA0301214051402944CC
:10152000494D03EBF1513544089E2C4483EA0105F3
:1015300015405D402C44454D01EBB4443544039EB9
:101540002A4481EA04051D404D402A44404D04EBE5
:1015500032323D442B4484EA020593440D406540F9
:101560002B443C4D02EBF3633544069E294482EA4A
:101570000305254055402944374D03EBF1514D44B7
:101580002C4483EA010515405D40254401EBB54537
:1015900081EA050404EA03024A405A44A6F5B82B3E
:1015A000089E05EB3232ABF2BE6B54405B442344E1
:1015B0002A4C344402EB33730B9E0C4485EA02013F
:1015C00059402144264C344403EB7151029E25447A
:1015D00082EA03044C402544224C444401EB354547
:1015E000144483EA01026A40224443E078A46AD7A3
:1015F000EECEBDC156B7C7E8DB702024AF0F7CF537
:101600002AC68747134630A8019546FDD8988069B9
:10161000AFF7448BBED75C892211906B2108B44987
:1016200062251EF640B340C0515A5E26AAC7B6E9ED
:101630005D102FD65314440281E6A1D8C8FBD3E72E
:10164000E6CDE121D60737C3870DD5F4ED145A4511
:1016500005E9E3A9F8A3EFFCD9026F6781F671876A
:1016600022619D6D0C38E5FD937198FD8A4C2A8DA1
:101670008E4379A6934C344405EB7222059E1C449C
:1016800081EA0503534023448F4C344402EB337307
:101690000A9E0C4485EA0201594021448B4C4C447B
:1016A00003EB7151254482EA03044C402C44884DDD
:1016B000354401EB3444019E154483EA0102624043
:1016C0002A44844D3D4404EB72221D4481EA040304
:1016D00053402B44804D354402EB3373049E294420
:1016E00084EA02055D4029447C4D354403EB715189
:1016F000079E254482EA03044C402C44784D35442F
:1017000001EB3444099E2A4483EA010565401544EF
:10171000744A324404EB7525039E134481EA0402A3
:101720006A401A44704B734405EB32720B4484EAEE
:101730000501514019446D4B634402EB71511C4447
:1017400085EA02034B401C44694B334401EB3444AB
:10175000019E1D4482EA010363402B44654D04EB66
:1017600073233544069E154463EA010262402A440D
:10177000614D03EBB2624D4462EA040929445F4DB6
:1017800089EA0309454449442C445D4D02EBB151BB
:101790003544049E61EA03081D4488EA0208444473
:1017A00001EB744464EA02034B402B44554D04EBB7
:1017B000F323754463EA010E15448EEA040E0EEB22
:1017C0000502514D03EBB262354462EA040E29442E
:1017D0000A9D8EEA030EA5F580164C4D7144A6F6BF
:1017E000833602EBB151264461EA03045440344489
:1017F000029E01EB7444354464EA02061D444E40E7
:101800007319089E424D04EBF323354463EA010645
:101810001544664072193F4D03EBB262654462EABB
:10182000040629443C4D5E403144079E02EBB15111
:10183000354461EA03062C44384D56403D44344457
:10184000059E1D4401EB744464EA02034B402B44A3
:10185000334D04EBF32335440B9E154463EA010238
:1018600062402A442F4D03EBB2623544039E0D447F
:1018700062EA0401594029442B4D02EBB151354431
:101880002A4E254461EA030454402C44099D01EB8F
:1018900074442E4464EA02051E4485EA01039D193E
:1018A00003681A440AEB040303EBF5230260436068
:1018B00083681C44C36819448460C1600DB0BDE8EE
:1018C000F08F00BF44EABEA4A9CFDE4B604BBBF64D
:1018D00070BCBFBEC67E9B28FA27A1EA8530EFD434
:1018E000051D880439D0D4D9E599DBE6F87CA21F20
:1018F0006556ACC4442229F497FF2A43A72394AB2E
:1019000039A093FCC3595B6592CC0C8FD15D848563
:101910004F7EA86FE0E62CFE144301A3A111084EF0
:10192000827E53F735F23ABDBBD2D72A91D386EBEC
:10193000094B036003F18833436003F12943A3F5A6
:101940009613A3F68B638360A3F18833C3600023EF
:10195000C0E90433704700BF012345672DE9F84310
:101960001446026905460E46E300C2F3C50800F1BD
:1019700018079B18036122BF43690133436112F4C6
:10198000FC7F436903EB5473436114D0C8F14009F1
:1019900007EB08004C4504D22246BDE8F84307F0A7
:1019A00027B9403C4A464E4407F022F944443946A0
:1019B0002846FFF76FFCA04606EB0409B8F13F0F7D
:1019C000A9EB08010AD94022384607F011F9394637
:1019D0002846A8F14008FFF75DFCEFE7A1096FF08A
:1019E0003F02384602FB014206EB8111D5E70000B9
:1019F00070B50B6901F1180506460C46C3F3C50323
:101A0000EA18501C8022EA54C3F13F02072A1FD86B
:101A1000002100F087F929462046FFF73BFC3822D9
:101A20000021284600F07EF92369294620462365D7
:101A300063696365FFF72EFC21461022304607F0EC
:101A4000D7F8204658220021BDE8704000F06AB95E
:101A5000C3F137020021E5E72DE9F84F4FF47A731F
:101A600006460D46002402FB03F7DFF85080DFF83E
:101A7000509098F900305FFA84FA5A1C01D0A342C2
:101A800010D159F824002A4631460368D3F820B013
:101A90003B46D847854205D1074B012083F800A07B
:101AA000BDE8F88F0134042CE3D14FF4FA7004F050
:101AB0001DFB0020F4E700BF44340020102200206A
:101AC0001422002070B504464FF47A76412C254646
:101AD00028BF412506FB05F004F008FB641BF5D187
:101AE00070BD0000002307B5024601210DF107007B
:101AF0008DF80730FFF7B0FF20B19DF8070003B065
:101B00005DF804FB4FF0FF30F9E700000A460421BE
:101B100008B5FFF7A1FF80F00100C0B2404208BD48
:101B2000074B0A4630B41978064B53F8214001465A
:101B300023682046DD69044BAC4630BC604700BFDB
:101B40004434002014220020A086010070B50A4E03
:101B500000240A4D04F030FF308028683388834227
:101B600008D904F025FF2B6804440133B4F5003F85
:101B70002B60F2D370BD00BF46340020003400203B
:101B800004F0E8BF00F1006000F500300068704725
:101B900000F10060920000F5003004F069BF000021
:101BA000054B1A68054B1B889B1A834202D91044C7
:101BB00004F0FEBE002070470034002046340020B0
:101BC00038B50446074D29B128682044BDE838409F
:101BD00004F006BF2868204404F0F0FE0028F3D08B
:101BE00038BD00BF003400200020704700F1FF50D6
:101BF00000F58F10D0F8000870470000064991F8F2
:101C0000243033B100230822086A81F82430FFF71A
:101C1000BFBF0120704700BF04340020014B18688B
:101C2000704700BF0010005C194B013803220844C4
:101C300070B51D68174BC5F30B042D0C1E88A6420A
:101C40000BD15C680A46013C824213460FD214F95C
:101C5000016F4EB102F8016BF6E7013A03F1080398
:101C6000ECD181420B4602D22C2203F8012B042432
:101C7000094A1688AE4204D1984284BF967803F888
:101C8000016B013C02F10402F3D1581A70BD00BF90
:101C90000010005C24220020C48D0008022803D11B
:101CA000024B4FF080529A61704700BF00100258FB
:101CB000022803D1024B4FF480529A61704700BF53
:101CC00000100258022804D1024A536983F4805359
:101CD0005361704700100258002310B5934203D09F
:101CE000CC5CC4540133F9E710BD0000013810B5D5
:101CF00010F9013F3BB191F900409C4203D11AB168
:101D00000131013AF4E71AB191F90020981A10BD97
:101D10001046FCE703460246D01A12F9011B0029BF
:101D2000FAD1704702440346934202D003F8011BE4
:101D3000FAE770472DE9F8431F4D144607468846D9
:101D400095F8242052BBDFF870909CB395F82430AE
:101D50002BB92022FF2148462F62FFF7E3FF95F8B9
:101D600024004146C0F1080205EB8000A24228BFD2
:101D70002246D6B29200FFF7AFFF95F82430A41B9D
:101D800017441E449044E4B2F6B2082E85F824604D
:101D9000DBD1FFF733FF0028D7D108E02B6A03EB34
:101DA00082038342CFD0FFF729FF0028CBD1002048
:101DB000BDE8F8830120FBE704340020024B1A78C9
:101DC000024B1A70704700BF4434002010220020DC
:101DD000F8B5194C194803F077FC2146174803F071
:101DE0009FFC24684FF47A70154ED4F89020154D5E
:101DF000D2F80438114F43F00203C2F80438FFF759
:101E000061FE2046104903F099FDD4F89020042487
:101E1000D2F8043823F00203C2F804384FF4E13357
:101E2000336055F8040BB84202D0314603F0AAFBE8
:101E3000013CF6D1F8BD00BFC4940008F048002072
:101E40002C34002014220020CC9400080C4B70B5D8
:101E50000C4D04461E780C4B55F826209A420DD0A6
:101E60000A4B002118221846FFF75CFF0460014668
:101E700055F82600BDE8704003F084BB70BD00BF7C
:101E80004434002014220020F04800202C3400208C
:101E900030B50A44084D91420DD011F8013B58402D
:101EA000082340F30004013B2C4013F0FF0384EAB5
:101EB0005000F6D1EFE730BD2083B8ED10B5084CE7
:101EC00001220849002001F0B3FE23783BB1064807
:101ED00003F0D0FA044803F003FB0023237010BD85
:101EE00048340020D48D0008A43600201D482DE978
:101EF000F041036D2BB901224FF48051503005F0B1
:101F000049F8194E33780BB1FFF7D8FF0324174F68
:101F10004FF00008134D15492846C7F8048003F018
:101F2000D1FA284603F00AF948B1013C284603F0EB
:101F3000D7FA14F0FF04EED1204634700FE00C49BC
:101F400001220C4801F074FE014618B1284603F046
:101F500091FAEAE7084800F011F801203070BDE876
:101F6000F08100BFA4360020483400203C2200202D
:101F7000D48D00084C340020D88D00080FB4002008
:101F800004B070470068704703460068596870479E
:101F90000B0A017043700B0C090E8370C1707047FF
:101FA000110A027003714170110C120E8170C2701F
:101FB0001A0A42711A0C1B0E8271C371704700001D
:101FC000C36A0239023B8B4283BF4389006C01FB29
:101FD0000300002070470000C2F307238A76CB7607
:101FE0000378032B01BF120C0A75120A4A75704759
:101FF00000F10B010022D30143EA520310F8012B38
:1020000052FA83F38842DAB2F5D1104670470000E5
:1020100010B5417804460020013102464901022AE8
:1020200016BFA35C032203EBC03302F101021EBF03
:102030009BB203EB500398B29142F0D810BD000060
:1020400002684AB1134613F8011B1F290DD93A291A
:10205000F9D1911C8B4202D04FF0FF3070471278BB
:10206000302AF9D1036000207047014B187870477F
:102070009836002038B50D46044618B909200023CB
:102080002B6038BD0368002BF8D01A78002AF5D0F1
:102090008188DA889142F1D1587804F0B3F910F0D0
:1020A0000100EBD12368EBE738B50D4640F2523121
:1020B000144602F0B9F9FF2807D9012C0BD9030AFD
:1020C000022468702B70204638BD30B1002CFAD045
:1020D00001242870F7E70024F5E70446F3E7000041
:1020E0002DE9F8430026D0F8008005460C468E7690
:1020F000836B002B4AD098F80030042B4BD1334629
:102100003546402720E0B7F5187F80F0C480F906F7
:1021100006F1010608BF0237D05B02372BB900F584
:10212000205292B2B2F5006F0DD305F11A01C5F13C
:10213000FF0240EA03402144FFF7B6FF002800F009
:10214000AA80054400200346D8F8102092F82310F6
:10215000B142D8D8002B40F09E80002D00F09B802B
:1021600000232544AB766373D8F81020137903F06D
:102170003701DB0621730BD402F13800FFF704FFAF
:10218000C4E9000193896381D3892381BDE8F88381
:1021900000200146F4E7C36C01335ED1EA6B0023F3
:1021A0002E26551E184615F8011F013020290CD087
:1021B000052908BFE521092804D10B2B9EBFE7188C
:1021C00001337E73E718013379730B28EBD1E118E3
:1021D00000204873A17E00294BD1002B40D06FF026
:1021E0000C0604F10D000825361B331810F8011BEE
:1021F000002938D02E298BB24AD0A3F141011929E8
:1022000003D8117B0D4200D020330373EDE7B9F101
:10221000000F05D100F520539BB2B3F5006F0BD32F
:1022200007F11A01C7F1FF0240EA09402144FFF714
:102230003BFF48B10744002002368146D8F80C30F5
:10224000985B0028E3D13846B9F1000F4FF0000247
:1022500018BF002023189A76A0E7B1463746EDE76D
:102260003F23A3760123234400219976137B03B9EE
:102270006373D37A02F11C0003F03F03237300233E
:10228000FFF780FE20606360D38A6381138B7CE755
:1022900010250B46B9E73F230125A37660E7000030
:1022A00038B50546002435F8020B08B9204638BD7C
:1022B00002F0EEF86308C2B203EBC43312FA83F300
:1022C0009AB2C0F3072303EB520303EBC2339CB271
:1022D000E9E7000037B5C37804461BB90025284656
:1022E00003B030BD00F14C01826C012340780191B4
:1022F00004F0AEF8054680B9A36BE070A06C226BC9
:10230000C31A9342EAD2A3780199022BE6D1024480
:102310000123607804F09CF8E1E70125DFE7000085
:1023200038B5836C05460C468B4210D0FFF7D2FFC0
:1023300060B92246012305F14C01687804F064F885
:1023400000281CBF4FF0FF340120AC6438BD0020D2
:10235000FCE7000038B500230446C3704FF0FF339C
:102360008364FFF7DDFF00284BD1B4F84A524AF6E8
:1023700055239D4207D10B22254904F14C0006F05C
:1023800027FC00283FD094F84C30EB2B03D01833B7
:10239000DBB2012B2ED84AF655239D4206D10822E6
:1023A0001C4904F19E0006F013FC48B3B4F8573002
:1023B000B3F5007F1ED194F85930DBB15A1E1A4292
:1023C00018D1B4F85A30ABB194F85C30013B012B12
:1023D00010D8B4F85D306BB1B4F85F307F2B06D8FD
:1023E00004F16C00FFF7CEFDB0F5803F02D3B4F8E6
:1023F000623053B94AF6552085420CBF02200320B3
:1024000038BD0420FCE70120FAE70020F8E700BF10
:10241000048E0008108E000802392DE9F04701F003
:1024200007044FF0010A466C05460AFA04F4174601
:10243000984606EB1136C1F3C809E4B23146284686
:102440000136FFF76DFF18B10120BDE8F08799460E
:1024500005EB090292F84C30234214BF0121002100
:10246000414513D06340013F82F84C3085F803A00A
:10247000EBD0640014F0FF04EAD109F10103012458
:102480004FF00009B3F5007FE1D1D7E70220DCE788
:1024900001290246F8B50C4640F28C800668F36AC2
:1024A0008B4240F287803378013B032B00F282801D
:1024B000DFE803F00229384B04EB5405B16B3046DA
:1024C00001EB5521FFF72CFF10B14FF0FF30F8BDA5
:1024D0006F1CC5F30805B16B3046354401EB57213D
:1024E00095F84C50FFF71CFF0028EED1C7F3080702
:1024F000E3073E4496F84C0045EA00204CBF000933
:10250000C0F30B00E3E7B16B304601EB1421FFF79A
:1025100007FF0028D9D1640004F4FF742644B6F8FC
:102520004C00D4E7B16B304601EBD411FFF7F8FE55
:102530000028CAD1A40006F14C0004F4FE74204423
:10254000FFF720FD20F07040C1E7D0E90430D579D5
:1025500053EA000101D0916801B95DBB9168022D79
:10256000A4EB01010DD1013B728940F1FF305B0A00
:1025700043EAC053B3FBF2F399421BD81CD0601C52
:10258000A5E7032D02D193698B42F8D8D3699BB993
:10259000B16B304601EBD411FFF7C2FE002894D195
:1025A000A0004C3600F4FE703044FFF7EBFC20F046
:1025B00000408CE701208AE76FF0004087E70000C9
:1025C000F8B5066804460D463378042B0CBF4FF06F
:1025D00080524FF400128A4201D80220F8BDCA0688
:1025E000FBD182680163D2B9022B13D83389B3EBD4
:1025F000551FF2D9F36BA363A36B6263002BECD07E
:1026000003EB55234C36C5F308050020A36335447E
:10261000E563E3E7F36BC271002BE7D01A467789D5
:102620007F02BD42114604D23046FFF7C9FCA063C9
:10263000E2E72046FFF72CFF431C024606D00128A4
:10264000CBD9F36A8342C8D9ED1BEAE70120C5E77D
:1026500001292DE9F04706460C46174608D9C36AFA
:102660008B4205D90378022B62D003D8012B22D0EC
:10267000022552E0033B012BFAD8816B01EBD41108
:10268000FFF74EFE0546002847D1A40006F14C0393
:1026900004F4FE741C443378042B07D0204627F042
:1026A0007047FFF76FFC00F0704007433946204643
:1026B000FFF76EFC2FE001EB5108816B01EB582115
:1026C000FFF72EFE054640BB14F0010406F14C094D
:1026D00008F1010AC8F3080808BFFBB230461FBF63
:1026E00019F8083003F00F023B0103F0F00318BFA4
:1026F000134309F808300123B16BF37001EB5A2141
:10270000FFF70EFE054640B9CAF3080A44B1C7F305
:10271000071709F80A700123F3702846BDE8F0870F
:1027200019F80A30C7F3032723F00F031F43F0E71C
:10273000816B01EB1421FFF7F3FD05460028ECD176
:10274000640006F14C0304F4FF741F551919C7F314
:1027500007274F70DFE70000F8B504460E4617461E
:10276000E3690BB91846F8BD012BA6EB03052068F9
:1027700014BFAA1C3A46691CFFF76AFF0028F2D171
:10278000E369013BE361EBE701292DE9F8430646E4
:102790000C461746056802D80220BDE8F883EB6AAC
:1027A0008B42F9D97AB9A14621463046A046FFF7B7
:1027B0006FFE0446B0B92B78042B02D1002F43D111
:1027C000F7710020E9E72B78042B02D1C379022BA3
:1027D000E9D04FF0FF3239462846FFF739FF00288D
:1027E000E1D0DAE70128D7D0421C01D10120D4E79B
:1027F0002B78042B19D1EA6AAB69023A93421CD3B5
:1028000008F10102A2420CD02B78042B08D100233E
:10281000A2EB090249462846FFF7FEFD0028BCD17D
:10282000A146EB6AA342BFD8C5E70022414628462D
:10283000FFF70EFF0028DED0AFE70133AB612B7945
:1028400043F001032B71DBE7F3798BB9B468BC4229
:1028500002D10223F371B4E721463046FFF718FE98
:10286000012899D9431CC1D001348442EFD0A8E794
:10287000032BA6D1B368BB42A3D8B2691344BB42B1
:102880009FD3E6E770B5C3790446032B06D1816870
:102890008369CD18A94203D10023E371002070BDE4
:1028A0004E1C20683246FFF7D3FE0028F7D1314690
:1028B000F0E700002DE9F74305460191FFF70AFD17
:1028C0000446002849D105F14C09019928464FF4E6
:1028D0000072FFF775FB2146A86407464846FFF7DC
:1028E00021FA6C896402B4F5004F28BF4FF400440C
:1028F000B4F5007F2FD9204604F00CFA804630B1A1
:1029000022460021640A0026FFF70CFA09E0640859
:10291000EEE72346BA194146687803F099FD18B9E5
:1029200026446B899E42F4D3404604F003FA68893A
:10293000801B18BF012003B0BDE8F08301366B890E
:102940009E42F4D20123BA194946687803F080FD0B
:102950000028F3D0EBE70026F1E70120EBE70000C9
:10296000F8B50446FFF7B6FC0546002842D12378A7
:10297000032B37D12779012F34D104F14C060146BE
:102980004FF400723046FFF7CDF9552341227221F2
:1029900084F84A32AA2304F50D7084F84F2084F895
:1029A0004B32522384F8301284F84C3084F84D3086
:1029B000612384F8311284F84E3084F83332A169EF
:1029C00084F83222FFF7E4FA616904F50E70FFF72C
:1029D000DFFA626B3B46314601326078A26403F055
:1029E00037FD257100226078114603F055FD00384F
:1029F00018BF0120F8BD000000232DE9F0430B6053
:102A000085B00F461546FFF71BFB061EC0F2B281CC
:102A1000804B53F82640002C00F0AE813C6005F05E
:102A2000FE0523786BB1607803F0ECFCC70708D48F
:102A30001DB110F0040500D00A25284605B0BDE8F8
:102A4000F0830023F0B22370607003F0C7FCC1076D
:102A500000F194810DB14207EED400212046FFF72A
:102A600079FC022840F099806E4604F2122304F2A9
:102A70005221324618461033FFF784FA42F8040B0D
:102A80008B42F7D1002556F8041B00297DD0204643
:102A9000FFF760FC012879D80128A26C40F0C080C3
:102AA00004F1570304F18C0113F8015B002D7BD175
:102AB0008B42F9D1B4F8B430B3F5807F74D194F877
:102AC000B830092B70D104F19400FFF75DFA4FF094
:102AD000FF33171841F10001BB4275EB010363D3CB
:102AE00004F1A000FFF74EFA94F8BA302063012BEE
:102AF000A37059D194F8B99003FA09F91FFA89F330
:102B00006381002B50D0444B04F1A800FFF73AFA40
:102B10000646984248D8831C626304F1A400E3622D
:102B2000FFF730FA00EB020804F19C00C4F8408083
:102B3000FFF728FA10441FFA89F2A06306FB02F39C
:102B400013EB080345EB05029F4271EB02032BD305
:102B50002E4604F1AC00FFF715FAE06365B963890E
:102B6000B34221D9E16B2046FFF72AFA81192046AA
:102B7000FFF7D6FB98B90136631993F84C30812BD7
:102B800014D02035C5F30805E8E703200135042DEE
:102B90007FF479AF042807D101E0042801D1012591
:102BA0004BE701287FF678AF0D2546E705F11400C5
:102BB00004F14C063044FFF7E5F901280546F3D946
:102BC000E36A8342F0D96189821E236C02FB0133E0
:102BD0006364A16B204601EBD511FFF7A1FB002830
:102BE000DDD105F07F0006EB8000FFF7CBF9431C39
:102BF00003D00135A842ECD0D6E70425C4E905008E
:102C0000064A257000251388E56101339BB21380C5
:102C1000E38012E79C360020FDFFFF7FA0360020F6
:102C2000B4F85730B3F5007FBED1B4F8626026B96E
:102C300004F17000FFF7A6F9064694F85C302663AD
:102C4000591EA3700129AFD894F859506581002D01
:102C5000AAD0691E2942A7D1B4F85D8018F00F0FE1
:102C6000A4F80880A0D1B4F85F0018B904F16C0092
:102C7000FFF788F9B4F85A10002995D006FB03FE37
:102C800001EB181CF44460458ED3A0EB0C00A84265
:102C9000B0FBF5F388D33E48834285D84FF6F570F4
:102CA00083426DD903259F1C114402EB0C03032DB5
:102CB000E7626263A16323644CD1B4F8763053EACF
:102CC00008037FF471AFBB0004F17800FFF75AF9F5
:102CD000E06303F2FF13B6EB532FFFF465AF4FF041
:102CE000FF33032DC4E905334FF08003237187D1EF
:102CF000B4F87C30012B83D1511C2046FFF710FB28
:102D000000287FF47DAFB4F84A224AF6552320719B
:102D10009A427FF475AF1F4B04F14C00FFF732F974
:102D200098427FF46DAF03F1FF5304F50C70FFF789
:102D300029F903F50053203398427FF461AF04F57D
:102D40000D70FFF71FF9A06104F50E70FFF71AF977
:102D5000606155E7B8F1000F3FF426AF7144022DD2
:102D60004FEA4703E1631EBFD91907F0010303EBE4
:102D70005103AEE70B2560E60C255EE603255CE615
:102D800040F6F575AB428CBF022501258BE700BFED
:102D9000F5FFFF0F525261412DE9F84F07460568D4
:102DA000884649B96E69C6B1EB6AB34298BF01263D
:102DB000AB69A3B9002405E0FFF76AFB01280446CC
:102DC00003D801242046BDE8F88F421C00F0D280D1
:102DD000EB6A8342F6D84646EAE70126E8E72A7816
:102DE000EB6A042A40F08380A6F1020A023B4FF00E
:102DF000010B9A4528BF4FF0000AD146696C28465E
:102E000001EB1931FFF78CFA00283BD109F00703D9
:102E1000EA6AC9F3C8010BFA03F3901EDBB26A1821
:102E20004C4609F1010992F84C20814502EA03025F
:102E300033BF5B0000234FF40071DBB228BF99461B
:102E4000B2B90234631E0333BCD80123214628469D
:102E50001A46FFF7E1FA0228B3D0012800F08A8071
:102E6000B8F1000F13D10223FB710028A9D130E083
:102E7000CA450AD0002BD2D10131B1F5007FBDD2B5
:102E80000123CCE74FF0FF34DCE70024DAE7FB79DD
:102E9000022B07D1731CA342E7D0BB68F31ABB61B6
:102EA0000323FB7108F10102FB69A24205D113B1B2
:102EB0000133FB61D9E70223FBE70BB90123FB6177
:102EC000224641463846FFF747FC00284FD10123F0
:102ED000FB61EA6AAB69023A6C6193429CBF03F101
:102EE000FF33AB612B7943F001032B716AE7464551
:102EF00014D1741C3846A34298BF02242146FFF720
:102F0000C7FA01283FF45DAF431C33D0E0B16B69D1
:102F1000012B03D9EA6A934238BF1E463446013476
:102F2000EB6AA34203D8012E7FF644AF0224214668
:102F30003846FFF7ADFA48B101283FF442AF0130FF
:102F400018D0B442EBD135E7002CE7D04FF0FF3278
:102F500021462846FFF77CFB48B9B8F1000FB8D0EE
:102F6000224641462846FFF773FB0028B1D00128CE
:102F70007FF427AF4FF0FF3424E700002DE9F8433A
:102F800006680446076B894633782037042B0CBF4C
:102F90004FF080534FF40013BB429CBF0023836368
:102FA000836B73B1C7F30808B8F1000F3CD101334C
:102FB000416B836339B93389B3EB571F34D800238E
:102FC000A36304200AE07389013B13EA57232BD142
:102FD000FFF75EFA0128054602D80220BDE8F88313
:102FE000421C01D10120F9E7F36A834216D8B9F1F6
:102FF000000FE4D0616B2046FFF7CEFE0546C8B156
:103000000128EAD0431CEDD001463046FFF752FCC0
:103010000028E7D1E37943F00403E3712946304601
:103020006563FEF7CDFFA0634C360020276346445E
:10303000E663D3E70720D1E7F8B50E460021044642
:103040000768FFF7BDFA98B90546A16B3846FFF748
:1030500067F968B93A78E36B042A1B780CD11B0630
:103060000ED5054601212046FFF788FF0028ECD049
:10307000042808BF072006E0E52B01D0002BF0D183
:103080000135B542EED1F8BDC16C4B1C2DE9F041C4
:1030900004460568066B1FD1E5274FF00108A16BB8
:1030A0002846FFF73DF998B92A78E36B042A09BF4F
:1030B0001A781F7002F07F021A7085F80380236B64
:1030C000B3420DD200212046FFF758FF0028E6D07A
:1030D000042808BF022003E0FFF772FA0028DBD0C3
:1030E000BDE8F0812DE9F04105460068A96B06694D
:1030F000FFF716F9044620B9EB6B1A78852A03D03E
:1031000002242046BDE8F081324603F1200153F845
:10311000040B8B4242F8040BF9D1777801377F0119
:10312000A7F16003B3F5007FEAD800212846FFF736
:1031300025FF04280446E3D00028E2D1A96B2868C3
:10314000FFF7EEF804460028DBD1EB6B1A78C02AB3
:10315000D6D106F1200203F1200153F8040B8B4273
:1031600042F8040BF9D196F823300F222C33B3FB2D
:10317000F2F3B7EB431FC3D34FF0400800212846BA
:10318000FFF7FCFE04280446BAD00028B9D1A96B89
:103190002868FFF7C5F804460028B2D1EB6B1A780F
:1031A000C12AADD1B8F5187F09D206EB080203F1A8
:1031B000200153F8040B8B4242F8040BF9D108F1BB
:1031C00020084745DAD8B8F5187F9AD83046FEF778
:1031D0001FFF7388834294D092E700000B6800229F
:1031E00010B5036004460B6A83604B6AC261C37109
:1031F00023F0FF03896AC0E90432C164FFF7E0F9F4
:1032000020B92046BDE81040FFF76CBF10BD00009C
:10321000F8B50368054601271C692046FEF7F8FE4D
:10322000A070000A6678E0702846E96CFFF7C8F9DC
:1032300020B1022828BF0220C0B2F8BDA96B2868BF
:10324000FFF76EF80028F4D1EB6B04F1200254F87C
:10325000041B944243F8041BF9D12B68DF70002E45
:10326000E7D000212846013EFFF788FEE0E7000096
:103270002DE9F8434FF0FF08064607680424454649
:103280004FF6FF79B16B11B9002C73D063E038466B
:10329000FFF746F8044600285DD1F06B0378002B59
:1032A0006ED03A78042A11D1852B4DD1336B30463C
:1032B000F364FFF717FF044600284CD13B691B79E4
:1032C00003F03F03B3712046BDE8F883C27AE52BD3
:1032D00002F03F02B27143D02E2B41D022F02001E8
:1032E00008293DD00F2A40D1590637D503F0BF0534
:1032F000336B90F80D80F364437B434530D1428BB0
:1033000072BB03780D21FC6823F04003DFF874E002
:10331000013B4B4301211EF801CB30F80CC009B32F
:10332000FF2B1DD824F813C06146013301320D2A4A
:10333000F1D10278520605D521B1FF2B10D8002219
:1033400024F81320013DEDB200213046FFF716FEB0
:103350000446002896D00023B363B4E7AB42CBD039
:10336000FF25F1E7CC45E1D0FAE72DB9FEF740FEA5
:10337000404501D10024A6E74FF0FF33F364A2E7F4
:103380000424E8E7AC8E00082DE9F04F002187B057
:103390000446D0F80090FFF713F9804670B999F809
:1033A0000030042B33D1D9F80C00FEF779FF074623
:1033B0002046FFF75DFF054620B18046404607B036
:1033C000BDE8F08FD9F810309A8CBA42F0D193F85A
:1033D00023B040265D4506D1D9F80C3033F81530BE
:1033E000002BE5D1EAE7F106D9F8103008BF023624
:1033F000985B01F04DF8D9F80C30824633F815008F
:1034000001F046F88245D3D102360135E2E74FF0AC
:10341000FF0A4FF0FF3B5546C4F84CB0A16B48463D
:10342000FEF77EFF00285CD1E66B3778002F77D05F
:10343000F27AE52F02F03F03A37103D0120704D5FF
:103440000F2B04D0C4F84CB04FE00F2B54D194F89C
:103450004B3058063FD4790645D5236B07F0BF079C
:1034600096F80DA0E364737B53453ED1738B002B1C
:103470003BD135780121D9F80C3005F03F05019397
:103480000D23013D5D43284B13F8012BB25A71B354
:10349000FF2D059329D81046049200F0F9FF6B1C0C
:1034A00003900293019B33F8150000F0F1FF03999C
:1034B00081421AD1049A029D1146059B1B4A9342F0
:1034C000E2D133785A0604D519B1019B33F815308F
:1034D0005BB97D1EEDB200212046FFF74FFD0028AD
:1034E0009CD080466AE7BD42BDD0FF25F3E74FF68A
:1034F000FF708242E2D0F8E72DB93046FEF778FD42
:1035000050453FF45BAF94F84B30DB079AD40B2265
:1035100004F14001304605F05BFB002892D14DE7F5
:103520004FF004084AE700BFAC8E0008B98E0008CF
:103530002DE9F04F90F84BB099B004461BF0A00570
:1035400040F068810668F26832F81530002B4AD1E5
:103550003378042B40F087800F230E352046B5FBCF
:10356000F3F5A91CFFF768FD8146002877D1236B8E
:103570000135A3EB4515E3795A07E56435D523F00A
:1035800004032046E371FFF77DF950BB4FF0FF3293
:10359000616B2046FFF7E0F818BBA3682BB3214608
:1035A00004A8FFF71BFEE0B970894FF40071D4E95D
:1035B0000423E0FB01233069C4E904233830FEF71B
:1035C000EFFC3069D4E904232830FEF7E9FCE37905
:1035D000326904A843F0010382F82130FFF718FE96
:1035E00018B181463BE00135AEE7D6E903544022ED
:1035F00000212046FEF796FB8523012140222370FF
:10360000C0234FF0C10C04EB010884F820300023E4
:103610001E469E46571C04F802C0F0B2023204F85F
:1036200007E021B135F8131009B10133DBB20F0AFD
:10363000A15408F802700232D706F2D135F813709F
:103640000136002FE6D184F82330831C28466370AE
:10365000FEF726FE84F82400000A84F82500484678
:1036600019B0BDE8F08F04F140070DF1100A1BF00E
:10367000010F97E807008AE8070000F0D380402395
:103680004FF0010884F84B30BC46F368B8F1050FE1
:103690009AE80700ACE803002CF8022B4FEA12422C
:1036A0008CF8002059D9981E424630F8021F002994
:1036B00042D10DF10F0C072102F00F0E91461209B5
:1036C0000EF13000392888BF0EF1370001390CF8AF
:1036D000010902D0B9F10F0FEED818AB7E205A18AD
:1036E00002F8580C38460022914206D010F801CB5F
:1036F00002F1010EBCF1200F31D104F13F0C07297A
:1037000002F1010297BF18AB20205818013198BF71
:1037100010F8580C072A0CF80200F0D92046FFF7E1
:1037200033FE8146002878D108F10108B8F1640F12
:10373000AAD14FF0070992E74FF0100C01F0010EEB
:1037400049080EEB4202D30344BF82F4883282F070
:103750002102BCF1010CF1D1A7E74246A9E772466C
:10376000C2E7216B2046A1EB4511FEF729FF8146F8
:1037700000287FF474AF4FF6FF783846FEF738FC28
:103780000190A16B3046FEF7CBFD814600287FF407
:1037900066AFE36BE9B2019A4FF00D0CD6F80CE07E
:1037A0005A734FF00F02DFF8E0A0DA724A1E187366
:1037B0000CFB02F284469876D87640451AF8019BB5
:1037C0000CF1010C18BF3EF8120003EB090B18BFF7
:1037D000013203F809004FEA1029002808BF4046CB
:1037E000BCF10D0F8BF80190E7D1404502D03EF8B7
:1037F00012200AB941F0400119700123002120462E
:10380000F370FFF7BBFB814600287FF428AF013D32
:10381000B7D11BE04FF0060921E704287FF41FAF62
:1038200084F84BB01BF0020F20461BBF0C350D2156
:103830000125B5FBF1F518BF01352946FFF7FCFB63
:10384000814600287FF40BAF013D8AD1A16B304641
:10385000FEF766FD814600287FF401AF0146202275
:10386000E06BFEF75FFAE36B03CF18605960BA783C
:1038700039889A72198194F84B30E26B03F018037F
:1038800013730123F370EAE6AC8E000810B504460A
:103890000A463430FEF776FB886004F13800FEF704
:1038A00073FBC2E9040194F8213003F00203D371E1
:1038B0000023D36110BD000003284B8B04BF8A8A0C
:1038C00043EA0243184670472DE9F04F0B7899B050
:1038D000044689462F2BD0F800B001D05C2B09D1CB
:1038E0004A461378914601322F2BFAD05C2BF8D040
:1038F000002301E0DBF81C30A3600023E3619BF8A8
:103900000030042B1ED1A368E3B1DBF82030214640
:1039100004A82362DBF824306362DBF82830A3625A
:10392000FFF75CFC0346002854D1DBF8102002F1BD
:103930003800FEF727FBC4E9040392F8213003F0B6
:103940000203E37199F800301F2B00F235818023C8
:103950000021204684F84B3019B0BDE8F04FFEF747
:103960002FBE49460B78894601312F2BFAD05C2BAC
:10397000F8D01F2B8CBF00250425012F2FD11388D1
:103980002E2B31D1002322F8173004F140029F4240
:103990008CBF2E21202101330B2B02F8011BF6D105
:1039A00045F02005204684F84B50FFF7EDFC94F8D5
:1039B0004B30002800F0E78004280BD1990603F073
:1039C000040240F1DC80002A00F0F6808023002011
:1039D00084F84B3019B0BDE8F08F0425CDE7022FF5
:1039E00002D153882E2BCAD0911E87BB002322F808
:1039F0001730002F00F0118132F8130019460133FF
:103A00002028F9D009B92E2801D145F00305901ED0
:103A100030F817302E2B01D0013FF9D14FF0203371
:103A20004FF0000A6364D0462364C4F8473008238B
:103A3000481C32F811600090F6B1202E03D02E2ED3
:103A40000DD1B84210D045F003050099F0E731F8E8
:103A50001730202B01D02E2BC8D1013FC5E79A4546
:103A600005D20099B9423BD10B2B30D101E00B2B91
:103A700027D145F003050B2394F84020E52A04BF25
:103A8000052284F84020082B04BF4FEA88085FFA1B
:103A900088F808F00C030C2B03D008F00303032B69
:103AA00001D145F00205A8073FF57CAF18F0010FE2
:103AB00018BF45F0100518F0040F18BF45F00805B1
:103AC00070E70099B94202D045F00305D4D84FEA17
:103AD00088080B234FF0080A00975FFA88F8B4E7CC
:103AE0007F2E15D9304640F25231CDE9022345F000
:103AF0000203019300F098FC10F0800F0646DDE908
:103B0000022316D000F07F0646498E5D019D46B324
:103B100031464548CDE9012305F0C8F8DDE9012328
:103B2000F8B9A6F1410189B219291ED848F0020856
:103B300010E0FF28EAD9591E8A4503D345F0030552
:103B40009A4682E704EB0A01000A0AF1010A019D84
:103B500081F8400004EB0A010AF1010A81F8406093
:103B600073E745F003055F26F4E7A6F1610189B22A
:103B700019299EBF203E48F00108B6B2EAE7002AA4
:103B800008BF052026E75A073FF524AFA379DB06D7
:103B900045D59BF80000042835D1A3682146E27979
:103BA00023622369DBF8100023F0FF0313436362F1
:103BB000E36CA362FFF76AFE23680027DA6819F84E
:103BC000010B00283FF409AF40F25231009200F09F
:103BD0004BFC054608B31F28009A7FF6FEAE2F283F
:103BE0003FF4BFAE5C283FF4BCAE7F2805D8014649
:103BF0000E4805F05BF8009A78B9FF2F0DD022F837
:103C000017500137DBE7216B0BF14C03C1F30801BF
:103C10001944FFF751FEA060CEE70620DAE6052042
:103C2000D8E600BF2C8E0008258E00081C8E0008E8
:103C30001FB5CDE9001003A814460391FEF700FA62
:103C4000002815DB0B4A52F820300BB10021197007
:103C5000019B0BB10021197042F820302CB10022D9
:103C600001A96846FEF7C8FE0446204604B010BD10
:103C70000B24FAE79C3600202DE9F04798B09046D7
:103C800005460191002800F0528102F03F0603A989
:103C900001A83246FEF7B0FE002840F04681039BA3
:103CA0004FF48C60049303F035F80746002800F0C9
:103CB0004081039B00F500720199D86004A81A6145
:103CC000FFF702FE044620B99DF95B30002BB8BF18
:103CD000062418F01C0F00F0CD80002C4CD0042CD2
:103CE00040D104A8FFF724FC044600283AD146F04E
:103CF0000806039B1A78042A40F083801869294635
:103D00002B60FFF7C3FD039B1E22002118690230C0
:103D1000FEF708F8039C00211A2220692630FEF7DE
:103D200001F8236920221A71246903F011F8014671
:103D3000012208342046FEF72BF9039B04A81B69D7
:103D400083F82120FFF764FA044658B9A96801B343
:103D500002462846FEF718FDAB68039A0446013B6D
:103D60005361B4B1384602F0E5FF0CB100232B607B
:103D7000204618B0BDE8F0879DF8163013F0110FFB
:103D800040F0848018F0040F40F0C98018F0080F4C
:103D9000AFD1039A31071399936C48BF46F04006A0
:103DA000E964AB641078042872D1069B9DF8171063
:103DB0002B62089B106923F0FF030B4329466B62BB
:103DC000179BAB62FFF762FDDDF80CA00024002218
:103DD00005F15008BAF8063021464046C5F800A063
:103DE000AB80002385F8306085F831406C64C5E90C
:103DF0000E234FF40072FDF795FFB20653D4002452
:103E0000B0E702F0A5FF0146009013980E30FEF7D0
:103E1000BFF8139800991630FEF7BAF8039C13996F
:103E20002078FFF749FD202300228046CB722046F0
:103E30001399FEF7D1F8139B002201211A775A77C4
:103E40009A77DA77039BD970B8F1000FA1D0414679
:103E500004A8D3F84890FEF797FC0446002881D1C7
:103E600049460398FEF75CFA039B044608F1FF30CD
:103E7000586176E7002C7FF475AF9DF81630DC06AC
:103E80004FD418F0020F84D0D80782D5072469E7F1
:103E9000FFF712FD0023A86001F11C00FEF772F885
:103EA0006B61286190E7D5E9046956EA0903A6D059
:103EB000BAF80AA0A9684FEA4A2AC5E90E69B245CC
:103EC00074EB09031BD300242964002C7FF44AAF50
:103ED000C6F30803002B92D0039C2046FEF770F82F
:103EE00008B3760A0123414646EAC95682196A6434
:103EF000607802F089FA041E18BF012432E72846D0
:103F0000FEF7C6FAB6EB0A06014669F10009012878
:103F100003D9431CD3D10124D6E70224D4E70824D3
:103F200020E704241EE702241CE704461EE70924B8
:103F30001EE711241CE700002DE9F04F994685B0DB
:103F40000023884603A90446C9F800301646FEF748
:103F500091F8054680BB94F831506DBB94F8303031
:103F600013F00103009300F0A68004F1500AD4E995
:103F70000432D4E90E011B1A62EB0102B34272F162
:103F8000000238BF1E46BEB1D4E90E10C1F30803CB
:103F9000002B40F08280039B5A894B0A013A43EA86
:103FA000C0531A401BD151EA000309D1A06801286F
:103FB0000DD8022584F83150284605B0BDE8F08FB1
:103FC000216C20460192FEF763FA019AEFE7431C49
:103FD00004D10123009D84F83130EDE72064DDF841
:103FE0000CB0216C5846FDF7EBFF0028E1D0B6F588
:103FF000007F02EB000731D3BBF80A1002EB56201A
:10400000730A88429BF8010088BF8B1A3A464146E2
:10401000019302F0F9F90028DBD194F93020019BDB
:10402000002A0BDA606CC01B984207D24FF4007272
:10403000514608EB4020FDF74FFE019B5F02D9F887
:104040000030F61BB8443B44C9F80030D4E90E32C6
:10405000DB1942F10002C4E90E3294E7626CBA4205
:104060001AD094F93030002B0DDA012351469BF819
:10407000010002F0EDF90028ABD194F8303003F0E4
:104080007F0384F83030039801233A465146407844
:1040900002F0BAF900289CD16764A16B4046C1F3D5
:1040A0000801C1F500775144B74228BF37463A4668
:1040B000FDF712FEC3E707257EE7000070B596B056
:1040C0000E460022019002A901A8FEF795FC0446C5
:1040D000E0B94FF48C6002F01DFE0546D8B1029B9A
:1040E00000F500720199D86002A81A61FFF7ECFB95
:1040F000044640B99DF95330002B0ADB1EB131460E
:1041000002A8FDF7EDFF284602F014FE204616B087
:1041100070BD0624F7E71124F8E7000070B5B8B0C9
:104120000222019003A901A8FEF766FC044608BB21
:10413000039B4FF48C60109302F0ECFD05460028C1
:1041400066D0039B00F500720199D86010A81A612F
:10415000FFF7BAFB044650B99DF88B30980655D44A
:10416000190653D49DF84630DA0706D507242846A9
:1041700002F0E0FD204638B070BD039B0493187830
:10418000042814D104A91869FFF780FB069E9DF846
:104190004630DB0610D410A8FEF776FF0446002850
:1041A000E5D156BB0398FEF7DBFB0446DFE71F991A
:1041B000FFF782FB0646EAE7039BDA69B242D5D0F5
:1041C00024930021269624A81B78042B01BFDDE947
:1041D0000823CDE928239DF817308DF89730FEF796
:1041E000EFF904460028C2D124A8FFF741F804469D
:1041F0000028BBD00428BAD1CDE70246314604A836
:10420000FEF7C2FA04460028B1D1CBE70624AEE798
:104210001124AFE7F0B5BDB0CDE900106846FDF759
:104220000FFF022203A901A8FEF7E6FB04460028BF
:1042300041D1039B4FF48C60149302F06BFD054653
:10424000002800F0EE80039B00F5007214AE019987
:10425000D8601A613046FFF737FB044640BB9DF833
:104260009B3013F0A00F40F0D880039B009F1A787A
:10427000042A68D11B6904AC03F1400C18680833A8
:1042800053F8041C2246634503C21446F6D150225B
:10429000314628A8FDF720FD394628A8FFF714FB72
:1042A000044600284CD12A9A169B9A4206D008242C
:1042B000284602F03FFD20463DB0F0BD349A209BD9
:1042C0009A42F4D128A8FFF733F904460028EFD129
:1042D000039B04AF1B6993F801E093F823C09C8C07
:1042E0003A46083303CAB24243F8080C43F8041CA8
:1042F0001746F5D1039B28A81B6983F801E0039BAF
:104300001A6982F823C01A6982F82440240A82F8C4
:1043100025401A691379D9065CBF43F02003137155
:10432000FEF776FF04460028C2D13046FEF7ACFE09
:1043300004460028BCD10398FEF712FB0446B7E7F9
:104340000428B5D1BEE7239A04AB02F1200C106813
:10435000083252F8041C1C46624503C42346F6D1B9
:104360005022314628A8FDF7B7FC394628A8FFF7A8
:10437000ABFA044600284CD12A9A169B9A4296D151
:10438000349A209B9A4292D128A8FFF7D1F804468C
:1043900000288DD137990DF11D030DF12D0001F18C
:1043A0000D0253F8044B834242F8044BF9D11888AC
:1043B000012710809B7893709DF81B30039CDA06D0
:1043C00058BF43F02003CB72E770CB7ADB06ACD545
:1043D000169A2A9B9A42A8D02078FFF76DFA0146D8
:1043E0002046FDF7EDFD0146C8B12046FDF798FFD8
:1043F000044600287FF45CAF039890F86D302E2BB4
:1044000093D12A9A00F16C01FDF7E6FD039BDF7062
:104410008BE704287FF44CAFB6E7062448E7022474
:1044200046E7112447E700007F2810B501D880B285
:1044300010BDB0F5803F13D240F2523399420FD1F4
:104440000849002231F8024B93B2844203D103F1B0
:104450008000C0B2ECE70132802AF3D11346F6E7C0
:104460000020E5E76C9100087F280DD940F2523317
:10447000994208D1FF2806D800F10040034B80384C
:1044800033F8100070470020704700BF6C9100089F
:10449000B0F5803FF0B522D21F4A83B21F49B0F574
:1044A000805F28BF0A46141D34F8042C2146AAB1A7
:1044B000934213D334F8025C2E0AEFB252FA85F518
:1044C000A84222DA082E09D8DFE806F0050A101201
:1044D0001416181A1C00801A34F810301846F0BD53
:1044E000981A00F001001B1A9BB2F7E7103BFBE79C
:1044F000203BF9E7303BF7E71A3BF5E70833F3E7F2
:10450000503BF1E7A3F5E353EEE70434002ECBD1A3
:1045100001EB4702C7E700BFBC8E0008B09000085F
:10452000084BC26A994228BF1946836C50688B4277
:1045300010B506D95A1E4C0002EB4103B3FBF4F34D
:10454000184410BD20BCBE0001F001038A0748BF1B
:1045500043F002034A0748BF43F008030A0748BF75
:1045600043F00403CA0648BF43F010038A06426BB7
:1045700048BF43F0200313434363704710B5074C13
:10458000204600F093FF064B0022C4E91023054BA0
:10459000A364054BE363054BE36410BDA436002020
:1045A0000070005200B4C404F8360020F83800202F
:1045B000C36A0BB90E4BC3620379012B0CD10D4BAF
:1045C000984209D10C4B5A6B42F480325A63DA6D2F
:1045D00042F48032DA65DB6D436C00221A65DA62E0
:1045E0001A605A605A624FF0FF329A63704700BFF8
:1045F0006C920008A4360020004502580379012B74
:1046000016D0436C00221A65DA621A605A605A6248
:104610004FF0FF329A63074B984209D1064B5A6B11
:1046200022F480325A63DA6D22F48032DA65DB6D6F
:10463000704700BFA43600200045025810B5446CF6
:104640000649FFF76DFF6060236842F2107043F087
:1046500003032360BDE8104001F048BD801A060046
:104660000129F8B5466C0B4F09D175680A493D40E0
:10467000FFF756FF054345F480557560F8BD746833
:1046800006493C40FFF74CFF044344F480547460F7
:10469000F4E700BF00ECFFFF80F0FA0240787D01F4
:1046A000436C00225A601A6070470000426C012976
:1046B000536823F4404304D0022905D001B9536064
:1046C000704743F48043FAE743F40043F7E7000000
:1046D000436C41F480519A60D9605A6B1206FCD544
:1046E00080229A637047000010B541F48851446CF1
:1046F000A260E160616B11F04502FBD0A26311F092
:10470000040203D0FFF720FF012010BD61691046AD
:104710001960FAE710B541F48851446CA260E16079
:10472000616B11F04502FBD0A26311F0050203D0CA
:10473000FFF70AFF012010BD616910461960FAE712
:1047400073B5134604460E46302282F31188426C3C
:10475000D26B32B14FF0FF314030019301F0D2FC07
:10476000019B606C00220265C263C262456B15F456
:10477000807504D185F31188012002B070BD4FF01F
:10478000FF31816382F31188012E06D90C21204666
:1047900002B0BDE87040FFF7BDBF1046EDE7000076
:1047A00073B5446C0E4600250192616BA1632565CB
:1047B000E562FFF7C9FE012E07D9019B2A460C21AD
:1047C00002B0BDE87040FFF7A5BF02B070BD0000A9
:1047D00010B541F49851446CA260E160616B11F036
:1047E0004502FBD0A26311F03F0203D0FFF7ACFEFD
:1047F000012010BD216A10461960E1695960A16964
:1048000099606169D960F4E72DE9F74304460191A5
:10481000006D01A91746984602F0D4FB0646002811
:104820004AD0626C2046DDF804905568C5F309054E
:1048300001356B00A56CB5FBF3F54FF47A73B5FB4E
:10484000F3F55D43556200F0F7FD50BB636C4FF02C
:10485000FF3201254146C3F8589020461D659A63F2
:104860004FF49572DA6342F207029F62DA62E36CF8
:104870000A9AFFF74FFFA0B9E26C104B11680B408A
:104880007BB929462046FFF75BFF054648B92E460F
:104890003A460199206D02F0BDFB304603B0BDE8F9
:1048A000F0833A460199206D02F0B4FBE26C0121DD
:1048B0002046FFF775FFF0E70126EEE708E0FFFD71
:1048C0002DE9F7431F46436C01924FF47A725D68FD
:1048D00004468846C5F3090501356E00856CB5FBB5
:1048E000F6F5B5FBF2F555435D6200F0A5FD20B18C
:1048F0000125284603B0BDE8F0837E0201A9206DA2
:10490000324602F05FFB05460028F1D0636C019A45
:10491000D4F84C909A6501221A654FF0FF329A63E1
:104920004FF49572DA639E62236BDB064B4658BFE9
:104930004FEA4828012F42461BD912212046FFF793
:10494000E9FEC0B9D9F80020104B13409BB9636C45
:1049500042F2930239462046DA62E26CFFF7F0FE3B
:10496000804640B932460199206D454602F052FB1F
:10497000BFE71121E2E732460199206D02F04AFBC0
:10498000E26C39462046FFF70BFFB2E708E0FFFD77
:104990002DE9F3411F46436C01924FF47A725D6832
:1049A00004468846C5F3090501356E00856CB5FBE4
:1049B000F6F5B5FBF2F555435D6200F03DFD20B123
:1049C0000125284602B0BDE8F0817E0201A9206DD4
:1049D000324602F02DFB05460028F1D0636C019AA7
:1049E0009A6501221A654FF0FF329A634FF48D7277
:1049F000DA639E62236BE66CDB06334658BF4FEAF0
:104A00004828012F424619D919212046FFF782FE76
:104A1000B0B932680F4B134093B9636C42F2910204
:104A200039462046DA62E26CFFF78AFE064638B95C
:104A300001993546206D02F027FBC2E71821E4E713
:104A40000199206D02F020FBE26C39462046FFF709
:104A5000A7FEB6E708E0FFFD12F0030F2DE9F041D5
:104A600007460C4615461E4617D00E44B44202D1E6
:104A70000020BDE8F0810123FA6B21463846FFF79C
:104A80001FFF0028F5D128464FF40072F96B05F599
:104A900000750134FDF720F9E8E7BDE8F041FFF7C4
:104AA0000FBF000012F0030F2DE9F04107460C463E
:104AB00015461E4617D00E44B44202D10020BDE870
:104AC000F08129464FF40072F86B05F50075FDF78B
:104AD00003F90123FA6B21463846FFF759FF0028F6
:104AE000EDD10134E8E7BDE8F041FFF751BF000028
:104AF00000207047302310B583F311880024436CE5
:104B000040302146DC6301F00BFB84F3118810BDBB
:104B1000026843681143016003B118477047000001
:104B2000024A136843F0C00313607047004400401A
:104B3000024A136843F0C003136070470048004006
:104B4000024A136843F0C0031360704700780040C6
:104B5000044B9A6C02439A641A6F104318671B6FD8
:104B6000704700BF0045025837B5274C274D2046F7
:104B700000F0FCFC04F11400009400234FF40072D8
:104B8000234900F097F94FF40072224904F13800EC
:104B90000094214B00F010FA204BC4E91735204C4B
:104BA000204600F0E3FC04F11400009400234FF4CD
:104BB00000721C4900F07EF94FF400721A4904F1AA
:104BC00038000094194B00F0F7F9194BC4E9173578
:104BD000184C204600F0CAFC04F1140000234FF4E6
:104BE00000721549009400F065F9144B4FF40072FF
:104BF000134904F13800009400F0DEF9114BC4E9C8
:104C0000173503B030BD00BFFC38002000E1F505CA
:104C1000403A002040400020214B00080044004062
:104C200068390020403C002040420020314B000801
:104C300000480040D4390020403E0020414B00088D
:104C4000404400200078004038B5264D0446037CDF
:104C5000002918BF0D46012B06D1234B984230D1B5
:104C60004FF40030FFF774FF2A68236EE16D03EB09
:104C70005203A566B3FBF2F36A68100442BF23F047
:104C8000070003F0070343EA4003CB60AB6843F03F
:104C900040034B60EB6843F001038B6042F4967372
:104CA00043F001030B604FF0FF330B62510505D554
:104CB00012F0102211D0B2F1805F10D084F864306D
:104CC00038BD0A4B984205D0094B9842CCD14FF0E1
:104CD0008040C7E74FF48020C4E77F23EEE73F23FF
:104CE000ECE700BF74920008FC380020683900200F
:104CF000D43900202DE9F047C66D05463768F469C0
:104D0000210734621AD014F0080118BF4FF48071E3
:104D1000E20748BF41F02001A3074FF0300348BF2E
:104D200041F04001600748BF41F0800183F31188E2
:104D3000281DFFF7EDFE002383F31188E2050AD555
:104D4000302383F311884FF48061281DFFF7E0FEC4
:104D5000002383F311884FF030094FF0000A14F05C
:104D6000200838D13B0616D54FF0300905F1380A36
:104D7000200610D589F31188504600F051F900281B
:104D800036DA0821281DFFF7C3FE27F080033360C1
:104D9000002383F31188790614D5620612D53023D7
:104DA00083F31188D5E913239A4208D12B6C33B1D0
:104DB00027F040071021281DFFF7AAFE37600023C7
:104DC00083F31188E30618D5AA6E1369ABB1506955
:104DD000BDE8F047184789F31188736A284695F8AB
:104DE0006410194000F0DCFB8AF31188F469B6E71F
:104DF000B06288F31188F469BAE7BDE8F087000073
:104E0000F8B51546826804460B46AA4200D285686A
:104E1000A1692669761AB5420BD218462A46FCF7D4
:104E20005BFFA3692B44A3612846A3685B1BA360B7
:104E3000F8BD0CD9AF1B18463246FCF74DFF3A4679
:104E4000E1683044FCF748FFE3683B44EBE7184671
:104E50002A46FCF741FFE368E5E7000083689342D8
:104E6000F7B50446154600D28568D4E90460361AC1
:104E7000B5420BD22A46FCF72FFF63692B446361CE
:104E80002846A3685B1BA36003B0F0BD0DD9324672
:104E9000AF1B0191FCF720FF01993A46E0683144CD
:104EA000FCF71AFFE3683B44E9E72A46FCF714FFE6
:104EB000E368E4E710B50A440024C361029B846000
:104EC000C16002610362C0E90000C0E9051110BDC4
:104ED00008B5D0E90532934201D1826882B982686F
:104EE000013282605A1C426119700021D0E90432FB
:104EF0009A4224BFC368436101F02CF9002008BD29
:104F00004FF0FF30FBE7000070B5302304460E463B
:104F100083F31188A568A5B1A368A269013BA360CA
:104F2000531CA36115782269934224BFE368A361EF
:104F3000E3690BB120469847002383F31188284684
:104F400007E03146204601F0F5F80028E2DA85F363
:104F5000118870BD2DE9F74F04460E461746984656
:104F6000D0F81C904FF0300A8AF311884FF0000BF4
:104F7000154665B12A4631462046FFF741FF0346F4
:104F800060B94146204601F0D5F80028F1D0002351
:104F900083F31188781B03B0BDE8F08FB9F1000FDF
:104FA00003D001902046C847019B8BF31188ED1A6E
:104FB0001E448AF31188DCE7C160C361009B8260F4
:104FC0000362C0E905111144C0E9000001617047A6
:104FD000F8B504460D461646302383F31188A768BA
:104FE000A7B1A368013BA36063695A1C62611D708D
:104FF000D4E904329A4224BFE3686361E3690BB1E8
:1050000020469847002080F3118807E0314620466B
:1050100001F090F80028E2DA87F31188F8BD00006B
:10502000D0E9052310B59A4201D182687AB9826825
:105030000021013282605A1C82611C7803699A4205
:1050400024BFC368836101F085F8204610BD4FF08E
:10505000FF30FBE72DE9F74F04460E46174698460A
:10506000D0F81C904FF0300A8AF311884FF0000BF3
:10507000154665B12A4631462046FFF7EFFE034646
:1050800060B94146204601F055F80028F1D00023D0
:1050900083F31188781B03B0BDE8F08FB9F1000FDE
:1050A00003D001902046C847019B8BF31188ED1A6D
:1050B0001E448AF31188DCE70379052B05BF836A58
:1050C000002001204B6004BF4FF400730B60704759
:1050D00070B55D1E866A04460D44B54205D9436B22
:1050E00043F080034363012070BD06250571FFF77F
:1050F000B3FC05232371F7E770B55D1E866A04468D
:105100000D44B54205D9436B43F08003436301204E
:1051100070BD07250571FFF7C5FC05232371F7E76F
:1051200038B505790446052D05D108230371FFF72D
:10513000DFFC257138BD0120FCE700000323F0B53A
:10514000037185B00446FFF779FA00222046114624
:10515000FFF7BEFA4FF4D57203AB08212046FFF7E4
:10516000D9FA0246B8B901232363039BC3F303238F
:10517000012B09D103AB37212046FFF7CBFA18B931
:10518000A44B039A1340ABB120460125FFF788FAE0
:105190000223237137E103AB002237212046FFF7BA
:1051A000B9FA28B99B4A039B1A40002A00F0A7804D
:1051B00002232363236B03F00F03022B40F0A9802B
:1051C0006425954E42F2107000F090FF03AB32461A
:1051D00001212046FFF788FA0028D5D1039B002B38
:1051E00080F293805A0003D5236B43F010032363AE
:1051F000002204F1080302212046FFF7E9FA0246E3
:105200000028C1D104F1380303212046FFF782FAB8
:105210000028B9D104F11805A26B092120462B46BC
:10522000FFF7D6FA0028AFD102ABA26B07212046C8
:10523000FFF770FA06460028A6D1236B03F00F0390
:10524000022B40F08F807E227F21284603F07EF9DA
:10525000012840F28780E76B42F2107000F046FFB1
:1052600008234FF40072394620460096FFF7CCFA27
:10527000002889D1384603F0B7F9236BA06203F008
:105280000F03022B72D103AB644A06212046FFF7BD
:1052900041FA002871D15F49039B1940B1FA81F1AD
:1052A00049092046FFF7DCF902AB4FF400721021E8
:1052B0002046FFF72FFA054600287FF465AF554ECC
:1052C000029B33427FF460AF236B13F00E0F03F0A9
:1052D0000F0273D0022A7FF457AFE36A19780129CD
:1052E00000F09480022900F09380002900F089806A
:1052F0004B4F2046FFF7DAF903AB3A4676E011460A
:1053000020462263FFF7E4F954E7013D7FF45AAFEA
:105310003AE7444D6426444A3E4F012B18BF1546D8
:1053200003AB002237212046FFF7F4F900287FF471
:105330002BAF039B3B427FF427AF03AB2A462921C7
:105340002046FFF7D1F900287FF41EAF039B002B06
:10535000FFF648AF013E3FF417AF42F2107000F085
:10536000C5FEDDE7284603F013F986E77E227F219C
:105370002846E66B03F0EAF808B9002191E700231C
:1053800040223146204600930623FFF73DFA0028CD
:10539000F3D1B3895BBA9B07EFD5244B402231464A
:1053A000204600930623FFF72FFA0028E5D1317C31
:1053B00001F00F010F3918BF012172E7E36A197874
:1053C000F9B101297FF4E0AE2046FFF76FF903AB96
:1053D000A26B37212046FFF79DF900287FF4D4AE59
:1053E000039B33427FF4D0AE03AB0222062120465A
:1053F000FFF790F900287FF4C7AE039B33427FF498
:10540000C3AE05232371284605B0F0BD084F70E7F1
:10541000084F6EE708E0FFFD0080FFC00001B90300
:105420000000B7030080FF5000001080F1FFFF80F4
:105430000001B7030002B70337B504460C4D01ABBA
:10544000A26B0D212046FFF765F978B9019B2B422D
:105450000BD1C3F34323042B08D0053B022B04D804
:105460004FF47A7000F042FEE9E7012003B030BD4E
:1054700008E0FFFD70B53023054683F311880379FA
:105480000024022B03D184F31188204670BD04232D
:10549000037184F311880226FFF7CEFF04462846E5
:1054A000FFF7FEF82E71F0E7FFF768B8044B0360D2
:1054B0000123037100234363C0E90A33704700BF2F
:1054C0008C92000810B53023044683F31188C16222
:1054D000FFF76EF802230020237180F3118810BDBE
:1054E00010B53023044683F31188FFF787F80023B3
:1054F0000122E362227183F3118810BD02684368C0
:105500001143016003B11847704700001430FFF7E2
:1055100021BD00004FF0FF331430FFF71BBD00002A
:105520003830FFF797BD00004FF0FF333830FFF7FA
:1055300091BD00001430FFF7E7BC00004FF0FF31D1
:105540001430FFF7E1BC00003830FFF741BD000028
:105550004FF0FF323830FFF73BBD0000012914BF88
:105560006FF0130000207047FFF7FEBA044B036092
:1055700000234360C0E9023301230374704700BF76
:10558000B092000810B53023044683F31188FFF76A
:105590005BFB02230020237480F3118810BD000000
:1055A00038B5C36904460D461BB904210844FFF70A
:1055B000A5FF294604F11400FFF78AFC002806DA4B
:1055C000201D4FF40061BDE83840FFF797BF38BD9C
:1055D000026843681143016003B118477047000037
:1055E00013B5406B00F58054D4F8A4381A681178CC
:1055F000042914D1017C022911D1197901231289BE
:105600008B4013420BD101A94C3002F0CDFED4F8EF
:10561000A4480246019B2179206800F0DFF902B01E
:1056200010BD0000143002F04FBE00004FF0FF33F9
:10563000143002F049BE00004C3002F021BF0000DF
:105640004FF0FF334C3002F01BBF0000143002F06B
:105650001DBE00004FF0FF31143002F017BE0000F5
:105660004C3002F0EDBE00004FF0FF324C3002F043
:10567000E7BE00000020704710B500F58054D4F854
:10568000A4381A681178042917D1017C022914D191
:105690005979012352898B4013420ED1143002F004
:1056A000AFFD024648B1D4F8A4484FF44073617985
:1056B0002068BDE8104000F07FB910BD406BFFF7D7
:1056C000DBBF0000704700007FB5124B01250426A8
:1056D000044603600023057400F1840243602946F8
:1056E000C0E902330C4B0290143001934FF4407325
:1056F000009602F061FD094B04F69442294604F13C
:105700004C000294CDE900634FF4407302F028FE90
:1057100004B070BDD8920008BD560008E1550008DD
:105720000A68302383F311880B790B3342F8230086
:105730004B79133342F823008B7913B10B3342F8C2
:10574000230000F58053C3F8A4180223037400203B
:1057500080F311887047000038B5037F044613B109
:1057600090F85430ABB90125201D0221FFF730FF1E
:1057700004F114006FF00101257700F0F7FC04F14B
:105780004C0084F854506FF00101BDE8384000F03F
:10579000EDBC38BD10B5012104460430FFF718FFF9
:1057A0000023237784F8543010BD000038B5044638
:1057B0000025143002F018FD04F14C00257702F0AA
:1057C000E7FD201D84F854500121FFF701FF20461A
:1057D000BDE83840FFF750BF90F8803003F0600319
:1057E000202B06D190F881200023212A03D81F2ADC
:1057F00006D800207047222AFBD1C0E91D3303E000
:10580000034A426707228267C3670120704700BFCF
:105810004422002037B500F58055D5F8A4381A6821
:10582000117804291AD1017C022917D11979012391
:1058300012898B40134211D100F14C04204602F032
:1058400067FE58B101A9204602F0AEFDD5F8A44884
:105850000246019B2179206800F0C0F803B030BDFA
:1058600001F10B03F0B550F8236085B004460D46F6
:10587000FEB1302383F3118804EB8507301D082126
:10588000FFF7A6FEFB6806F14C005B691B681BB1C5
:10589000019002F097FD019803A902F085FD0246F0
:1058A00048B1039B2946204600F098F8002383F373
:1058B000118805B0F0BDFB685A691268002AF5D05E
:1058C0001B8A013B1340F1D104F18002EAE700009A
:1058D000133138B550F82140ECB1302383F31188EF
:1058E00004F58053D3F8A4281368527903EB82039C
:1058F000DB689B695D6845B104216018FFF768FEAD
:10590000294604F1140002F085FC2046FFF7B4FE9E
:10591000002383F3118838BD7047000001F0A2BC5A
:1059200001234022002110B5044600F8303BFCF76B
:10593000F9F90023C4E9013310BD000010B530238C
:10594000044683F311882422416000210C30FCF7C7
:10595000E9F9204601F0A8FC02230020237080F31F
:10596000118810BD70B500EB8103054650690E46E5
:105970001446DA6018B110220021FCF7D3F9A069AF
:1059800018B110220021FCF7CDF931462846BDE8B8
:10599000704001F089BD000083682022002103F0DF
:1059A000011310B5044683601030FCF7BBF92046A4
:1059B000BDE8104001F004BEF0B4012500EB810405
:1059C00047898D40E4683D43A469458123600023F5
:1059D000A2606360F0BC01F021BE0000F0B40125BC
:1059E00000EB810407898D40E4683D4364690581CB
:1059F00023600023A2606360F0BC01F097BE00004A
:105A000070B5022300250446242203702946C0F8FD
:105A100088500C3040F8045CFCF784F9204684F888
:105A2000705001F0D5FC63681B6823B129462046FD
:105A3000BDE87040184770BD0378052B10B50446CB
:105A40000AD080F88C300523037043681B680BB1C3
:105A5000042198470023A36010BD000001780529A8
:105A600006D190F88C20436802701B6803B1184778
:105A70007047000070B590F87030044613B10023F1
:105A800080F8703004F18002204601F0BDFD6368AB
:105A90009B68B3B994F8803013F0600535D00021CD
:105AA000204602F0AFF80021204602F09FF863681C
:105AB0001B6813B1062120469847062384F87030EE
:105AC00070BD204698470028E4D0B4F88630A26F15
:105AD0009A4288BFA36794F98030A56F002B4FF0DE
:105AE000300380F20381002D00F0F280092284F857
:105AF000702083F3118800212046D4E91D23FFF78D
:105B00006DFF002383F31188DAE794F8812003F016
:105B10007F0343EA022340F20232934200F0C58041
:105B200021D8B3F5807F48D00DD8012B3FD0022B70
:105B300000F09380002BB2D104F188026267022248
:105B4000A267E367C1E7B3F5817F00F09B80B3F5FF
:105B5000407FA4D194F88230012BA0D1B4F88830D2
:105B600043F0020332E0B3F5006F4DD017D8B3F520
:105B7000A06F31D0A3F5C063012B90D86368204695
:105B800094F882205E6894F88310B4F88430B047AB
:105B9000002884D0436863670368A3671AE0B3F5FD
:105BA000106F36D040F6024293427FF478AF5C4BE0
:105BB00063670223A3670023C3E794F88230012BB5
:105BC0007FF46DAFB4F8883023F00203A4F8883076
:105BD000C4E91D55E56778E7B4F88030B3F5A06FE8
:105BE0000ED194F88230204684F88A3001F04EFCC1
:105BF00063681B6813B10121204698470323237073
:105C00000023C4E91D339CE704F18B036367012380
:105C1000C3E72378042B10D1302383F31188204667
:105C2000FFF7BAFE85F311880321636884F88B506F
:105C300021701B680BB12046984794F88230002BE6
:105C4000DED084F88B300423237063681B68002B3C
:105C5000D6D0022120469847D2E794F884302046D7
:105C60001D0603F00F010AD501F0C0FC012804D085
:105C700002287FF414AF2B4B9AE72B4B98E701F0E7
:105C8000A7FCF3E794F88230002B7FF408AF94F878
:105C9000843013F00F01B3D01A06204602D501F06C
:105CA000C9FFADE701F0BAFFAAE794F88230002BF4
:105CB0007FF4F5AE94F8843013F00F01A0D01B06EA
:105CC000204602D501F09EFF9AE701F08FFF97E78B
:105CD000142284F8702083F311882B462A46294623
:105CE0002046FFF769FE85F31188E9E65DB11522CC
:105CF00084F8702083F3118800212046D4E91D2305
:105D0000FFF75AFEFDE60B2284F8702083F311881A
:105D10002B462A4629462046FFF760FEE3E700BFF0
:105D200008930008009300080493000838B590F821
:105D300070300446002B3ED0063BDAB20F2A34D82E
:105D40000F2B32D8DFE803F03731310822323131FE
:105D50003131313131313737856FB0F886309D427E
:105D600014D2C3681B8AB5FBF3F203FB12556DB95D
:105D7000302383F311882B462A462946FFF72EFE4F
:105D800085F311880A2384F870300EE0142384F818
:105D90007030302383F31188002320461A461946B9
:105DA000FFF70AFE002383F3118838BDC36F03B1E8
:105DB00098470023E7E70021204601F023FF002158
:105DC000204601F013FF63681B6813B106212046CB
:105DD00098470623D7E7000010B590F870300446C6
:105DE000142B29D017D8062B05D001D81BB110BD14
:105DF000093B022BFBD80021204601F003FF0021C4
:105E0000204601F0F3FE63681B6813B106212046AB
:105E10009847062319E0152BE9D10B2380F8703041
:105E2000302383F3118800231A461946FFF7D6FD65
:105E3000002383F31188DAE7C3689B695B68002B52
:105E4000D5D1C36F03B19847002384F87030CEE7F3
:105E50000023826880F8243083691B689968914226
:105E6000FBD25A68036042601060586070470000BF
:105E70000023826880F8243083691B689968914206
:105E8000FBD85A6803604260106058607047000099
:105E900008B50846302383F3118891F82430032B8A
:105EA00005D0042B0DD02BB983F3118808BD8B6A64
:105EB00000221A604FF0FF338362FFF7C9FF00230F
:105EC000F2E7D1E9003213605A60F3E7034610B5F8
:105ED0001B68984203D09C688A689442F8D25A683A
:105EE0000B604A601160596010BD0000FFF7B0BF41
:105EF000064BD96881F824001868026853601A605C
:105F00000122D86080F82420FAF77CBA40460020AD
:105F10000C4B30B5DD684B1C87B004460FD02B46C8
:105F2000094A684600F0B6F92046FFF7E1FF009BFA
:105F300013B1684600F0B8F9A86A07B030BDFFF7A2
:105F4000D7FFF9E740460020915E0008044B1A682D
:105F5000DB6890689B68984294BF002001207047DE
:105F600040460020094B10B51C68D8682268536071
:105F70001A600122DC6084F82420FFF779FF0146D3
:105F80002046BDE81040FAF73DBA00BF4046002069
:105F9000044B1A68DB6892689B689A4201D9FFF744
:105FA000E1BF70474046002038B50123084C00256A
:105FB0002370656002F046FB02F06CFB0549064861
:105FC00002F042FC0223237085F3118838BD00BF24
:105FD000E8480020109300084046002000F09AB9DD
:105FE000EFF3118020B9EFF30583302282F311889B
:105FF0007047000010B530B9EFF30584C4F308040E
:1060000014B180F3118810BDFFF7C2FF84F311882B
:10601000F9E70000034A516853685B1A9842FBD8BD
:10602000704700BF001000E08B604B630023CA6123
:1060300000F128020B6302230A618B84012388612B
:1060400081F8263001F11003C26A4A611360C3620D
:1060500001F12C030846CB6270470000D0E9013102
:10606000026841F8183CA1F19C033839CB60036900
:1060700041F8243C436941F8203C034B41F8043C7F
:10608000C3680248FFF7D0BF1D0400084046002047
:1060900008B5FFF7E3FFBDE80840FFF727BF0000A2
:1060A00038B50E4BDC6804F12C05A062E06AA8420A
:1060B0000FD194F826303BB994F825309B0702BFE6
:1060C000D4E9043213605A600F20BDE83840FFF76E
:1060D0000FBF0368E362FFF709FFE7E740460020D0
:1060E000302383F31188FFF7DBBF000008B50146BA
:1060F000302383F311880820FFF70AFF002383F37E
:10610000118808BD054BDB6821B10360986203204C
:10611000FFF7FEBE4FF0FF30704700BF4046002043
:1061200003682BB10022026018469962FFF7DEBEB9
:1061300070470000064BDB6839B1426818605A604E
:10614000136043600420FFF7E3BE4FF0FF30704759
:10615000404600200368984206D01A6802605060EA
:1061600018469962FFF7C2BE7047000038B5044672
:106170000D462068844200D138BD036823605C600E
:106180008562FFF7B3FEF4E7036810B59C68A2428E
:106190000CD85C688A600B604C602160596099681B
:1061A0008A1A9A604FF0FF33836010BD121B1B6880
:1061B000ECE700000A2938BF0A2170B504460D46F5
:1061C0000A26601902F038FA02F020FA041BA542F0
:1061D00003D8751C04462E46F3E70A2E04D9012085
:1061E000BDE8704002F0F8BB70BD0000F8B5144B7C
:1061F0000D460A2A4FF00A07D96103F110018260A7
:1062000038BF0A224160196914460160486018616C
:10621000A81802F001FA02F0F9F9431B0646A3425E
:1062200006D37C1C28192746354602F005FAF2E70A
:106230000A2F04D90120BDE8F84002F0CDBBF8BD1B
:1062400040460020F8B506460D4602F0DFF90F4A39
:10625000134653F8107F9F4206D12A460146304626
:10626000BDE8F840FFF7C2BFD169BB68441A2C19DA
:1062700028BF2C46A34202D92946FFF79BFF22469E
:1062800031460348BDE8F840FFF77EBF4046002096
:1062900050460020C0E90323002310B45DF8044BEE
:1062A0004361FFF7CFBF000010B5194C2369984236
:1062B0000DD08168D0E9003213605A609A680A44B0
:1062C0009A60002303604FF0FF33A36110BD0268A2
:1062D000234643F8102F53600022026022699A423D
:1062E00003D1BDE8104002F0A1B9936881680B4466
:1062F000936002F08BF92269E1699268441AA24224
:10630000E4D91144BDE81040091AFFF753BF00BF9C
:10631000404600202DE9F047DFF8BC8008F1100767
:106320002C4ED8F8105002F071F9D8F81C40AA6829
:10633000031B9A423ED814444FF00009D5E90032BD
:10634000C8F81C4013605A60C5F80090D8F81030A7
:10635000B34201D102F06AF989F31188D5E903311A
:1063600028469847302383F311886B69002BD8D0D7
:1063700002F04CF96A69A0EB040982464A450DD245
:10638000022002F029FB0022D8F81030B34208D1D5
:1063900051462846BDE8F047FFF728BF121A2244AD
:1063A000F2E712EB09092946384638BF4A46FFF79B
:1063B000EBFEB5E7D8F81030B34208D01444C8F863
:1063C0001C00211AA960BDE8F047FFF7F3BEBDE845
:1063D000F08700BF504600204046002010B560B94D
:1063E000074804790368053C9B6818BF0124984757
:1063F00008B144F00404204610BD0124FBE700BFAF
:10640000A4360020FFF7EABF2DE9F047884617467B
:106410009A460446B0B90D4E3579052D05D00324B2
:106420000DE0013D15F0FF050ED0326853463946A8
:106430003046D2F814904246C8470028F1D1204691
:10644000BDE8F0870424FAE70124F8E7A436002029
:106450002DE9F047884617469A460446B0B90D4ED6
:106460003579052D05D003240DE0013D15F0FF051C
:106470000ED03268534639463046D2F8189042461C
:10648000C8470028F1D12046BDE8F0870424FAE788
:106490000124F8E7A436002037B50C46154670B93C
:1064A00051B101290BD10748694603681B6A984717
:1064B00010B9019B04462B60204603B030BD042474
:1064C000FAE700BFA436002000207047FEE7000076
:1064D000704700004FF0FF30704700004B6843608A
:1064E0008B688360CB68C3600B6943614B6903624F
:1064F0008B6943620B6803607047000008B53A4B34
:1065000040F2FF713948D3F888200A43C3F8882045
:10651000D3F8882022F4FF6222F00702C3F8882013
:10652000D3F88830324B1A6C0A431A649A6E0A43C5
:106530009A66304A9B6E1146FFF7D0FF00F58060E7
:1065400002F11C01FFF7CAFF00F5806002F138017B
:10655000FFF7C4FF00F5806002F15401FFF7BEFFB2
:1065600000F5806002F17001FFF7B8FF00F5806070
:1065700002F18C01FFF7B2FF00F5806002F1A80183
:10658000FFF7ACFF00F5806002F1C401FFF7A6FF42
:1065900000F5806002F1E001FFF7A0FF00F58060E8
:1065A00002F1FC01FFF79AFF02F58C7100F58060A3
:1065B000FFF794FF01F0CEFB0F4BD3F8902242F08F
:1065C0000102C3F89022D3F8942242F00102C3F8EA
:1065D00094220522C3F898204FF06052C3F89C2003
:1065E000064AC3F8A02008BD004402580000025823
:1065F000004502582493000800ED00E01F00080346
:1066000008B501F0C5FDFFF7CFFC0D4BDA6B42F08A
:106610004002DA635A6E22F040025A665B6E094B02
:106620001A6842F008021A601A6842F004021A60FE
:1066300000F032FD00F032FBBDE8084000F0B4B8D5
:10664000004502580018024801207047002070479A
:106650007047000002290CD0032904D00129074803
:1066600018BF00207047032A05D8054800EBC20078
:106670007047044870470020704700BF2895000805
:1066800054220020DC94000870B59AB005460846F4
:10669000144601A900F0C2F801A8FBF73BFB431C1C
:1066A0000022C6B25B001046C5E900342370032304
:1066B000023404F8013C01ABD1B202348E4201D85D
:1066C0001AB070BD13F8011B013204F8010C04F874
:1066D000021CF1E708B5302383F311880348FFF764
:1066E00099F8002383F3118808BD00BFF04800200B
:1066F00090F8803003F01F02012A07D190F8812022
:106700000B2A03D10023C0E91D3315E003F0600319
:10671000202B08D1B0F884302BB990F88120212AA1
:1067200003D81F2A04D8FFF757B8222AEBD0FAE77C
:10673000034A426707228267C3670120704700BF90
:106740004B22002007B5052917D8DFE801F01916FC
:1067500003191920302383F31188104A0121019075
:10676000FFF700F9019802210D4AFFF7FBF80D48E9
:10677000FFF71CF8002383F3118803B05DF804FBD6
:10678000302383F311880748FEF7E6FFF2E7302352
:1067900083F311880348FEF7FDFFEBE77C940008C4
:1067A000A0940008F048002038B50C4D0C4C2A4647
:1067B0000C4904F10800FFF767FF05F1CA0204F174
:1067C00010000949FFF760FF05F5CA7204F11800CF
:1067D0000649BDE83840FFF757BF00BFC861002039
:1067E0005422002058940008629400087194000814
:1067F00070B5044608460D46FBF78CFAC6B2204633
:10680000013403780BB9184670BD32462946FBF7B0
:106810006DFA0028F3D10120F6E700002DE9F047DA
:1068200005460C46FBF776FA2B49C6B22846FFF719
:10683000DFFF08B10736F6B228492846FFF7D8FF30
:1068400008B11036F6B2632E0BD8DFF88C80DFF873
:106850008C90234FDFF894A02E7846B92670BDE8BF
:10686000F08729462046BDE8F04702F02DBA252ED4
:106870002ED1072241462846FBF738FA70B9194B4A
:10688000224603F10C0153F8040B8B4242F8040B2F
:10689000F9D11B8807350E341380DDE708224946FD
:1068A0002846FBF723FA98B9A21C0F4B197802323D
:1068B0000909C95D02F8041C13F8011B01F00F015E
:1068C0005345C95D02F8031CF0D118340835C3E7FD
:1068D000013504F8016BBFE7489500087194000882
:1068E0005F9500085095000800E8F11F0CE8F11FC3
:1068F000BFF34F8F044B1A695107FCD1D3F8102115
:106900005207F8D1704700BF0020005208B50D4B68
:106910001B78ABB9FFF7ECFF0B4BDA68D10704D556
:106920000A4A5A6002F188325A60D3F80C21D20721
:1069300006D5064AC3F8042102F18832C3F80421BF
:1069400008BD00BF266400200020005223016745D7
:1069500008B5114B1B78F3B9104B1A69510703D5D1
:10696000DA6842F04002DA60D3F81021520705D508
:10697000D3F80C2142F04002C3F80C21FFF7B8FF16
:10698000064BDA6842F00102DA60D3F80C2142F0DB
:106990000102C3F80C2108BD26640020002000522B
:1069A0000F289ABF00F58060400400207047000067
:1069B0004FF4003070470000102070470F2808B5D2
:1069C0000BD8FFF7EDFF00F500330268013204D168
:1069D00004308342F9D1012008BD0020FCE700000B
:1069E0000F2838B505463FD8FFF782FF1F4CFFF749
:1069F0008DFF4FF0FF3307286361C4F814311DD8B1
:106A00002361FFF775FF030243F02403E360E368AB
:106A100043F08003E36023695A07FCD42846FFF75C
:106A200067FFFFF7BDFF4FF4003100F08FFA2846F3
:106A3000FFF78EFFBDE83840FFF7C0BFC4F8103144
:106A4000FFF756FFA0F108031B0243F02403C4F82C
:106A50000C31D4F80C3143F08003C4F80C31D4F875
:106A600010315B07FBD4D9E7002038BD002000526D
:106A70002DE9F84F05460C46104645EA0203DE06AE
:106A800002D00020BDE8F88F20F01F00DFF8BCB076
:106A9000DFF8BCA0FFF73AFF04EB0008444503D140
:106AA0000120FFF755FFEDE720222946204602F09E
:106AB0008FF810B920352034F0E72B4605F120027D
:106AC0001F68791CDDD104339A42F9D105F178436E
:106AD0001B481C4EB3F5801F1B4B38BF184603F1F3
:106AE000F80332BFD946D1461E46FFF701FF0760C3
:106AF000A5EB040C336804F11C0143F0020333607E
:106B0000231FD9F8007017F00507FAD153F8042FA6
:106B10008B424CF80320F4D1BFF34F8FFFF7E8FE10
:106B20004FF0FF332022214603602846336823F0CC
:106B30000203336002F04CF80028BBD03846B0E7BF
:106B4000142100520C200052142000521020005238
:106B50001021005210B5084C237828B11BB9FFF75B
:106B6000D5FE0123237010BD002BFCD02070BDE8A2
:106B70001040FFF7EDBE00BF266400202DE9F04F66
:106B80000D4685B0814658B111F00D0614BF202284
:106B9000082211F00803019304D0431E034269D078
:106BA000002435E0002E37D009F11F0121F01F0924
:106BB0004FF00108314F05F00403DFF8CCA005EADF
:106BC000080BBBF1000F32D07869C0072FD408F151
:106BD00001080C37B8F1060FF3D19EB9284D49468C
:106BE000A819019201F078FD0446002839D1203619
:106BF000019AA02EF3D1494601F06EFD044600280B
:106C00002FD1019A49461F4801F066FD044660BB3A
:106C1000204605B0BDE8F08F0029C9D101462846BD
:106C2000029201F059FD0446D8B9029AC0E713B1A7
:106C300078694107CBD5AC0702D578698007C6D5FE
:106C4000019911B178690107C1D549460AEB48108D
:106C5000CDE9022301F040FD0446DDE902230028CE
:106C6000B5D04A460021204601E04A460021FBF704
:106C700059F8CDE70246002E96D199E770950008A5
:106C80006864002028640020486400200021FFF789
:106C900075BF00000121FFF771BF000070B5144DF2
:106CA0000124144E40F2FF3200210120FBF73AF894
:106CB00006EB441001342A6955F80C1F01F0F8FC6A
:106CC000062CF5D137254FF4C0542046FFF7E2FFDC
:106CD000014628B122460848BDE8704001F0E8BCF2
:106CE000C4EBC404013D4FEAD404EED170BD00BF33
:106CF0007095000848640020286400200421FFF7F4
:106D00003DBF00004843FFF7C1BF000008B101F0DC
:106D100055BD7047B0F5805F10B5044607D8FFF742
:106D2000EDFF28B92046BDE81040FFF7AFBF0020B7
:106D300010BD0000FFF7EABF08B501F055FE034A99
:106D4000D2E90032C01842EB010108BD08650020FD
:106D5000434BD3E900232DE9F34113437CD0FFF7E4
:106D6000EBFF404A00230027F9F766FB06460D4675
:106D70003D4A0023F9F760FB0023144630462946BC
:106D8000394AF9F759FB4FF461613C23ADF80170C2
:106D9000B4FBF1F5B4FBF3F601FB154103FB16461A
:106DA0004624B1FBF3F1314BF6B28DF80040984226
:106DB0003CD84FF0640C4FF4C87EA30704F26C7209
:106DC00025D1B2FBFCF30CFB132313BBB2FBFEF388
:106DD0000EFB1322B2FA82F35B0903F26D18621CF8
:106DE0008045D2B217D90FB18DF800400022204C57
:106DF0004FF00C0C17460CFB0343D4B2013213F8CE
:106E000004C084450CD8A0EB0C000127F5E7002353
:106E1000E3E70123E1E7A0EB080014460127CCE7F4
:106E20000FB18DF80140431C8DF802309DF8010030
:106E3000431C9DF800005038400640EA43509DF83E
:106E4000023040EA034040EA560040EAC52040EAEA
:106E5000411002B0BDE8F0814FF40410F9E700BF23
:106E60000865002040420F008051010090230B0074
:106E7000B89500080244074BD2B210B5904200D139
:106E800010BD441C00B253F8200041F8040BE0B2DE
:106E9000F4E700BF504000580E4B30B51C6F24047F
:106EA00005D41C6F1C671C6F44F400441C670A4C1B
:106EB00002442368D2B243F480732360074B9042AC
:106EC00000D130BD441C51F8045B00B243F820509F
:106ED000E0B2F4E70044025800480258504000581D
:106EE00007B5012201A90020FFF7C4FF019803B0F4
:106EF0005DF804FB13B50446FFF7F2FFA04205D08E
:106F0000012201A900200194FFF7C6FF02B010BDC5
:106F100010B56424013C4FF47A70FFF7E7F814F0E1
:106F2000FF04F7D1084B4FF0807214249A6103F5E7
:106F3000805308229A61013C4FF47A70FFF7D6F82B
:106F400014F0FF04F7D110BD000002580144BFF354
:106F50004F8F064B884204D3BFF34F8FBFF36F8F21
:106F60007047C3F85C022030F4E700BF00ED00E09A
:106F70000144BFF34F8F064B884204D3BFF34F8FBA
:106F8000BFF36F8F7047C3F870022030F4E700BF83
:106F900000ED00E070B5054616460C4601201021B4
:106FA000FFF7B0FE286046733CB1204636B1FFF7CC
:106FB000A5FE2B68186000B19C6070BDFFF76AFEEB
:106FC000F7E7000070B50E461546044600B30B689F
:106FD00043608368934210D213B10068FFF796FEB6
:106FE000637B28462BB1FFF789FE206020B9A060A3
:106FF00070BDFFF74FFEF8E7A560206805F11F019F
:10700000306021F01F01FFF7A1FF01202073EFE79F
:107010000120EDE710B5044640B10068884205D173
:10702000606808B1FAF758FE0023237310BD000012
:1070300070B50E461546044620B383689A4210D9AF
:1070400013B10068FFF762FE637B28462BB1FFF7A0
:1070500055FE206020B9A06070BDFFF71BFEF8E769
:10706000A560316819B12A462068FAF735FE206814
:1070700005F11F01306021F01F01FFF779FF0120AA
:107080002073E9E70120E7E720B103688B4204BFE2
:107090000023037370470000034B1A681AB9034AB0
:1070A000D2F8D0241A6070471065002000400258C2
:1070B00008B5FFF7F1FF024B1868C0F3806008BD08
:1070C0001065002070B5BFF34F8FBFF36F8F1A4A62
:1070D0000021C2F85012BFF34F8FBFF36F8F536977
:1070E00043F400335361BFF34F8FBFF36F8FC2F888
:1070F0008410BFF34F8FD2F8803043F6E074C3F3AF
:10710000C900C3F34E335B0103EA0406014646EAB5
:1071100081750139C2F86052F9D2203B13F1200F7A
:10712000F2D1BFF34F8F536943F480335361BFF300
:107130004F8FBFF36F8F70BD00ED00E0FEE70000E2
:10714000214B2248224A70B5904237D3214BC11EB1
:10715000DA1C121A22F003028B4238BF00220021EF
:10716000FAF7E0FD1C4A0023C2F88430BFF34F8FCA
:10717000D2F8803043F6E074C3F3C900C3F34E3352
:107180005B0103EA0406014646EA81750139C2F84B
:107190006C52F9D2203B13F1200FF2D1BFF34F8F85
:1071A000BFF36F8FBFF34F8FBFF36F8F0023C2F812
:1071B0005032BFF34F8FBFF36F8F70BD53F8041B76
:1071C00040F8041BC0E700BF20970008206700209C
:1071D000206700202067002000ED00E0054B996B40
:1071E00021EA000199631A6E22EA00021A661B6EF8
:1071F000704700BF0045025870B5D0E92443002213
:107200004FF0FF359E6804EB42135101D3F800099B
:10721000002805DAD3F8000940F08040C3F80009DF
:10722000D3F8000B002805DAD3F8000B40F08040BB
:10723000C3F8000B013263189642C3F80859C3F82B
:10724000085BE0D24FF00113C4F81C3870BD000099
:10725000890141F02001016103699B06FCD41220E1
:10726000FEF7D8BE10B50A4C2046FEF759FB094B75
:10727000C4F89030084BC4F89430084C2046FEF710
:107280004FFB074BC4F89030064BC4F8943010BD48
:107290001465002000000840F4950008B065002047
:1072A000000004400096000870B503780546012BE5
:1072B00058D13F4BD0F89040984254D13D4B0E21CD
:1072C00065209A6B42F000629A631A6E42F0006287
:1072D0001A661B6E384BD3F8802042F00062C3F868
:1072E0008020D3F8802022F00062C3F88020D3F8F9
:1072F000803000F037FF314BE360314BC4F8003889
:107300000023D5F89060C4F8003EC02323604FF4FA
:107310000413A3633369002BFCDA01230C203361CF
:10732000FEF778FE3369DB07FCD41220FEF772FE0D
:107330003369002BFCDA00262846A660FFF75CFFC5
:107340006B68C4F81068DB68C4F81468C4F81C687B
:1073500063BB1C4BA3614FF0FF336361A36843F031
:107360000103A36070BD184B9842C9D1114B4FF077
:1073700080609A6B42F000729A631A6E42F000725B
:107380001A661B6E0C4BD3F8802042F00072C3F8D3
:107390008020D3F8802022F00072C3F88020D3F838
:1073A0008030FFF71BFF0E214D20A2E7074BD1E7EE
:1073B0001465002000450258004402584014004063
:1073C00003002002003C30C0B0650020083C30C003
:1073D000F8B5D0F89040054600214FF000662046F1
:1073E000FFF736FFD5F8941000234FF001128F6895
:1073F0004FF0FF30C4F83438C4F81C2804EB4312B3
:1074000001339F42C2F80069C2F8006BC2F8080954
:10741000C2F8080BF2D20B68D5F89020C5F8983066
:10742000636210231361166916F01006FBD1122057
:10743000FEF7F0FDD4F8003823F4FE63C4F80038FA
:10744000A36943F4402343F01003A3610923C4F864
:107450001038C4F814380B4BEB604FF0C043C4F83D
:10746000103B094BC4F8003BC4F81069C4F800395C
:10747000D5F8983003F1100243F48013C5F8982032
:10748000A362F8BDD095000840800010D0F890208D
:1074900090F88A10D2F8003823F4FE6343EA01130F
:1074A000C2F80038704700002DE9F84300EB810373
:1074B000D0F890500C468046DA680FFA81F94801FE
:1074C000166806F00306731E022B05EB41134FF0FE
:1074D000000194BFB604384EC3F8101B4FF00101F1
:1074E00004F1100398BF06F1805601FA03F3916985
:1074F00098BF06F5004600293AD0578A04F1580192
:10750000374349016F50D5F81C180B430021C5F8CB
:107510001C382B180127C3F81019A7405369611EA6
:107520009BB3138A928B9B08012A88BF5343D8F8D8
:107530009820981842EA034301F140022146C8F816
:107540009800284605EB82025360FFF781FE08EBA6
:107550008900C3681B8A43EA845348341E4364018C
:107560002E51D5F81C381F43C5F81C78BDE8F883A8
:1075700005EB4917D7F8001B21F40041C7F8001BA1
:10758000D5F81C1821EA0303C0E704F13F030B4AB6
:107590002846214605EB83035A60FFF759FE05EBA9
:1075A0004910D0F8003923F40043C0F80039D5F869
:1075B0001C3823EA0707D7E7008000100004000208
:1075C000D0F894201268C0F89820FFF715BE00008C
:1075D0005831D0F8903049015B5813F4004004D082
:1075E00013F4001F0CBF0220012070474831D0F86F
:1075F000903049015B5813F4004004D013F4001F8D
:107600000CBF02200120704700EB8101CB68196A92
:107610000B6813604B6853607047000000EB8103F8
:1076200030B5DD68AA691368D36019B9402B84BFEF
:10763000402313606B8A1468D0F890201C4402EB3E
:107640004110013C09B2B4FBF3F46343033323F06C
:10765000030343EAC44343F0C043C0F8103B2B6824
:1076600003F00303012B0ED1D2F8083802EB4110CE
:1076700013F4807FD0F8003B14BF43F0805343F0F5
:107680000053C0F8003B02EB4112D2F8003B43F03C
:107690000443C2F8003B30BD2DE9F041D0F89060C2
:1076A00005460C4606EB4113D3F8087B3A07C3F8AE
:1076B000087B08D5D6F814381B0704D500EB8103E6
:1076C000DB685B689847FA071FD5D6F81438DB07E4
:1076D0001BD505EB8403D968CCB98B69488A5A68F5
:1076E000B2FBF0F600FB16228AB91868DA689042FD
:1076F0000DD2121AC3E90024302383F311882146E6
:107700002846FFF78BFF84F31188BDE8F081012341
:1077100003FA04F26B8923EA02036B81CB68002B26
:10772000F3D021462846BDE8F041184700EB81031D
:107730004A0170B5DD68D0F890306C692668E66063
:1077400056BB1A444FF40020C2F810092A6802F010
:107750000302012A0AB20ED1D3F8080803EB42143F
:1077600010F4807FD4F8000914BF40F0805040F03E
:107770000050C4F8000903EB4212D2F8000940F0AF
:107780000440C2F800090122D3F8340802FA01F1DA
:107790000143C3F8341870BD19B9402E84BF40208E
:1077A000206020681A442E8A8419013CB4FBF6F448
:1077B00040EAC44040F00050C6E700002DE9F8431D
:1077C000D0F8906005460C464F0106EB4113D3F804
:1077D000088918F0010FC3F808891CD0D6F81038B2
:1077E000DB0718D500EB8103D3F80CC0DCF81430AC
:1077F000D3F800E0DA68964530D2A2EB0E024FF0E3
:1078000000091A60C3F80490302383F31188FFF74E
:107810008DFF89F3118818F0800F1DD0D6F8343809
:107820000126A640334217D005EB84030134D5F876
:107830009050D3F80CC0E4B22F44DCF8142005EBD0
:107840000434D2F800E05168714514D3D5F83438C7
:1078500023EA0606C5F83468BDE8F883012303FA75
:1078600001F2038923EA02030381DCF80830002BCC
:10787000D1D09847CFE7AEEB0103BCF810008342AC
:1078800028BF0346D7F8180980B2B3EB800FE3D8BE
:107890009068A0F1040959F8048FC4F80080A0EBA7
:1078A00009089844B8F1040FF5D818440B449060C7
:1078B0005360C8E72DE9F84FD0F8905004466E6940
:1078C000AB691E4016F480586E6103D0BDE8F84FD6
:1078D000FEF796B8002E12DAD5F8003E9B0705D0C9
:1078E000D5F8003E23F00303C5F8003ED5F8043870
:1078F000204623F00103C5F80438FEF7AFF837053A
:1079000005D52046FFF778FC2046FEF795F8B00431
:107910000CD5D5F8083813F0060FEB6823F4705334
:107920000CBF43F4105343F4A053EB6031071BD555
:107930006368DB681BB9AB6923F00803AB6123788C
:10794000052B0CD1D5F8003E9A0705D0D5F8003E9E
:1079500023F00303C5F8003E2046FEF77FF8636876
:10796000DB680BB120469847F30200F1BA80B702FA
:1079700026D5D4F8909000274FF0010A09EB471262
:10798000D2F8003B03F44023B3F5802F11D1D2F895
:10799000003B002B0DDA62890AFA07F322EA03039F
:1079A000638104EB8703DB68DB6813B1394620464B
:1079B00098470137D4F89430FFB29B689F42DDD9D5
:1079C000F00619D5D4F89000026AC2F30A1702F043
:1079D0000F0302F4F012B2F5802F00F0CA80B2F566
:1079E000402F09D104EB8303002200F58050DB68AF
:1079F0001B6A974240F0B0803003D5F8185835D54F
:107A0000E90303D500212046FFF746FEAA0303D56C
:107A100001212046FFF740FE6B0303D502212046DB
:107A2000FFF73AFE2F0303D503212046FFF734FE6C
:107A3000E80203D504212046FFF72EFEA90203D554
:107A400005212046FFF728FE6A0203D506212046BD
:107A5000FFF722FE2B0203D507212046FFF71CFE6D
:107A6000EF0103D508212046FFF716FE700340F111
:107A7000A780E90703D500212046FFF79FFEAA074C
:107A800003D501212046FFF799FE6B0703D502219C
:107A90002046FFF793FE2F0703D503212046FFF76B
:107AA0008DFEEE0603D504212046FFF787FEA806CB
:107AB00003D505212046FFF781FE690603D506217F
:107AC0002046FFF77BFE2A0603D507212046FFF755
:107AD00075FEEB0574D520460821BDE8F84FFFF789
:107AE0006DBED4F890904FF0000B4FF0010AD4F81F
:107AF00094305FFA8BF79B689F423FF638AF09EBF3
:107B00004713D3F8002902F44022B2F5802F20D188
:107B1000D3F80029002A1CDAD3F8002942F0904259
:107B2000C3F80029D3F80029002AFBDB3946D4F832
:107B30009000FFF78DFB22890AFA07F322EA03037C
:107B4000238104EB8703DB689B6813B13946204629
:107B500098470BF1010BCAE7910701D1D0F80080DB
:107B6000072A02F101029CBF03F8018B4FEA182893
:107B70003FE704EB830300F58050DA68D2F818C0C1
:107B8000DCF80820DCE9001CA1EB0C0C00218F4282
:107B900008D1DB689B699A683A449A605A683A440B
:107BA0005A6029E711F0030F01D1D0F800808C450D
:107BB00001F1010184BF02F8018B4FEA1828E6E7C2
:107BC000BDE8F88F08B50348FFF774FEBDE808402C
:107BD00000F068BF1465002008B50348FFF76AFE8F
:107BE000BDE8084000F05EBFB0650020D0F89030DE
:107BF00003EB4111D1F8003B43F40013C1F8003B03
:107C000070470000D0F8903003EB4111D1F80039F3
:107C100043F40013C1F8003970470000D0F89030E9
:107C200003EB4111D1F8003B23F40013C1F8003BF2
:107C300070470000D0F8903003EB4111D1F80039C3
:107C400023F40013C1F8003970470000044BDA6BCD
:107C50000243DA635A6E104358665B6E704700BF8A
:107C6000004502583A4B4FF0FF31D3F8802062F0C4
:107C70000042C3F88020D3F8802002F00042C3F80D
:107C80008020D3F88020D3F88420C3F88410D3F860
:107C900084200022C3F88420D3F88400D86F40F0F9
:107CA000FF4040F4FF0040F4DF4040F07F00D86721
:107CB000D86F20F0FF4020F4FF0020F4DF4020F0D8
:107CC0007F00D867D86FD3F888006FEA40506FEA1A
:107CD0005050C3F88800D3F88800C0F30A00C3F8F6
:107CE0008800D3F88800D3F89000C3F89010D3F838
:107CF0009000C3F89020D3F89000D3F89400C3F814
:107D00009410D3F89400C3F89420D3F89400D3F8D7
:107D10009800C3F89810D3F89800C3F89820D3F8C7
:107D20009800D3F88C00C3F88C10D3F88C00C3F8FB
:107D30008C20D3F88C00D3F89C00C3F89C10D3F8A7
:107D40009C10C3F89C20D3F89C3000F0D3B900BF3E
:107D50000044025808B50122504BC3F80821504B8B
:107D60005A6D42F002025A65DA6F42F00202DA6797
:107D70000422DB6F4B4BDA605A689104FCD54A4A07
:107D80001A6001229A60494ADA6000221A614FF4AF
:107D900040429A61434B9A699204FCD51A6842F4B6
:107DA00080721A60424B1A6F12F4407F04D04FF475
:107DB00080321A6700221A671A6842F001021A60BC
:107DC0003B4B1A685007FCD500221A611A6912F061
:107DD0003802FBD1012119604FF0804159605A6788
:107DE000344ADA62344A1A611A6842F480321A60FC
:107DF0002F4B1A689103FCD51A6842F480521A601E
:107E00001A689204FCD52D4A2D499A6200225A63C1
:107E1000196301F57C01DA6301F5E77199635A642E
:107E2000284A1A64284ADA621A6842F0A8521A608C
:107E30001F4B1A6802F02852B2F1285FF9D148228C
:107E40009A614FF48862DA6140221A621F4ADA644A
:107E50001F4A1A651F4A5A651F4A9A6532231F4AEC
:107E60001360136803F00F03022BFAD1104A136951
:107E700043F003031361136903F03803182BFAD19D
:107E80004FF00050FFF7E2FE4FF08040FFF7DEFEBC
:107E90004FF00040BDE80840FFF7D8BE0080005119
:107EA000004502580048025800C000F004000001DC
:107EB000004402580000FF01008890083220600052
:107EC00063020901470E0508DD0BBF0120000020F9
:107ED000000001100910E000000101100020005214
:107EE0004FF0B04208B5D2F8883003F00103C2F871
:107EF000883023B1044A13680BB150689847BDE835
:107F0000084000F0CFBD00BF986600204FF0B0429F
:107F100008B5D2F8883003F00203C2F8883023B1E4
:107F2000044A93680BB1D0689847BDE8084000F058
:107F3000B9BD00BF986600204FF0B04208B5D2F836
:107F4000883003F00403C2F8883023B1044A13696F
:107F50000BB150699847BDE8084000F0A3BD00BFD1
:107F6000986600204FF0B04208B5D2F8883003F090
:107F70000803C2F8883023B1044A93690BB1D06971
:107F80009847BDE8084000F08DBD00BF986600200E
:107F90004FF0B04208B5D2F8883003F01003C2F8B1
:107FA000883023B1044A136A0BB1506A9847BDE880
:107FB000084000F077BD00BF986600204FF0B04346
:107FC00010B5D3F8884004F47872C3F88820A3066B
:107FD00004D5124A936A0BB1D06A9847600604D55B
:107FE0000E4A136B0BB1506B9847210604D50B4A10
:107FF000936B0BB1D06B9847E20504D5074A136C1D
:108000000BB1506C9847A30504D5044A936C0BB18F
:10801000D06C9847BDE8104000F044BD9866002041
:108020004FF0B04310B5D3F8884004F47C42C3F855
:108030008820620504D5164A136D0BB1506D984720
:10804000230504D5124A936D0BB1D06D9847E00417
:1080500004D50F4A136E0BB1506E9847A10404D596
:108060000B4A936E0BB1D06E9847620404D5084A50
:10807000136F0BB1506F9847230404D5044A936FD4
:108080000BB1D06F9847BDE8104000F00BBD00BFAA
:108090009866002008B50348FCF72CFDBDE80840B1
:1080A00000F000BDA436002008B50348FCF722FE0E
:1080B000BDE8084000F0F6BCFC38002008B50348D5
:1080C000FCF718FEBDE8084000F0ECBC6839002061
:1080D00008B50348FCF70EFEBDE8084000F0E2BC1E
:1080E000D439002008B500F039FDBDE8084000F0A3
:1080F000D9BC0000062108B5084600F033F8062177
:10810000072000F02FF80621082000F02BF80621A8
:10811000092000F027F806210A2000F023F80621A4
:10812000172000F01FF80621282000F01BF8092175
:108130007A2000F017F80921312000F013F8072108
:10814000322000F00FF80C21262000F00BF80C2153
:10815000272000F007F80C215220BDE8084000F06D
:1081600001B80000090100F16043012203F56143F9
:10817000C9B283F8001300F01F039A4043099B0023
:1081800003F1604303F56143C3F880211A6070472F
:1081900008B5FFF767FD00F0AFFCFDF7E5F9FDF767
:1081A00083F9FDF7BBFBFDF78DFAFEF751FABDE849
:1081B000084000F029BA000030B50433039C017276
:1081C000002104FB0325C160C0E90653049B03633F
:1081D000059BC0E90000C0E90422C0E90842C0E9EB
:1081E0000A11436330BD00000022416AC260C0E949
:1081F0000411C0E90A226FF00101FDF7B7BF0000CA
:10820000D0E90432934201D1C2680AB9181D7047FF
:1082100000207047036919600021C2680132C26002
:10822000C269134482699342036124BF436A0361B4
:10823000FDF790BF38B504460D46E3683BB162696F
:108240000020131D1268A3621344E36207E0237A3F
:1082500033B929462046FDF76DFF0028EDDA38BD19
:108260006FF00100FBE70000C368C269013BC36017
:108270004369134482699342436124BF436A436163
:1082800000238362036B03B11847704770B5302336
:10829000044683F31188866A3EB9FFF7CBFF054693
:1082A00018B186F31188284670BDA36AE26A13F8F4
:1082B000015B9342A36202D32046FFF7D5FF002360
:1082C00083F31188EFE700002DE9F84F04460E46CE
:1082D000174698464FF0300989F311880025AA46C1
:1082E000D4F828B0BBF1000F09D141462046FFF772
:1082F000A1FF20B18BF311882846BDE8F88FD4E99F
:108300000A12A7EB050B521A934528BF9346BBF1FF
:10831000400F1BD9334601F1400251F8040B914242
:1083200043F8040BF9D1A36A403640354033A362C9
:10833000D4E90A239A4202D32046FFF795FF8AF335
:108340001188BD42D8D289F31188C9E730465A4610
:10835000F9F7C2FCA36A5E445D445B44A362E7E7AD
:1083600010B5029C0433017203FB0421C460C0E910
:1083700006130023C0E90A33039B0363049BC0E98F
:108380000000C0E90422C0E90842436310BD0000B8
:10839000026A6FF00101C260426AC0E90422002251
:1083A000C0E90A22FDF7E2BED0E904239A4201D1D6
:1083B000C26822B9184650F8043B0B60704700238E
:1083C0001846FAE7C3680021C2690133C3604369F4
:1083D000134482699342436124BF436A4361FDF7BA
:1083E000B9BE000038B504460D46E3683BB12369C9
:1083F00000201A1DA262E2691344E36207E0237AB7
:1084000033B929462046FDF795FE0028EDDA38BD40
:108410006FF00100FBE7000003691960C268013AD0
:10842000C260C269134482699342036124BF436AF4
:10843000036100238362036B03B118477047000098
:1084400070B530230D460446114683F31188866AC1
:108450002EB9FFF7C7FF10B186F3118870BDA36A6C
:108460001D70A36AE26A01339342A36204D3E169F7
:1084700020460439FFF7D0FF002080F31188EDE794
:108480002DE9F84F04460D46904699464FF0300AC4
:108490008AF311880026B346A76A4FB94946204699
:1084A000FFF7A0FF20B187F311883046BDE8F88FB1
:1084B000D4E90A073A1AA8EB0607974228BF1746DD
:1084C000402F1BD905F1400355F8042B9D4240F87D
:1084D000042BF9D1A36A40364033A362D4E90A23BE
:1084E0009A4204D3E16920460439FFF795FF8BF3E4
:1084F00011884645D9D28AF31188CDE729463A46F4
:10850000F9F7EAFBA36A3D443E443B44A362E5E736
:10851000D0E904239A4217D1C3689BB1836A8BB117
:10852000043B9B1A0ED01360C368013BC360C36950
:108530001A4483699A42026124BF436A036100239B
:1085400083620123184670470023FBE701F01F03F5
:10855000F0B502F01F0456095A1C0123B6EB511F57
:1085600050F8265003FA02F34FEA511703F1FF3394
:108570003DBF50F82720C4F12000134003EA050056
:108580003BBF03FA00F225FA04F0E0401043F0BDCF
:1085900070B57E227F210546FFF7D8FF18B101286C
:1085A00019D0002070BD3E2249212846FFF7CEFF9A
:1085B0002F22044631212846FFF7C8FF0646013422
:1085C0005022023653212846B440FFF7BFFF093836
:1085D00004FA00F0E6E7302245212846FFF7B6FF0F
:1085E00001308002DEE7000090F8D63090F8D72006
:1085F0001B0403EB026390F8D42090F8D5001344D9
:1086000003EB00207047000000F084BA014B586A69
:10861000704700BF000C0040034B002258631A61F2
:108620000222DA60704700BF000C0040014B0022BC
:10863000DA607047000C0040014B5863704700BF80
:10864000000C0040024B034A1A60034A5A6070470C
:10865000646600202067002000000220074B49428A
:1086600010B55C68201A08401968821A8A4203D340
:10867000A24201D85A6010BD0020FCE764660020C9
:1086800008B5302383F31188FFF7E8FF002383F355
:10869000118808BD0448054B03600023C0E901337D
:1086A0000C3000F017B900BF6C660020818600080E
:1086B000CB1D083A23F00703591A521A10B4D208F6
:1086C0000024C0E9004384600C301C605A605DF8EF
:1086D000044B00F0FFB800002DE9F74F364FCD1DD9
:1086E0008846002818BF0746082A4FEAD50538BF34
:1086F000082207F10C003C1D9146019000F02CF976
:10870000019809F10701C9F1000E2246246864B9F5
:1087100000F02CF93B68CBB308224946E8009847A3
:10872000044698B340E9027830E004EB010CD4F839
:1087300004A00CEA0E0C0AF10106ACF1080304EBEC
:10874000C6069E42E1D9A6EB0C0CB5EBEC0F4FEA46
:10875000EC0BDAD89C421DD204F10802AB45A3EB26
:1087600002024FEAE202626009D9691CED4303EBA1
:10877000C1025D445560256843F8315022601C46B3
:10878000C3F8048044F8087B00F0F0F8204603B0FA
:10879000BDE8F08FAA45216802D111602346EEE7BB
:1087A000013504EBC50344F8351003F10801761ACE
:1087B000F6105E601360F1E76C66002073B5044646
:1087C000A0F1080550F8080C54F8043C061D0C30C4
:1087D00007330190DB0844F8043C00F0BDF8334651
:1087E00001989E421A6801D0AB4228D20AB1954244
:1087F00025D244F8082C54F8042C1D60013254F89A
:10880000081C05EBC206B14206D14E68324444F85A
:10881000042C0A6844F8082C5E68711C03EBC10143
:108820008D4207D154F8042C013232445A6054F876
:10883000082C1A6002B0BDE8704000F097B81346EB
:10884000CFE70000FEE7000070B51E4B0025044690
:1088500086B058600E460563816300F0FBF804F1B2
:108860002803A5606563C4E90A3304F11003C4E971
:1088700004334FF0FF33C4E90044C4E90635FFF781
:10888000C5FE2B46024604F13C012046C4E90823FC
:1088900080230D4A6567FDF7C7FB7368E0600B4AEC
:1088A00003620123009280F824306846F268019246
:1088B0003269CDE90223064BCDE90435FDF7E8FB2B
:1088C00006B070BDE8480020149600080C96000819
:1088D000458800080023C0E90000836003617047F9
:1088E00070B51C4B05468468DE685CB3B44213D196
:1088F00003690133036170BDA36094F8243083B130
:10890000062B15D1A06A2146D4E9003213605A60C3
:10891000FDF7DCFAA36A9C68B368A2689A42EBD3BD
:1089200006E0D4E90032204613605A60FDF7DEFA13
:1089300028463146FDF7CAFAB5620620BDE8704008
:10894000FDF7D6BA0369866001330361336BC360F8
:108950003063D0E74046002008B5302383F3118808
:10896000FFF7BEFF002383F3118808BD194BD968B8
:1089700083688B4210B520D1302383F311880269BC
:10898000013A0261B2B90468C368A0420B631ED009
:108990004A6B9BB901238A60036103681A6802600D
:1089A00050601A6B8360C26018631846FDF79EFA28
:1089B000FDF7EEFA002383F3118810BD1C68A34273
:1089C00003D0A468A24238BF2246DB68E1E7826098
:1089D000F0E700BF40460020024A536B1843506343
:1089E000704700BF4046002070B5104E82B0FDF7C2
:1089F000F7FA0546FFF70AFE3268034690423360F5
:108A000037BF0B4A0A495168146836BF0131D1E9B2
:108A1000004151600419284641F100010191FDF720
:108A2000E9FA2046019902B070BD00BF8C660020B3
:108A300090660020EFF30983054968334A6B22F002
:108A400001024A6383F30988002383F31188704786
:108A500000EF00E0302080F3118862B60D4B0E4A23
:108A6000D96821F4E0610904090C0A430B49DA6072
:108A7000D3F8FC2042F08072C3F8FC20084AC2F808
:108A8000B01F116841F0010111602022DA7783F8EC
:108A90002200704700ED00E00003FA0555CEACC59A
:108AA000001000E0302310B583F311880E4B5B6893
:108AB00013F4006314D0F1EE103AEFF309844FF091
:108AC0008073683CE361094BDB6B236684F30988A0
:108AD000FDF73CFA10B1064BA36110BD054BFBE757
:108AE00083F31188F9E700BF00ED00E000EF00E03C
:108AF0002F040008320400080023054A19460133F8
:108B0000102BC2E9001102F10802F8D1704700BF32
:108B1000986600200E4B9A6C42F008029A641A6F15
:108B200042F008021A670B4A1B6FD36B43F008032D
:108B3000D363C722084B9A624FF0FF32DA620022F9
:108B40009A615A63DA605A6001225A611A6070476A
:108B5000004502580010005C000C0040094A08B5AE
:108B60001169D3680B40D9B29B076FEA010111610B
:108B700007D5302383F31188FDF730FA002383F300
:108B8000118808BD000C0040FEF7C0B8012838BFAE
:108B9000012010B504462046FEF778F830B900F001
:108BA00007F808B900F00CF88047F4E710BD0000A2
:108BB000024B1868BFF35B8F704700BF1867002037
:108BC00008B5062000F056F80120FDF77FFC0000F4
:108BD00010B501390244904201D1002005E003782C
:108BE00011F8014FA34201D0181B10BD0130F2E76C
:108BF000884210B501EB020402D98442234607D80B
:108C0000431EA14208D011F8012B03F8012FF8E709
:108C1000024401468A4200D110BD13F8014D02F80A
:108C2000014DF7E71F2938B504460D4604D9162330
:108C300003604FF0FF3038BD426C12B152F8213062
:108C40004BB9204600F030F82A4601462046BDE8E0
:108C5000384000F017B8012B0AD0591C03D1162355
:108C600003600120E7E7002442F8254028469847A2
:108C70000020E0E7024B01461868FFF7D3BF00BFB2
:108C80007422002038B5074D0023044608461146DB
:108C90002B60FDF71FFC431C02D12B6803B123603E
:108CA00038BD00BF1C670020FDF70EBCC9B20346EB
:108CB00010F8012B1AB18A42F9D1184670470029E1
:108CC00018BF0023F9E70000034611F8012B03F851
:108CD000012B002AF9D1704710B50139034632B192
:108CE00011F8014F03F8014B013A002CF7D11A4457
:108CF0000021934200D110BD03F8011BF9E70000E9
:108D00004D4435002D2D0A002F6172647570696C19
:108D10006F742E6162696E002F6172647570696C88
:108D20006F742D7665726966792E6162696E002FA7
:108D30006172647570696C6F742D666C6173682EF6
:108D40006162696E002F6172647570696C6F742D59
:108D5000666C61736865642E6162696E0000000074
:108D60000000000000000000F10E00088D0F000858
:108D70003D110008C50F0008850F00080000000025
:108D800000000000ED0E0008990F000875110008A2
:108D9000E90E0008F50E000853544D333248373FB2
:108DA0003F3F0053544D3332483733782F373278B2
:108DB0000053544D3332483734332F3735332F3740
:108DC0003530000001105A000310590001205800EE
:108DD000032056002F0000005375636365737366AC
:108DE000756C6C79206D6F756E74656420534443A7
:108DF0006172642028736C6F77646F776E3D2575A0
:108E0000290A0000EB769045584641542020200066
:108E10004641543332202020000000002A3A3C3ED4
:108E20007C223F7F002B2C3B3D5B5D004355454141
:108E30004141414345454549494941414592924F48
:108E40004F4F5555594F554F9C4F9E9F41494F5538
:108E5000A5A5A6A7A8A9AAABACADAEAFB0B1B2B359
:108E6000B4414141B8B9BABBBCBDBEBFC0C1C2C3A9
:108E7000C4C54141C8C9CACBCCCDCECFD1D145455F
:108E80004549494949D9DADBDCDD49DF4FE14F4F3C
:108E90004F4FE6E8E85555555959EEEFF0F1F2F32A
:108EA000F4F5F6F7F8F9FAFBFCFDFEFF0103050700
:108EB000090E10121416181C1E00000061001A037F
:108EC000E0001703F8000703FF000100780100012C
:108ED000300132010601390110014A012E017901E8
:108EE000060180014D00430281018201820184015B
:108EF000840186018701870189018A018B018B0129
:108F00008D018E018F0190019101910193019401D6
:108F1000F60196019701980198013D029B019C0181
:108F20009D0120029F01A001A001A201A201A401B4
:108F3000A401A601A701A701A901AA01AB01AC01E7
:108F4000AC01AE01AF01AF01B101B201B301B30198
:108F5000B501B501B701B801B801BA01BB01BC0147
:108F6000BC01BE01F701C001C101C201C301C401BE
:108F7000C501C401C701C801C701CA01CB01CA01AB
:108F8000CD011001DD0101008E01DE011201F301AE
:108F90000300F101F401F401F80128012202120199
:108FA0003A020900652C3B023B023D02662C3F025F
:108FB00040024102410246020A015302400081017F
:108FC0008601550289018A0158028F015A029001D7
:108FD0005C025D025E025F02930161026202940123
:108FE0006402650266026702970196016A02622CBA
:108FF0006C026D026E029C01700271029D0173028F
:1090000074029F0176027702780279027A027B026B
:109010007C02642C7E027F02A60181028202A901E9
:109020008402850286028702AE014402B101B201C8
:1090300045028D028E028F0290029102B7017B03DE
:109040000300FD03FE03FF03AC0304008603880353
:1090500089038A03B1031103C2030200A303A3031C
:10906000C4030803CC0303008C038E038F03D803CF
:109070001801F2030A00F903F303F403F503F603FE
:10908000F703F703F903FA03FA033004200350044B
:109090001007600422018A043601C1040E01CF04C6
:1090A0000100C004D0044401610526040000000052
:1090B0007D1D0100632C001E9601A01E5A01001F99
:1090C0000806101F0606201F0806301F0806401F4E
:1090D0000606511F0700591F521F5B1F541F5D1FBB
:1090E000561F5F1F601F0806701F0E00BA1FBB1FB0
:1090F000C81FC91FCA1FCB1FDA1FDB1FF81FF91FAC
:10910000EA1FEB1FFA1FFB1F801F0806901F0806AF
:10911000A01F0806B01F0400B81FB91FB21FBC1F54
:10912000CC1F0100C31FD01F0206E01F0206E51F6F
:109130000100EC1FF31F0100FC1F4E210100322132
:1091400070211002842101008321D0241A05302CC3
:109150002F04602C0201672C0601752C0201802C63
:109160006401002D260841FF1A030000C700FC001F
:10917000E900E200E400E000E500E700EA00EB00BF
:10918000E800EF00EE00EC00C400C500C900E600F6
:10919000C600F400F600F200FB00F900FF00D60064
:1091A000DC00F800A300D800D7009201E100ED0038
:1091B000F300FA00F100D100AA00BA00BF00AE002F
:1091C000AC00BD00BC00A100AB00BB009125922506
:1091D000932502252425C100C200C000A9006325F3
:1091E000512557255D25A200A500102514253425FD
:1091F0002C251C2500253C25E300C3005A255425B9
:1092000069256625602550256C25A400F000D00056
:10921000CA00CB00C8003101CD00CE00CF00182518
:109220000C2588258425A600CC008025D300DF00EE
:10923000D400D200F500D500B500FE00DE00DA0053
:10924000DB00D900FD00DD00AF00B400AD00B100CF
:109250001720BE00B600A700F700B800B000A800B5
:10926000B700B900B300B200A025A00001000000C3
:109270000000000000960000000000000000000058
:1092800000000000000000000000000000000000DE
:10929000496600084D6600083D51000875540008F5
:1092A000D1500008F950000821510008B9500008B9
:1092B0000000000029550008155500085155000808
:1092C0003D5500084955000835550008215500084E
:1092D0000D5500085D5500080000000041560008CB
:1092E0002D560008695600085556000861560008BA
:1092F0004D560008395600082556000875560008D6
:1093000000000000010000000000000063300000C9
:109310000C9300080000000000000000B846002088
:10932000E84800200000812A00000000AAAAAAAA9A
:1093300000000024FFFE00000000000000A00A0062
:109340000001000000000000AAAAAAAA0000000074
:10935000FFFF000000000000000000001400AA56FB
:1093600000000000AAAAAAAA14005554FFFF00009A
:1093700000000000CCCC0C0020681A0000000000A7
:10938000AAAA8AAA10541500FFFF0000000C70075B
:10939000770000004081020100100000AAAAAAAADA
:1093A00000410100F7FF000000000070070000000E
:1093B0000000000000000000AAAAAAAA0000000005
:1093C000FFFF00000000000000000000000000009F
:1093D00000000000AAAAAAAA00000000FFFF0000E7
:1093E000000000000000000000000000000000007D
:1093F000AAAAAAAA00000000FFFF000000000000C7
:10940000000000000000000000000000AAAAAAAAB4
:1094100000000000FFFF000000000000000000004E
:109420000000000000000000AAAAAAAA0000000094
:10943000FFFF00000000000000000000000000002E
:1094400000000000AAAAAAAA00000000FFFF000076
:1094500000000000000000004375626550696C6FF9
:109460007400437562654F72616E67652B2D424CC7
:10947000002553455249414C2500000002000000E0
:109480000000000061580008D1580008400040006A
:1094900098610020A8610020020000000000000088
:1094A000030000000000000019590008000000003F
:1094B00010000000B8610020000000000100000062
:1094C000000000001465002001010200456700084B
:1094D00055660008F1660008D566000843000000E4
:1094E000E494000809024300020100C032090400AC
:1094F0000001020201000524001001052401000101
:10950000042402020524060001070582030800FF67
:1095100009040100020A00000007050102400000E2
:10952000070581024000000012000000309500088D
:109530001201100102000040AE2D5810000201027D
:10954000030100000403090425424F415244250051
:10955000437562654F72616E6765506C757300305C
:109560003132333435363738394142434445460089
:109570000000002000000200020000000000003097
:1095800000000400080000000000002400000800A3
:10959000040000000004000000FC000002000000C5
:1095A00000000430008000000800000000000038C7
:1095B00000000100010000001F1C1F1E1F1E1F1FB6
:1095C0001E1F1E1F1F1D1F1E1F1E1F1F1E1F1E1FB3
:1095D00000000000755A00082D5D0008D95D0008E4
:1095E000400040004C6600204C6600200100000056
:1095F0005C660020800000004001000008000000C0
:1096000000010000001000000800000069646C65A3
:10961000000000006D61696E002C043804043808F5
:109620000C10141C202425260000000000006404F7
:109630000100040000000000000C0010283034007D
:10964000286EFF7F010000002704000000000000DA
:1096500000001E0000000000FF000000F048002095
:10966000FC38002068390020D439002000000000B8
:10967000988D000883040000A38D000850040000AA
:10968000B18D0008010000000000000000960000FD
:109690000000080096000000000800000400000020
:1096A00044950008000000000000000000000000D9
:1096B00000000000000000000000000078220020F0
:1096C000000000000000000000000000000000009A
:1096D000000000000000000000000000000000008A
:1096E000000000000000000000000000000000007A
:1096F000000000000000000000000000000000006A
:020000040801F1
:020000040802F0
:1000000000060030F10D020875800E086103020839
:10001000F17F0E08E97F0E08ED7F0E08F30D020850
:10002000F30D0208F30D0208F30D02082DF7140872
:10003000F30D0208F30D0208F30D0208F30D020898
:10004000F30D0208F30D0208F30D0208F30D020888
:10005000F30D0208F30D0208F57A1508217B150847
:100060004D7B1508797B1508A57B15082106150819
:100070004906150875061508A1061508CD061508C8
:10008000F50615082107150811021508596E0E0806
:10009000416F0E08C96E0E08B16F0E08D17B1508AE
:1000A000F30D0208357D1508F30D0208497D15088A
:1000B0005D7D1508F30D0208717D1508290F1508DF
:1000C0009D0F15081110150885101508D91D150864
:1000D000ED1D1508F30D0208BD7C1508D17C15082F
:1000E000357C1508F30D0208F30D0208F30D020824
:1000F000F30D0208F30D0208F30D02084D07150871
:10010000F30D0208A97C1508857D1508F30D02087A
:10011000E57C1508F30D0208F30D0208F30D020843
:1001200079071508A1071508CD071508F90715085F
:1001300025081508F30D0208F30D0208F30D020857
:10014000F30D0208F30D0208F30D0208F30D020887
:100150004D08150879081508A5081508F97C150833
:10016000F30D0208F30D0208F30D0208F30D020867
:10017000F30D020865771508F30D0208F30D020868
:10018000F30D0208F30D02080D7D1508217D1508F9
:10019000011E1508F30D0208F30D0208F30D020805
:1001A000F30D0208F30D0208F30D0208F30D020827
:1001B000F30D0208F30D0208F30D0208F9101508FB
:1001C0006D111508F30D0208F30D0208F30D020876
:1001D000F30D020851771508F30D0208F30D02081C
:1001E000F30D0208F30D0208F30D0208F30D0208E7
:1001F000F30D0208F30D0208F30D0208F30D0208D7
:10020000F30D0208F30D0208F30D0208F30D0208C6
:10021000F30D0208F30D0208F30D0208F30D0208B6
:10022000F30D0208F30D0208F30D0208F30D0208A6
:10023000F30D0208F30D0208F30D02083102150850
:10024000F30D0208D9031508010415082D0415083B
:100250005904150885041508B1041508DD041508AE
:1002600009051508F30D0208F30D0208F30D020845
:10027000F30D0208F30D0208F30D0208F30D020856
:10028000F30D0208F30D0208F30D0208F30D020846
:10029000F30D0208F30D0208F30D0208F30D020836
:1002A000F30D0208F30D0208F30D0208F30D020826
:1002B000F30D0208F30D0208F30D0208F30D020816
:1002C000F30D0208F30D0208F30D0208F30D020806
:1002D000F30D0208F30D0208F30D0208F30D0208F6
:1002E000094F020871A30208D9AD03084945040863
:1002F00051B7050885340808293A080851DC080870
:10030000A157090851600908D563090831160A0880
:10031000F9A20A0821D10B08650B0C08C11A0C08B8
:100320002D730E0869780E08B9940E089D2A1008DE
:1003300051CC10089D1A11086DA211083904130838
:100340000545130809621308A1A41308CDD11308A9
:1003500025DE1308A5191408AD24140800000000B8
:10036000EFF30383EFF30982EFF30881DFF814D092
:100370002DE9FE4F684601F011F8BDE8FE4F8D46AD
:10038000704700006C2C0030F1EE101AA0EC200A2F
:1003900001607047A0EC108A704700BF81F00041F7
:1003A00002E000BF83F0004330B54FEA41044FEA5A
:1003B000430594EA050F08BF90EA020F1FBF54EAF5
:1003C000000C55EA020C7FEA645C7FEA655C00F091
:1003D000E2804FEA5454D4EB5555B8BF6D420CDD62
:1003E0002C4480EA020281EA030382EA000083EAE5
:1003F000010180EA020281EA0303362D88BF30BD85
:1004000011F0004F4FEA01314FF4801C4CEA1131DA
:1004100002D0404261EB410113F0004F4FEA033339
:100420004CEA133302D0524263EB430394EA050FC4
:1004300000F0A780A4F10104D5F1200E0DDB02FA33
:100440000EFC22FA05F2801841F1000103FA0EF2C7
:10045000801843FA05F359410EE0A5F120050EF18D
:10046000200E012A03FA0EFC28BF4CF0020C43FABE
:1004700005F3C01851EBE37101F0004507D54FF0CB
:10048000000EDCF1000C7EEB00006EEB0101B1F51B
:10049000801F1BD3B1F5001F0CD349085FEA300061
:1004A0004FEA3C0C04F101044FEA445212F5800F6C
:1004B00080F09A80BCF1004F08BF5FEA500C50F109
:1004C000000041EB045141EA050130BD5FEA4C0CEC
:1004D000404141EB0101013C28BFB1F5801FE9D249
:1004E00091F0000F04BF01460020B1FA81F308BF6C
:1004F0002033A3F10B03B3F120020CDA0C3208DD38
:1005000002F1140CC2F10C0201FA0CF021FA02F112
:100510000CE002F11402D8BFC2F1200C01FA02F182
:1005200020FA0CFCDCBF41EA0C019040E41AA2BFA7
:1005300001EB0451294330BD6FEA04041F3C1CDA6F
:100540000C340EDC04F11404C4F1200220FA04F08F
:1005500001FA02F340EA030021FA04F345EA030139
:1005600030BDC4F10C04C4F1200220FA02F001FAFB
:1005700004F340EA0300294630BD21FA04F029467D
:1005800030BD94F0000F83F4801306BF81F4801116
:100590000134013D4EE77FEA645C18BF7FEA655C89
:1005A00029D094EA050F08BF90EA020F05D054EA5B
:1005B000000C04BF1946104630BD91EA030F1EBF60
:1005C0000021002030BD5FEA545C05D14000494164
:1005D00028BF41F0004130BD14F580043CBF01F557
:1005E000801130BD01F0004545F0FE4141F470013D
:1005F0004FF0000030BD7FEA645C1ABF1946104618
:100600007FEA655C1CBF0B46024650EA013406BF18
:1006100052EA033591EA030F41F4002130BD00BFD7
:1006200090F0000F04BF0021704730B54FF4806494
:1006300004F132044FF000054FF0000150E700BF15
:1006400090F0000F04BF0021704730B54FF4806474
:1006500004F1320410F0004548BF40424FF0000161
:100660003EE700BF42004FEAE2014FEA31014FEAA4
:1006700002701FBF12F07F4393F07F4F81F06051F3
:10068000704732F07F4208BF704793F07F4F04BF3E
:1006900041F40021704730B54FF4607401F000451B
:1006A00021F000411CE700BF50EA010208BF70477B
:1006B00030B54FF000050AE050EA010208BF70476C
:1006C00030B511F0004502D5404261EB41014FF4D5
:1006D000806404F132045FEA915C3FF4D8AE4FF0DD
:1006E00003025FEADC0C18BF03325FEADC0C18BFC0
:1006F000033202EBDC02C2F1200300FA03FC20FA11
:1007000002F001FA03FE40EA0E0021FA02F114445D
:10071000BDE600BF80F0004002E000BF81F0004174
:1007200042001FBF5FEA410392EA030F7FEA226C97
:100730007FEA236C6AD04FEA1262D2EB1363C1BF27
:10074000D218414048404140B8BF5B42192B88BF96
:10075000704710F0004F40F4000020F07F4018BFB9
:10076000404211F0004F41F4000121F07F4118BFD9
:10077000494292EA030F3FD0A2F1010241FA03FC81
:1007800010EB0C00C3F1200301FA03F100F0004369
:1007900002D5494260EB4000B0F5000F13D3B0F131
:1007A000807F06D340084FEA310102F10102FE2AA0
:1007B00051D2B1F1004F40EBC25008BF20F0010010
:1007C00040EA03007047490040EB0000013A28BFAF
:1007D000B0F5000FEDD2B0FA80FCACF1080CB2EB32
:1007E0000C0200FA0CF0AABF00EBC25052421843B0
:1007F000BCBFD0401843704792F0000F81F4000155
:1008000006BF80F400000132013BB5E74FEA410327
:100810007FEA226C18BF7FEA236C21D092EA030F93
:1008200004D092F0000F08BF0846704790EA010F0D
:100830001CBF0020704712F07F4F04D1400028BF3A
:1008400040F00040704712F100723CBF00F500001C
:10085000704700F0004343F0FE4040F40000704752
:100860007FEA226216BF08467FEA236301464202FE
:1008700006BF5FEA412390EA010F40F48000704711
:100880004FF0000304E000BF10F0004348BF4042B7
:100890005FEA000C08BF704743F0964301464FF0F3
:1008A00000001CE050EA010208BF70474FF000034F
:1008B0000AE000BF50EA010208BF704711F0004390
:1008C00002D5404261EB41015FEA010C02BF844660
:1008D0000146002043F0B64308BFA3F18053A3F5BF
:1008E0000003BCFA8CF2083AA3EBC25310DB01FA06
:1008F00002FC634400FA02FCC2F12002BCF1004F8A
:1009000020FA02F243EB020008BF20F0010070471A
:1009100002F1200201FA02FCC2F1200250EA4C006E
:1009200021FA02F243EB020008BF20EADC707047B4
:100930007BB972B90029BEBF00204FF0004106E02C
:1009400008BF00281CBF6FF000414FF0FF3000F0DF
:100950004DBAADF1080C6DE904CE002909DB002B7E
:100960001ADB00F0DBF8DDF804E0DDE9022304B077
:100970007047404261EB4101002B1BDB00F0CEF8D9
:10098000DDF804E0DDE9022304B0404261EB4101FF
:10099000524263EB43037047524263EB430300F060
:1009A000BDF8DDF804E0DDE9022304B0404261EB6C
:1009B00041017047524263EB430300F0AFF8DDF8AA
:1009C00004E0DDE9022304B0524263EB43037047C5
:1009D00053B94AB9002908BF00281CBF4FF0FF31A6
:1009E0004FF0FF3000F002BAADF1080C6DE904CE13
:1009F00000F094F8DDF804E0DDE9022304B070476C
:100A000030B1012390FAA0F0B0FA80F0184470479A
:100A100008460029FBD02123F4E700BF430803F078
:100A20005533C01A830803F0333300F033301844D1
:100A300000EB101000F00F3000EB002000EB004046
:100A4000000E704707EE900AF5EEC07AF1EE10FA4C
:100A500001D400F023B8F1EE677A08B517EE900ADA
:100A600000F01CF8404261EB410108BD08B50246A8
:100A70000B4643EC172BB5EEC07BF1EE10FA03D416
:100A8000BDE8084000F02AB8B1EE477B51EC170BE7
:100A900000F024F8404261EB410108BD9FED0B6B73
:100AA00007EE900A9FED0B5BB7EEE77A27EE066B39
:100AB000BCEEC66BB8EE464BA4EE457BFCEEC77BA6
:100AC00016EE101A17EE900A704700BF00000000E3
:100AD0000000F03D000000000000F0419FED0B6BB6
:100AE00041EC170B9FED0B5B27EE066BBCEEC66B64
:100AF000B8EE464BA4EE457BFCEEC77B16EE101A13
:100B000017EE900A704700BFAFF3008000000000AE
:100B10000000F03D000000000000F0412DE9F0472A
:100B2000089D04468E46002B4DD18A42944669D9D1
:100B3000B2FA82F252B101FA02F3C2F1200120FAB4
:100B400001F10CFA02FC41EA030E94404FEA1C4802
:100B5000210CBEFBF8F61FFA8CF708FB16E341EAFE
:100B6000034306FB07F199420AD91CEB030306F184
:100B7000FF3080F01F81994240F21C81023E6344A5
:100B80005B1AA4B2B3FBF8F008FB103344EA034449
:100B900000FB07F7A7420AD91CEB040400F1FF335E
:100BA00080F00A81A74240F207816444023840EA9B
:100BB0000640E41B00261DB1D4400023C5E90043D4
:100BC0003146BDE8F0878B4209D9002D00F0EF8057
:100BD0000026C5E9000130463146BDE8F087B3FA8A
:100BE00083F6002E4AD18B4202D3824200F2F98072
:100BF000841A61EB030301209E46002DE0D0C5E975
:100C0000004EDDE702B9FFDEB2FA82F2002A40F0C0
:100C10009280A1EB0C014FEA1C471FFA8CFE0126C3
:100C2000200CB1FBF7F307FB131140EA01410EFB67
:100C300003F0884208D91CEB010103F1FF3802D20E
:100C4000884200F2CB804346091AA4B2B1FBF7F008
:100C500007FB101144EA01440EFB00FEA64508D92B
:100C60001CEB040400F1FF3102D2A64500F2BB8068
:100C70000846A4EB0E0440EA03409CE7C6F12007B7
:100C8000B34022FA07FC4CEA030C20FA07F401FAFD
:100C900006F31C43F9404FEA1C4900FA06F3B1FB86
:100CA000F9F8200C1FFA8CFE09FB181140EA0141EB
:100CB00008FB0EF0884202FA06F20BD91CEB010188
:100CC00008F1FF3A80F08880884240F28580A8F1E0
:100CD00002086144091AA4B2B1FBF9F009FB101132
:100CE00044EA014100FB0EFE8E4508D91CEB0101D0
:100CF00000F1FF346CD28E456AD90238614440EA73
:100D00000840A0FB0294A1EB0E01A142C846A646F2
:100D100056D353D05DB1B3EB080261EB0E0101FA7B
:100D200007F722FA06F3F1401F43C5E900710026D8
:100D30003146BDE8F087C2F12003D8400CFA02FC2E
:100D400021FA03F3914001434FEA1C471FFA8CFE3E
:100D5000B3FBF7F007FB10360B0C43EA064300FB2E
:100D60000EF69E4204FA02F408D91CEB030300F1CC
:100D7000FF382FD29E422DD9023863449B1B89B283
:100D8000B3FBF7F607FB163341EA034106FB0EF30C
:100D90008B4208D91CEB010106F1FF3816D28B42B9
:100DA00014D9023E6144C91A46EA004638E72E4685
:100DB000284605E70646E3E61846F8E64B45A9D27D
:100DC000B9EB020864EB0C0E0138A3E74646EAE7EC
:100DD000204694E74046D1E7D0467BE7023B61449A
:100DE00032E7304609E76444023842E7704700BF03
:100DF00002E000F000F8FEE772B6374880F308889A
:100E0000364880F3098836483649086040F20000C9
:100E1000CCF200004EF63471CEF200010860BFF350
:100E20004F8FBFF36F8F40F20000C0F2F0004EF61C
:100E30008851CEF200010860BFF34F8FBFF36F8F70
:100E40004FF00000E1EE100A4EF63C71CEF20001C8
:100E50000860062080F31488BFF36F8F35F16EFEB3
:100E600034F1C2FB4FF055301F491B4A91423CBF41
:100E700041F8040BFAE71D49184A91423CBF41F87A
:100E8000040BFAE71A491B4A1B4B9A423EBF51F822
:100E9000040B42F8040BF8E700201849184A914265
:100EA0003CBF41F8040BFAE735F18AFE34F1D8FC77
:100EB000144C154DAC4203DA54F8041B8847F9E78B
:100EC00001F0F8FA114C124DAC4203DA54F8041B4D
:100ED0008847F9E735F172BE000600300022003085
:100EE0000000020808ED00E00000003000060030BD
:100EF000087C1A0800220030742A0030782A00305A
:100F00006C290230E00202085C0302085C0302085C
:100F10005C0302082DE9F04F2DED108AC1F80CD0CA
:100F2000D0F80CD0BDEC108ABDE8F08F002383F31D
:100F300011882846A047002034F184F8FEE733F1F9
:100F400083FE00DFFEE7000070B54FF0FF0C4CF4AD
:100F5000E06C1CEA11541DBF1CEA135594EA0C0FF7
:100F600095EA0C0F00F0DEF82C4481EA030621EA32
:100F70004C5123EA4C5350EA013518BF52EA03356D
:100F800041F4801143F4801338D0A0FB02CE4FF01F
:100F90000005E1FB02E506F00042E0FB03E54FF04F
:100FA0000006E1FB03569CF0000F18BF4EF0010E47
:100FB000A4F1FF04B6F5007F64F5407404D25FEA43
:100FC0004E0E6D4146EB060642EAC62141EA5551F6
:100FD0004FEAC52040EA5E504FEACE2EB4F1FD0C38
:100FE00088BFBCF5E06F1ED8BEF1004F08BF5FEAB6
:100FF000500E50F1000041EB045170BD06F0004668
:1010000046EA010140EA020081EA0301B4EB5C0414
:10101000C2BFD4EB0C0541EA045170BD41F480110C
:101020004FF0000E013C00F3AB8014F1360FDEBF31
:10103000002001F0004170BDC4F10004203C35DA0D
:101040000C341BDC04F11404C4F1200500FA05F390
:1010500020FA04F001FA05F240EA020001F0004231
:1010600021F0004110EBD37021FA04F642EB0601A7
:101070005EEA430E08BF20EAD37070BDC4F10C04D1
:10108000C4F1200500FA04F320FA05F001FA04F295
:1010900040EA020001F0004110EBD37041F1000181
:1010A0005EEA430E08BF20EAD37070BDC4F120058C
:1010B00000FA05F24EEA020E20FA04F301FA05F2F4
:1010C00043EA020321FA04F001F0004121FA04F29C
:1010D00020EA020000EBD3705EEA430E08BF20EA6C
:1010E000D37070BD94F0000F0FD101F000464000A6
:1010F00041EB010111F4801F08BF013CF7D041EA28
:10110000060195F0000F18BF704703F0004652002B
:1011100043EB030313F4801F08BF013DF7D043EAFC
:101120000603704794EA0C0F0CEA135518BF95EAB2
:101130000C0F0CD050EA410618BF52EA4306D1D139
:1011400081EA030101F000414FF0000070BD50EA58
:10115000410606BF1046194652EA430619D094EAE2
:101160000C0F02D150EA013613D195EA0C0F05D1CC
:1011700052EA03361CBF104619460AD181EA030120
:1011800001F0004141F0FE4141F470014FF00000D8
:1011900070BD41F0FE4141F4780170BD4FEA41025B
:1011A00012F5001215D211D56FF47873B3EB6252B9
:1011B00012D94FEAC12343F0004343EA505311F0E0
:1011C000004F23FA02F018BF404270474FF0000072
:1011D000704750EA013005D111F0004008BF6FF0B0
:1011E000004070474FF00000704700BF4FEA4102D7
:1011F000B2F1E04324BFB3F5001CDCF1FE5C0DD975
:1012000001F0004C4FEAC0024CEA5070B2F1004FBE
:1012100040EB830008BF20F00100704711F0804FC1
:1012200021D113F13872BCBF01F00040704741F486
:1012300080114FEA5252C2F11802C2F1200C10FA8A
:101240000CF320FA02F018BF40F001004FEAC1236E
:101250004FEAD32303FA0CFC40EA0C0023FA02F312
:101260004FEA4303CCE77FEA625307D150EA0133E8
:101270001EBF4FF0FE4040F44000704701F00040B8
:1012800040F0FE4040F40000704700BF01F0FF0155
:10129000102A2BDB10F0070F08D010F8013B013AA1
:1012A0008B422DD010F0070F42B3F6D1F0B441EAD3
:1012B000012141EA014122F007047FF000070023E9
:1012C000F0E80256083C85EA010586EA010685FA3F
:1012D00047F5A3FA87F586FA47F6A5FA87F68EB999
:1012E000EED1F0BC01F0FF0102F0070232B110F8BC
:1012F000013B013A83EA010313B1F8D100207047A2
:1013000001387047002D06BF35460338073815F001
:10131000010F07D1013015F4807F02BF013015F4B1
:10132000C03F0130F0BC0138704700BFEC46A0E878
:10133000F05F4FF000007047B0E8F05FE54608004E
:1013400008BF0120704700BF10F8012B11F8013BC6
:10135000012A28BF9A42F7D0D01A7047034613F8E3
:10136000012B002AFBD1181A01387047A8B110B51B
:1013700004460AE000F08AFA14F8041C54E9030356
:101380001B1AB3FBF1F200F081FA204654F80C3B33
:10139000082201210133EDD110BD70472DE9F04F36
:1013A0000023A7B00293C36A009013F0040FD0E9A2
:1013B000002118BF0A46D9064FF0E021D3694CBF7F
:1013C00002F1200002F168000192DB0903F004033E
:1013D00003430393D1F8883D03F4A003B3F5A00FB2
:1013E00001D10123029393694FF004094F4D4FF04F
:1013F00001081B884E4C03F47F43A3F53E43B3FA28
:1014000083F35B09049329E000F03EF9FFF7AEFF98
:101410004FF0E023D3F8003D03F47023B3F5402FE1
:101420000ED0444A4FF0FF3305A88DF81C9005926A
:1014300014328DF828800692CDE90833FFF796FF25
:101440002B68A34206D03C4B0422012105A805933A
:1014500000F01CFA00F064FB00285ED103A82C60A9
:1014600000F000FC04220121344800F00FFA0422AD
:10147000012102A800F00AFA10220121019800F0CF
:1014800005FA0098202201210C3000F0FFF90198A4
:1014900004220121103000F0F9F90422012103A8EF
:1014A00000F0F4F901980C220121143000F0EEF95B
:1014B0000C220121009800F0E9F9029BDA07A3D57C
:1014C000009BDB6ADB0622D415A80DF1140AFEF797
:1014D00061FFDDF804E0D4460EF120060EF1600B4A
:1014E0003068103656F80C1C674656F8082C0CF17C
:1014F000100C56F8043C5E450FC7F1D1DEF86030A1
:10150000259384225046012100F0C0F97CE70DF1BB
:10151000140A5046FEF738FFF3E7049B1BB1019A0B
:1015200093690233936127B0BDE8F08F782A0030C9
:10153000ED55CEAC28ED00E0ACCE55EDE80C16082C
:1015400038B527206D2531F1DDFB124A124B4FF0E3
:10155000FF34D2F89000114940F48020C2F8900086
:10156000D2F8900020F48020C2F890000D20D2F82C
:1015700090209A6C42F480229A641A6F42F480227E
:101580001A6701221B6F064BCD600C6208601A704F
:1015900038BD00BF004402580045025800480040D2
:1015A000A42C0030002953D02DE9F84F0746894676
:1015B0000026284DDFF8A480274C17F801AB2B78C4
:1015C0004FEA1A1218F802B0002B3CD0C4F828B029
:1015D000E369580604D435F177FAE3695906FAD578
:1015E0000AF00F0A2B7818F80AA04BB3C4F828A009
:1015F000E3695A0604D435F167FAE3695B06FAD564
:101600000136B14522D03107D7D12B784FF00D0BE1
:10161000DFF84CA08BB1C4F828B0E3695A0604D4B3
:1016200035F152FAE3695B06FAD51AF801BFBBF14E
:10163000000FC2D02B78002BEDD1FFF781FFEAE736
:10164000FFF77EFFD2E7FFF77BFFBFE7BDE8F88F2C
:10165000704700BFA42C003000480040700D1608F1
:1016600074181708014B1868704700BFFCFF1F086B
:10167000014B0248C01A704780841A0800002008F5
:101680000048704780841A08724943F69822724BCA
:1016900009682DE9F04F0A441B7883B002EB030977
:1016A00033F1D0F9002800F09B806C4F04466C4B5E
:1016B0000225DFF8D4810126FF1ADFF8C8A12EE049
:1016C0001846019134F1FEFD0199A8BB206AAB4692
:1016D0000BF101030BEB4B0E04F13C058944DBB22B
:1016E00001440AEB8E0CB94503EB43034AF82E4044
:1016F000CCF804500BF102058CF808600AEB830C5F
:10170000EDB24AF823008CF80860CCF804104FD2F0
:10171000204633F1A7F90446E8B13A2D1BD8206AD8
:10172000404505D0211AE369002BC9D1AB46CFE76C
:101730004C4BA3EB0801F6E705EB450C01350AEB32
:101740008C005FFA85FB0672E3694AF82C300D3392
:101750004360206ABCE7B7EB090129D40BF1030B06
:10176000414E42482B465FFA8BF5341A8C424CDCD2
:1017700004EB090203EB4303BF1A4AF823000122DA
:101780000AEB8303002F1A723A465E6010DB38487A
:10179000384BC11A914205EB450249DD01354AF843
:1017A00022301F440AEB8203EDB201225F601A72FD
:1017B0003B2D1ED94FF0FF330122CAF8C4328AF8FC
:1017C000CC22CAF8C8322C4B1B782BB12B4A2C4B9D
:1017D00012681B68CAE900232A4803B0BDE8F08FED
:1017E0001E4F1F4BFF1AB7EB09012BD50225DFF85F
:1017F00094A005EB45054FF0FF3201210AEB85036C
:101800004AF8252019725A60DDE703EB43030144CF
:1018100001224AF823000AEB8303154859601A7223
:101820000022144B1746C11A914205EB4502B5DC64
:101830004AF8223001350AEB82030122EDB25860EA
:101840001A72B5E7084E032508480223DFF834A0D2
:10185000341A8BE7942C00306C2C003000002008E8
:1018600080841A08002200306C290230782A003067
:10187000000004307029023000220030982C003023
:10188000902C003004220030000600309A4B1B7868
:101890002DE9F04F824685B00E4693462BB9974B03
:1018A0001B782BBB05B0BDE8F08F022900F0EE805D
:1018B000042900F0B580012900F0AE80904D2B780E
:1018C0000D27DFF858828F4C7BB1A762E3695A0677
:1018D00004D435F1F9F8E3695B06FAD518F8017F0D
:1018E000002FDCD02B78002BEFD1FFF729FEECE79F
:1018F000854B4FF00009854A9B1A0093CB45D1D008
:10190000834F844C38682578031D009A2B449342FA
:1019100079D2202D51D0022E24D0042E0DD0012EAC
:10192000ECD12378DFF8F0815A1C22701AF80920D4
:1019300009F1010908F80320E0E7DFF8DC81002560
:10194000434620789AF80010421CE9400835D2B28C
:1019500008F80010202A227018D0202DF1D109F1AA
:101960000109CBE725789AF80030DFF8AC8108F858
:1019700005300135EDB2202D257030D06B1C09F1FA
:1019800001092370002308F80530B7E738685F497C
:1019900001920844194634F141FA39684FF00003C6
:1019A000019A203123705C4B3960002118463AF1CE
:1019B00063FD35F189F8584BCFE7544B2A46564919
:1019C000184434F12BFA3B6800212A462033524850
:1019D00021703B603AF150FD35F176F89BE74B4BB7
:1019E0002A4638684146184434F118FA3B68002109
:1019F0002A462033404621703B603AF13DFD35F1E7
:101A000063F82578BAE7444A4FF0FF312023D161CB
:101A1000237005B0BDE8F08F1146FFF7C3FD4DE719
:101A2000002A3FF44BAF02460027354D0DF10C085C
:101A300052F8043B334C0092039301910137042187
:101A40004046FFF7AFFDBB451ED0009ABE0752F8D7
:101A5000043B00920393F1D12A780D26DFF8BC9065
:101A60007AB1A662E369580604D435F12DF8E3692A
:101A70005906FAD519F8016F002EDFD02A78002A0E
:101A8000EFD1FFF75DFDECE7019E18E7002A3FF478
:101A900015AF024600271A4D0DF10C0832F8023B33
:101AA000184C0092ADF80C300191013702214046EC
:101AB000FFF778FDBB45E7D0009A790732F8023B83
:101AC0000092ADF80C30F0D12A780D26DFF84C905A
:101AD0007AB1A662E3695A0604D434F1F5FFE369EA
:101AE0005B06FAD519F8016F002EDED02A78002A9D
:101AF000EFD1FFF725FDECE76D2C00300022003020
:101B0000A42C0030004800400000200880841A08FF
:101B1000942C00306C2C0030702C00307418170896
:101B2000F8B5324B1A782AB9314A1078F0B9012247
:101B30001A70F8BD2F4E0D252F4F304C3B7893B1C6
:101B4000A562E3695A0604D434F1BEFFE3695B067B
:101B5000FAD516F8015F002DF0D1294B58680038EE
:101B600018BF0120F8BDFFF7EBFCE9E7254D264E35
:101B70002B68264C26481A1D3178241A0A44A242A2
:101B800006D239BB9C421CD8002034F1F1F9E4E7BD
:101B9000204A4FF0FF31D1612022327018442022B8
:101BA0001C4934F13BF92A68337800211948134461
:101BB000202231702B603AF15FFC34F185FF2B68F5
:101BC000E0E7144920221448CB6134F127F934F1BD
:101BD0007BFFD9E703F120029442DFD81F29DDD82B
:101BE0000C4AD36120223270D8E700BF6D2C003040
:101BF00000220030EC0C1608A42C003000480040F5
:101C00009C2C0030942C00306C2C003000002008FC
:101C100080841A08702C0030E0FF1F080E4B1B78E0
:101C200010B5B3B1642100200C4A0D4CD3699B065A
:101C3000FCD5536ADBB28B424FF0640101D0002027
:101C4000F4E70130C0B20E2801D0015DEEE70020BC
:101C500010BDFFF775FCE5E7A42C003000480040FC
:101C6000FC0C16082DE9F04102680646EFF30581E9
:101C7000D9205369C9B2C6F0BDF9674B1B782BB99F
:101C8000664C2378002B37D1BDE8F081644B0D27DB
:101C9000DFF8B081634D644C96E8030083E80300ED
:101CA0002B7833B3A762E3695F0604D434F10CFFE9
:101CB000E3695806FAD518F8017F002FF0D1736850
:101CC0000BB32B784227DFF88081574C73B1A762A2
:101CD000E369590604D434F1F7FEE3695A06FAD5EC
:101CE00018F8017F1FB32B78002BF0D1FFF728FCE9
:101CF000EDE7FFF725FCD5E73568002D47D1002338
:101D00002370BDE8F081DFF844814327464C2B78EF
:101D1000002B6AD0A762E3695B0604D434F1D4FED9
:101D2000E3695F06FAD518F8017F002FEFD1DFF8DD
:101D3000208120273C4C2B78002B53D0A762E369ED
:101D4000580604D434F1C0FEE3695906FAD518F8F0
:101D5000017F002FEFD1FFF761FF2B78DFF8F480D0
:101D60000D27314C83B1A762E3695A0604D434F1DC
:101D7000ABFEE3695B06FAD518F8017F002F3FF44C
:101D80007FAF2B78002BEED1FFF7DAFBEBE728468D
:101D900034F198FA0028B2D0284634F1BBFA00F2A8
:101DA0001450854231D3214BA5F214521A602846B3
:101DB00034F1C6FA05F5E053834220D81C4A13607B
:101DC00000231C481C4A03601C481D49801A0B70E4
:101DD00002D10DE083420BD252F8041B04330131CF
:101DE000F8D08CE7FFF7ACFBA8E7FFF7A9FB91E77A
:101DF00034F16AFE0120BDE8F04134F1B9B828465B
:101E000034F19EFA0A4B1860DAE7284634F182FA78
:101E1000064B1860CBE700BF6D2C0030002200306D
:101E20009C2C0030A42C003000480040982C00303E
:101E3000902C0030942C003080841A080000200878
:101E40006C2C00300C0D1608140D1608680D1608C1
:101E5000200D160874181708094B10B584B0D3F874
:101E6000184900946A46D3F81C490194D3F82049D4
:101E7000D3F82439CDE90243C3F08CF804B010BD87
:101E8000B07C003070B5857F0DB1284670BD04462A
:101E90000E460C48022104F03FFE60B904210948B7
:101EA00004F03AFE054630B92046074A3146C2F0F2
:101EB00041F8284670BD31462046BDE87040C3F069
:101EC000F5B900BFB02C0030840D160870B590B085
:101ED00005460E46C2F0CEFA044610B9204610B0B0
:101EE00070BD10212846C1F0A3FB0028F6D00021C8
:101EF0002E2204A803913AF1BFFA0EF089FA0021CC
:101F0000322303AA0DF0DEFC04460028E6D103A923
:101F1000034B3246284600911021C1F091FBDDE7CA
:101F2000B00D1608F8B53C4F3B7813B10025284694
:101F3000F8BD012406463C70C3F030FA054630B9BE
:101F4000364A38702846137823431370F8BD6EF074
:101F500059FA21466DF018F9314803F0FDFE314B76
:101F60001C710B2458F052F857F08CFF611E11F0D1
:101F7000FF04F7D10EF04CFA2B4AD0F8F831C2F832
:101F80000C3390F87432D9073DD4284B0121284CEA
:101F90001B68D86A03681B689847214809F034FD1C
:101FA00001212448BEF0A8FF6EF02CFA04F58053FE
:101FB00094F8182193F88C1F6DF0E2FAA4F5804094
:101FC00003F0BCFE69F034FA68F0C0FD0023A4F50C
:101FD00080403B7000F0EEF904460028A7D17BF06A
:101FE000E7FB0421144A71F0E5FF20213046C1F0DF
:101FF0001FFB00289BD0114B012220213046254693
:10200000C1F01EFB93E79B07BFD42146A2F5C04059
:1020100003F0B2F8B9E700BFA52C003098B6003045
:10202000B02C003078B60030B08C0030AC2C0030D2
:10203000B06C0030648C0030BC0D1608DC0D160846
:10204000274B2DE9F04193F8913084B023B9002457
:10205000204604B0BDE8F081C3F0C4FA044600286D
:10206000F5D00EF0D5F905460CF0D8FDC8B9002121
:102070001C48BEF041FF1C4836F058FA6EF0C2F919
:1020800000216DF081F8194B00211B68D86A0368A4
:102090001B689847164804F029FD204604B0BDE8A7
:1020A000F0811DF0B5FE90F92430022BDFD100261F
:1020B00000275FFA86F801AA2846013641460197B3
:1020C000029703970DF048FA10B9032EF1D1CEE72D
:1020D0001DF09EFE01AA41461DF008F8F5E700BF7D
:1020E000B08C0030648C00309C870030AC2C003009
:1020F000B02C003098F00ABC0AF03EBB80F034B837
:1021000069F0DAB82DF0C2B86DF0FAB913F0DEB9A3
:1021100080F03ABC7AF0F6B87AF0ECBE11F076BAFC
:102120000AF04EBB09F000BF5BF098BE20F048BA41
:1021300080F03ABC09F0E6BF03F064B805F0E6BCF5
:1021400000F0BEBB04F0B0BA09F07CBD2DF02ABC93
:1021500010B5044642F62800012120440EF03EF856
:1021600046F618102044BDE810400BF05FBF00BFDA
:1021700010B544F2404400F5C043044493F8911074
:102180002046A7F0C7FD2046BDE81040A7F00CBDD3
:1021900010B5044609F07CFE102120460AF0CCFA66
:1021A00000B910BD204601F033FE2FF017FB2CF0D4
:1021B00047F842F268002044BDE81040A8F0D4BFC0
:1021C00010B5044604F066F8204604F03DF92046B8
:1021D00003F0A6FF204603F051FF7CF073FE7CF075
:1021E000BDFC45F6CC002044BDE8104002F0B0BE76
:1021F00010B5044645F640202044BDF0D7FC2046EB
:1022000003F04EFE204603F0ADFD204603F0F8FD3E
:10221000204604F091F8204604F0DCF9204604F052
:1022200027FA42F2C8702044BDE810408DF08ABE03
:1022300010B4044C21200C60082110705DF8044B90
:10224000196070473812160838B5044646F2203037
:10225000204412F00FF81DF0DBFD90F92130F3B1AE
:1022600090F84033DBB145F6F87004F63C052044A5
:1022700071F06EF80346B7EE001A9E2093ED000A47
:10228000DFED070A30F02AFA94F970382846012B5E
:1022900008BF85ED0E0ABDE838401DF025B938BDF0
:1022A00000000000FFF7D0BF10B5012182B0044646
:1022B0000AF042FA38B9802120460AF03DFA002897
:1022C0003DD102B010BD204601F052FE46F6D412B8
:1022D00045F6B47146F6181004F5DC432244214457
:1022E00020440BF0ADFD4FF4805120460AF024FA53
:1022F0000028E0D045F6301046F6AC326521204487
:10230000224401906CF056FD46F6A44266210198E5
:1023100022446CF04FFD46F69C52672101982244FE
:102320006CF048FD47F2C0026821019822446CF02D
:1023300041FD802120460AF0FFF90028C1D04FF46A
:10234000002120460AF0F8F90028BAD12FF046FA09
:1023500002B0BDE810402BF043BE00BFFFF7A4BFA2
:1023600000F5A042844610B592F8893F13F00104AD
:1023700005D092F8AD3FDB070AD4012010BD45F629
:102380007450084A0421604471F014FE204610BDC8
:1023900045F67450044A0421604471F00BFE00209D
:1023A00010BD00BF4C0E16086C0E1608002301204D
:1023B0000B607047F0B5054642F628068BB02E44F8
:1023C00002A817F0ABFE02A930460EF00BF8044647
:1023D00010B120460BB0F0BD05F544701EF0C2F9F7
:1023E0000028F6D12C4B06A89FED2C6A13ED027A3B
:1023F000DFED2B5A009427EE067AD3ED006A53EDF9
:10240000017A66EEA56A67EE867ABDEEC77AFDEEC2
:10241000E66AFDEEE77A17EE101A16EE903A17EE1E
:10242000902A17F093FE0898D8B10999C9B130F0F5
:1024300097FD044638B306A930460CF0F3FC044679
:10244000C8B145F674570621164A2F44384671F034
:10245000B1FD30460EF0FAF94221384677F09CFE85
:10246000B7E745F67450104A0421284471F0A2FDE4
:1024700020460BB0F0BD45F674500C4A04212844A8
:1024800071F098FDA5E745F67450094A04212844E7
:1024900071F090FD9DE700BF788500308096184B65
:1024A0000000C8420C0F1608800E1608DC0E160835
:1024B000B00E160838B5054C0A46054B014624688F
:1024C000256820462C68A047002038BDAC2C003081
:1024D000B02C003010B5044668F0AAFF46F6D412BE
:1024E000436F04F5A041224401F6B470C36004F5C3
:1024F000DC405364C0F8143391F88C3F133B012B3C
:1025000000D810BD1046BDE81040B7F047BE00BF70
:1025100030B5022183B004460AF00EF9002873D1C9
:102520004FF4003120460AF007F9002852D140212B
:1025300020460AF001F900283AD14FF48061204684
:102540000AF0FAF800283FD1202120460AF0F4F8DA
:1025500060B1514DD5F8280503689B68984710BBBA
:10256000D5F828050368DB689847E0B1802120464C
:102570000AF0E2F830B94FF4802120460AF0DCF886
:1025800000287FD02FF02AF92BF050FD1021204693
:102590000AF0D2F820BB4FF4004120460AF0CCF8F4
:1025A00050BB03B030BD04F5DC40BAF0CFFFDDE72F
:1025B00045F6301020446BF05BFF4FF480612046FD
:1025C0000AF0BAF80028BFD045F6301020446BF06E
:1025D000FBFFB9E745F6B4702044BFF0F5FFA6E76E
:1025E00046F6D4102044B7F013FF4FF400412046C4
:1025F0000AF0A2F80028D4D047F6B830204403B03F
:10260000BDE8304080F086BD012120460AF094F8F4
:10261000002885D1204601F0ABFC46F6D41245F6E1
:10262000B47146F6181004F5DC43224421442044DA
:102630000BF006FC4FF4805120460AF07DF800288C
:102640003FF46EAF45F6301046F6AC3265212044BB
:10265000224401906CF0AEFB46F6A442019866213C
:1026600022446CF0A7FB46F69C5201986721224455
:102670006CF0A0FB47F2C0026821019822446CF084
:1026800099FB4DE74FF4002120460AF055F8002849
:102690007FF478AF7AE700BFB0AC0030FFF738BF07
:1026A000F8B5044646F64C0000212B4D04F5A04633
:1026B0002044FFF7E7FB04F5C04796F8883FA87170
:1026C00060F30003204686F8883F0AF021F897F867
:1026D0009130E8714FF6FF7120466B710AF02CF8CB
:1026E00070BB97F891302BB37EF02AF920460AF0A0
:1026F00059F81A4B04F580461B68DB6A93F89C5026
:1027000015B196F81A3113B386F81A5168F090FE95
:1027100068F024FB46F6D4102044B7F04DFB68F077
:1027200087FE68F01BFB47F21C002044BDE8F84020
:10273000A3F0C0BD45F6B4702044C0F0CDF9D3E796
:10274000D6F8882F0721204601F040FCC9E7C5F0E4
:10275000C9FCC6F81C01D7E778B60030AC2C0030B5
:10276000FFF79EBF10B506480C46BBF087FFDFEDB4
:10277000057A012020EE270A84ED000A10BD00BF73
:10278000789E00300AD7233C10B508480C46BBF0B1
:1027900089FF07EE900A9FED067A0120F8EEE77AAE
:1027A00067EE877AC4ED007A10BD00BF789E0030D6
:1027B0000AD7233C70B500F5804415460E464FF409
:1027C000FA524FF47A712DED048B82B0B4F9840380
:1027D000F0EE408AB0EE608A8DED011A2FF0EAFF2C
:1027E00007EE900AA4F884030B20B8EEE71A9DEDDB
:1027F000010ADFED290A2FF071FFB4F98433DFED10
:10280000276AB0EE409A07EE103AB8EEC77AC7EEE4
:10281000267A67EEA88A27EE888A28EEA87AA8EE9C
:10282000087AB7EEC77AB5EE407BF1EE10FA2CD4F9
:10283000B1EEC76BB7EEC66BB4EEC69AF1EE10FA06
:1028400005D5C9EE067A68EEA78A28EE278A9FED9D
:10285000149A28EE090A35F173FEF0EE407A28EE5C
:10286000890AF0EE678A36F1DDFC28EE800A36F13F
:1028700015F8DFED0C7A20EE270A86ED000A85EDCB
:10288000008A02B0BDEC048B70BDB0EE470B36F190
:102890005DFEB0EE406BCDE700007A4400A08C45B1
:1028A000D40237399F0CB34544F2244307EE901A03
:1028B0000344F8EEE77A93ED000A27EE800A7047AA
:1028C00070B5044682B042F6280004F5A04601A97E
:1028D00020440DF0A7F8D6F8703D834207D0054696
:1028E00046F6D4102044B8F017FAC6F8705D02B06E
:1028F00070BD00BF104A10B5137804460133DBB237
:10290000032B137005D846F6E003034493ED000A49
:1029100010BD46F6FC00002320441370BDF0D6F82D
:1029200046F6D401214430F099FA46F6E0032344F8
:1029300083ED000A10BD00BFA62C003038B5044658
:1029400046F6FC002DED028B2044BDF0C5F805468F
:1029500032F042FD2046B0EE408A09F0D9FE30B197
:10296000DFED127AB4EEE78AF1EE10FA07DC46F6F4
:10297000F003BDEC028B234493ED000A38BDD5ED86
:10298000000A95ED010A36F173FE9FED097ADFED3D
:10299000097A46F6F00320EE070A234420EE270AC0
:1029A00083ED000ABDEC028B38BD00BF00401C4621
:1029B000E02E65420000C84200F5A04270B52DED42
:1029C000068B92F8AC1F11F0010404D09FED3F0A72
:1029D000BDEC068B70BD034600F58046D2F8200999
:1029E000F0EE408A03F5C0457CF09AFAB6F9B633AA
:1029F00007EE900A9FED36AAB0EE680A08EE103A8C
:102A000005F6B803B8EEE79ADFED300AB8EEC88AEB
:102A1000D3ED007AB0EE4A1A672028EE278A2FF00D
:102A20005DFEF0EE408A4FF4C8722146B6F9B60357
:102A300079EE489A2FF0BEFEA6F8B603F4EEE89AB7
:102A4000F1EE10FA16DDB6F9B233B3B3002BB8BF0E
:102A50005B429BB207EE903AF8EEE77A78EEE98AAD
:102A600067EEA88A88EEA90AFDEEC07A17EE903AC2
:102A700019B209E038EE098AB4EEE88AF1EE10FAEC
:102A800007D421469FED110AA5F81013BDEC068B63
:102A900070BDB6F9B03378EEC88A3AEE488A07EED0
:102AA000903AF8EEE77A67EEA88A88EE880AFDEE9B
:102AB000C07A17EE903A19B2E6E7B6F9B033002BB8
:102AC000B8BF5B429BB207EE903AC5E7000000003A
:102AD00000007A4442F62803D2ED007A91ED006AB4
:102AE0000344D3ED925AD3ED956A26EEE77A67EE6A
:102AF000A57AA6EE257AE6EE267A81ED007AC2ED79
:102B0000007A704700F58040B0F9B23333B9B0F9BC
:102B1000B0030028B8BF404280B2704783EAE37038
:102B2000A0EBE37080B2704700207047704700BF91
:102B3000704700BF704700BF704700BF002070475C
:102B4000002070470020704701207047704700BF89
:102B50000020704700207047704700BF704700BFDB
:102B6000002070470D4B93F88C1F102912D80122BA
:102B70000B4B8A401340002B0BBF502058201022D3
:102B80001822084B93F891300BB142F0C00040F08E
:102B90000100704750201022F3E700BFB07C0030E6
:102BA00098000100B08C0030014B93F88C03704703
:102BB000B06C0030704700BF10B5044675F07EFD64
:102BC0000548BEF0DDF9054A034606212046BDE86A
:102BD000104075F05BBD00BF648C0030D414160843
:102BE00008B50B4870F0B4FB0346B7EE001A9E2000
:102BF000DFED080A93ED000A2FF070FDDFED067A95
:102C000020EE270ABDEEC00A10EE103A18B208BD39
:102C1000A88C0030000000000000C842014802F00B
:102C2000A3BD00BFB02C003000B583B008460191B1
:102C300018F098F838B10199054805F0F3FE002026
:102C400003B05DF804FB042003B05DF804FB00BF93
:102C5000CCB20030014802F08FBA00BFB02C003077
:102C6000014802F0DFBA00BFB02C0030074A40F63E
:102C7000C51310B540F6C53492F9482C002A08BF98
:102C80001C4673F0FFFF204310BD00BFB09C003016
:102C9000044B93F8893F13F0010301D118467047A4
:102CA00073F05ABEB07C0030044B93F8893F13F0A8
:102CB000010301D11846704774F054B9B07C00305C
:102CC00010B52DED048B84B00DF0A2FB04466846D0
:102CD00017F024FA694620460DF056FB164A92F882
:102CE0008C3F033B012B04D9002004B0BDEC048BC6
:102CF00010BD02F58052DDED017A02F58B53D2F85A
:102D0000080EB8EEE79A93ED008BBCF0E1FEB7EE4B
:102D1000C00A9FED0A7A38EE408BB7EEC88B78EE8A
:102D2000097A67EE877AFDEEE77A17EE903A18B2E5
:102D300004B0BDEC048B10BDB07C00300AD7233C3E
:102D400010B5044618F058F8204610BD08B54B6978
:102D5000012B03D0BDE8084073F0FABF7AF028FDDC
:102D6000024A062171F026F9032008BDE014160876
:102D70000D4810B590F891406CB9A0F5C040FFF730
:102D8000EFFA30B110F0F8FC012110F0BBFA204648
:102D900010BD042010BD7AF00BFD044A062171F02D
:102DA00009F9042010BD00BFB08C003008151608CA
:102DB000144B93F88C3F033B012B01D90020704743
:102DC00000B5114883B034F0E5FF9FED106AF1EED5
:102DD000046A9FED0F7AC0EE067A67EEA67AF4EEEB
:102DE000C77AF1EE10FA03D4FF2003B05DF804FBBC
:102DF000FCEEE77ACDED017A9DF8040003B05DF8B2
:102E000004FB00BFB07C0030189E00300000C842B8
:102E100000007F43084B93F849281AB913F8542C43
:102E2000120701D00520704793F89130002B0CBF9A
:102E300003200420704700BFB08C003030B589B04B
:102E400004460022164803A9B6F016FD10B3257CEF
:102E5000C5F048F9DDED037A00219FED127A0446B2
:102E60000591832267EE877A069110230021019253
:102E70002846FDEEE77A009304940E23ADF81E1069
:102E800004AA17EE904A8F21ADF81C4072F0C8FAE0
:102E900009B030BD204676F081FE09B030BD00BFDC
:102EA000706D00300000C842F0B5A94E8DB00446E8
:102EB0000DF0AEFAB6F8C4330546D80709D4990721
:102EC0005AD45A0700F1A5801B0700F1EE800DB01F
:102ED000F0BDA04B95EDC35AA3F10C02D3ED005AFF
:102EE00013ED036A183253ED026A9FED9B7A06F5E3
:102EF0002F53126825EE075ADFED987A93ED007A8A
:102F00000C33CDF82520622227EE277A1B689449DE
:102F100065EEA75A019221228DED087A26EE276AE6
:102F2000009266EEA76A91ED007A012103AA207C47
:102F300067EE277ACDF829308DF824101923C221A5
:102F40008DED045ACDED055A8DED066ACDED076A7B
:102F5000CDED037A72F064FA207C72F0E1F9074655
:102F6000207C73F015FA00F121039F42C0F0E98044
:102F7000B6F8C4339907A4D5D5EDC44A0222794BDB
:102F80009FED757ADFED757A64EE874A53ED025A4C
:102F900013ED037A53ED016A65EEA75A13ED066A45
:102FA00093ED005A66EEA76A8DF8242026EE276A74
:102FB0009A6825EE275AD96867EE277A6223CDF8FA
:102FC00029202122CDF825100193C2211923009236
:102FD00003AA207CCDED044A8DED055ACDED075AAC
:102FE0008DED036ACDED086ACDED067A72F018FA20
:102FF000207C72F095F90746207C73F0C9F900F146
:1030000021039F42C0F09D80B6F8C4335A077FF574
:103010005BAFD5EDC54A0322534B9FED4F7ADFEDF1
:103020004F7A64EE874A53ED025A13ED037A53ED5B
:10303000016A65EEA75A13ED066A93ED005A66EE33
:10304000A76A8DF8242026EE276A9A6825EE275A6B
:10305000D96867EE277A6223CDF829202122CDF89E
:1030600025100193C2211923009203AA207CCDEDE3
:10307000044A8DED055ACDED075A8DED036ACDED6D
:10308000086ACDED067A72F0CBF9207C72F048F92F
:103090000746207C73F07CF900F121039F4250D356
:1030A000B6F8C4331B077FF512AFD5EDD47A2120D3
:1030B000DFED2E6A62252E4B77EEA67A9FED277AFA
:1030C000D3ED304A93ED365AD3ED335AF1EE677AA9
:1030D00093ED346A25EE075AD3ED356A65EE875ACB
:1030E000D3F8E42026EE076AD3F8E01066EE876A8C
:1030F000042324EE877A0195CDF8252003AA8DF8C4
:10310000243019230090CDF82910C221207C8DEDA8
:10311000037ACDED047A8DED055ACDED065A8DED8D
:10312000076ACDED086A72F07BF9207C72F0F8F83E
:103130000546207C73F02CF900F121039D42BFF479
:10314000C6AE207C0DB0BDE8F04071F0D5B900BF2F
:10315000B06C003074980030E02E65420AD7233CF2
:103160005C9800306C990030649A00300AE81C4189
:10317000B09C00302DE9F04F0C4605462DED028B3A
:103180004B7AA5B0897AE27A43EA012343EA024303
:10319000562B18D8442B26D9453B112B40D8DFE8B5
:1031A00013F048009F003F003F003F003F003F00FA
:1031B0003F003F003F003F003F003F00B5003F00A1
:1031C0000B013F00C701764A1A4422F07F42012AD0
:1031D00026D8017C2246734825B0BDEC028BBDE8A1
:1031E000F04F69F081B8012B1AD1E5781F22002138
:1031F00016A8954228BF154639F13EF904F10C0195
:1032000016A82A4639F1EEF8179B9A0003D5189BA9
:103210009B0040F14E8225B0BDEC028BBDE8F08FE3
:103220002146284625B0BDEC028BBDE8F04F79F071
:1032300077BF5D4DE279B5F98C339A42EBD1E678F0
:103240001E22002116A8964228BF164639F114F90D
:1032500004F10C0116A8324639F1C4F89DF8622039
:10326000B5F98A339A42D6D19DF86500BDF974103C
:1032700003900B91BDF95E00BDF9721000900A91A8
:10328000BDF97000BDF96E10BDF96640BDF8632050
:10329000BDF860300494CDE90810BDF96C00BDF9AB
:1032A0006A10CDE90610BDF96800BDF95810059007
:1032B000A5F5804005F58055CDE90132BDF95C30BA
:1032C000BDF95A2004F0C6F9C4F00CFFC5F8980FF8
:1032D0007AF06EFA0446C4F005FFC4F8A4019AE738
:1032E000314EE279B6F98C339A4294D1C4F0FAFEA9
:1032F00006F58056034621462846C6F8983F25B075
:10330000BDEC028BBDE8F04F78F0C6B8E578272217
:10331000002116A8954228BF154639F1ADF804F1F1
:103320000C0116A82A4639F15DF89DF87E305A0640
:1033300000F1CD8113F0C00F7FF46DAFDFED1B0AFC
:10334000B7EE001A40F28A209DED1E0A2FF0C6F952
:10335000F6EE000AB0EE408A2FF01EF8002840F08A
:10336000F481B6EE000AB4EEC08AF1EE10FA40F332
:10337000198238EE400A0E4BD3ED797A30EE000A0E
:1033800020EE270A189812A9179C199A1A9B1390D5
:10339000084812941492159306F0B0F93BE700BF69
:1033A0007AFFFF00F8A80030B06C00300000000089
:1033B000B09C003008B30030E5783522002116A813
:1033C000954228BF154639F157F804F10C0116A8AB
:1033D0002A4639F107F8C84B93F88C2F042A09D0F4
:1033E000032A7FF418AF03F5405393F8CC37032B2F
:1033F0007FF411AF9DF88C500C2D3FF60CAF41F2CD
:103400008233EB40DB4313F001067FF404AFBDF8D9
:103410008840002314F0070904F0380704F4E07A28
:1034200004F4806804F4006B0F931093119328D177
:103430009FEDB26AA5F10802DDED186AA5F10C0353
:10344000DDED197A012A9DED177A66EE866A67EE40
:10345000C67AB3FA83F327EE067A4FEA5313CDED1B
:10346000106ACDED117A8DED0F7A40F27981002B43
:1034700040F07681EA1F022A40F26A81002B40F078
:1034800067810022129213921492DFB99FED9B6A1A
:10349000A5F10803DDED1B6ADDED1C7A012B9DED26
:1034A0001A7A66EE866A67EEC67A27EE067ACDED60
:1034B000136ACDED147A8DED127A40F202810C2D53
:1034C00000F0FF80B8F1000F40F012819DED200A5E
:1034D000A5F109069FED8A7ADFED887AB6FA86F6BD
:1034E00020EE070A760920EE270ABBF1000F40F014
:1034F0002981DDED210A9FED827ADFED807A60EE91
:10350000870A60EEA70AA30640F00881BAF1000F0F
:103510003FF481AEBBFA8BF0B8FA88F312AA0FA978
:1035200040095B09CDE90006764806F0D1F972E65C
:10353000E6783522002116A8964228BF164638F1B3
:103540009BFF04F10C0116A8324638F14BFF6A4A82
:1035500092F88C3F042B1BD0032B12D0022B7FF44C
:103560005AAEBDF88840660714D4DFED647A9DED4D
:10357000197A654B27EE277AB7EEC77A83ED007B81
:1035800049E602F5405292F8CC37032B7FF443AE64
:10359000BDF8884014F007014FF0000204F4E07613
:1035A000084618BF012114F038030F92109214BF7F
:1035B000012700271192002844D0B3FA83F3A00614
:1035C0004FEA531321D0002B3FF425AE00293FF4DE
:1035D00022AE002E3FF41FAE9FED486A12A9DDED2A
:1035E0001A6A9DED1B7ADDED1C7A66EE866A27EE7F
:1035F000067A444867EEC67ACDED126A8DED137AED
:10360000CDED147A05F0D8FF05E6002E3FF403AEA9
:103610009FED3A6A12AADDED1A6A0FA99DED1B7A99
:10362000DDED1C7A66EE866A27EE067A354867EE8F
:10363000C67ACDED126A8DED137ACDED147A05F0D0
:10364000D5FFE8E5DDE91789404649462FF088FCBB
:1036500000283FF4E0AD28460EAA9DF88C1079F0C2
:103660000BFD00283FF4D7ADDDED197A41469FED03
:10367000237A4A460E9B12A867EE877A0093FDEEE6
:10368000E77A17EE903A16F061FD12A80FA916F02E
:10369000FFFE00283FF4BFADA406B6D0002E3FF4D5
:1036A000BAAD002F3FF4B7AD0FA9164806F03AFFA8
:1036B000B1E5164825B0BDEC028BBDE8F04FBCF07B
:1036C00097BA13AA12A91248FFF704FAFAE6C4F04F
:1036D00009FD16AC0F4B03F59D65C3F8E4040FCC50
:1036E0000FC50FCC0FC594E8030085E8030092E5F1
:1036F0009FED090AF9E600BFB07C00300000C84227
:10370000E02E654208B30030109E0030F086003095
:10371000B02C0030B0AC00300000000047BBB9F165
:10372000000F25D0BAF1000F3FF475ADBBFA8BF353
:10373000B8FA88F212A921485B090096520906F0EE
:1037400095F868E5DFED1E0ADDE69FED1D0A19E636
:103750001C48BCF0B9F901460FA833F097FE90E67B
:1037600010AA0FA918480D93FFF7B4F90D9B81E635
:10377000B9FA89F3002F4FEA531308BF0023002B37
:103780003FF449ADBAF1000F3FF445ADBBFA8BF3FE
:10379000B8FA88F20FA900965B090848520906F0AA
:1037A000FBFE38E5094B38EE400AD3ED7A7A30EE6D
:1037B000000AF0EEE77A20EE270AE3E508B30030CE
:1037C00000000000AC950030B02C0030B09C003000
:1037D0000C207047014B93F88C0F7047B07C003081
:1037E00038B5122104462DED028B70F097FE20B9FA
:1037F00000252846BDEC028B38BDB6EE008A0720B6
:103800007DF026FCF7EE008A4C492046F0EE487A1F
:10381000E0EE087A38EEE70A76F0AAFF1221204699
:1038200070F07CFE0028E3D006207DF011FCA0EEB5
:10383000088A4349204638EEC80A76F099FF1221DB
:10384000204670F06BFE0028D2D03E4D20463E4907
:10385000D5F8B038002BB8BF03339B1000EE103AF8
:10386000B8EEC00A76F084FF1221204670F056FEB2
:103870000028BDD0B6EE008AB5207DF0E9FB3349C3
:103880002046F0EE487AE0EE087AB0EE670A76F06D
:103890006FFF1221204670F041FE0028A8D03C2086
:1038A0007DF0D6FBA0EE088A29492046B0EE480AF2
:1038B00076F05EFF1221204670F030FE002897D08F
:1038C00005F6B8032349204693ED000A76F050FF31
:1038D0001221204670F022FE002889D095F8BC38CD
:1038E00020461D4900EE103AB8EE400A76F040FF3F
:1038F0001221204670F012FE00283FF479AF95F8AF
:10390000BD382046154900EE103AB8EE400A76F070
:103910002FFF1221204670F001FE054600283FF4DB
:1039200067AF0F4B2046DFED0F7A93ED000A0E498B
:1039300080EE270A76F01CFF5BE700BF241516080F
:103940002C151608B08C00303415160840151608D2
:1039500048151608501516085C151608681516083F
:1039600070B400300000C84274151608272938B515
:1039700006D0442911D10125FFF732FF284638BD72
:103980001221044670F0CAFD05460028F6D0217CBD
:10399000044868F081FB284638BDBDE838407AF01D
:1039A000B5B800BFF8A80030024B93F8880FC0F3F9
:1039B00000107047B07C003091ED000AB5EEC00AEF
:1039C000F1EE10FA1EDBDFED1D7AB4EEE70AF1EE40
:1039D00010FA17D89FED1A7A10B5D1ED037A82B09C
:1039E0000C46F0EEE76AF4EEC76AF1EE10FA0FD477
:1039F000F7EE000AB0EE670A2EF0CEFC20B90220E6
:103A000002B010BD0220704794ED000AD4ED037A95
:103A1000FCEEE77A94ED027AD4ED010A0948CDED87
:103A2000007AFDEEC77A9DF80020CDED017A9DF970
:103A3000041004F07DFF002002B010BD0000B4436C
:103A400000000034CCB2003010B58B8B86B08C46B1
:103A5000B22B2BD0864608D8152B37D0732B10D11C
:103A600006B0BDE81040FFF7A7BFD12B36D0B3F5A5
:103A7000967F45D1264890F8913073B9042006B05E
:103A800010BD112B3CD102221021224804F066F80F
:103A90000028F3D0002006B010BD02220321A0F5BB
:103AA000C04004F05BF80028E8D0F3E7D1ED017ADC
:103AB000F5EEC07AF1EE10FAE0DD9FED170A174837
:103AC00027EE800ABAF06CFF0020E4E70222092109
:103AD000104804F043F80028DCD1CFE701F10C04D2
:103AE000EE460FCCAEE80F0094E803008EE803002A
:103AF00008489CE80E0007F0E5FF0028CAD1BDE7A2
:103B00006146704606B0BDE810407AF01FBC00BFA9
:103B1000B08C0030B02C00300000C842789E0030DD
:103B200008B50A4B93F88C3F033B012B01D90020C9
:103B300008BD0748BAF0B6FD2EF07EFD054B83FBAD
:103B40000023C017C0EBA310C0B208BDB07C00308A
:103B5000789E00301F85EB51F0B52DED048B9FED65
:103B6000338A8DB09FED320A0446324833F06EFC42
:103B700021EE081A304860EE089A20EE889A277CD9
:103B8000BDEEC11A11EE103A1DB2BAF08BFD07EE70
:103B9000900A2948F8EEE77A67EE887AFDEEE77A30
:103BA00017EE903A1CB2BAF069FD20EE080ADFED7C
:103BB000237AB4EEE70AF1EE10FA33D5FCEEC07AC0
:103BC00017EE903A9EB21E4B93ED008BA3F58B53EC
:103BD000D3F8080EBBF07CFFB7EEC00ADFED137A16
:103BE0001A230021B72238EE408B384608910991FC
:103BF0003E21B7EEC88BADF82850ADF82A40CDED88
:103C0000059A28EE278A8DED069AADF82C60CDE94D
:103C1000003205AA8DED078A71F002FC0DB0BDECF3
:103C2000048BF0BD4FF6FF76CDE700BF0AD7233CEB
:103C30009F0CB345CC960030789E003000FF7F4744
:103C4000109E003008B50F4B93F88C3F033B012BBF
:103C500001D9002008BD0C48BAF010FD9FED0B7A89
:103C6000DFED0B7A20EE070AB4EEE70AF1EE10FA68
:103C700005D5BCEEC00A10EE103A98B208BD4FF65A
:103C8000FF7008BDB07C0030789E00306F12833A20
:103C900000FF7F47F6EE007A91ED007AB4EEE77A06
:103CA000F1EE10FA01DC04207047012205210348DF
:103CB00008B5FEF7C5F9002008BD00BFFC94003030
:103CC0000020704700207047002070470120704797
:103CD00090F888308B4204D900EB8100D0F88C003A
:103CE00070470020704700BF90F888308B4204D99D
:103CF00000EB8100D0F88C0070470020704700BFB7
:103D0000FA207047014B93F88A037047B06C00307B
:103D100070B50446D0E90650266A40F4E05345F4F5
:103D2000F842E36146F4E053A2612B4A236292F821
:103D30008C1F02390E290FD8DFE801F00808080EA1
:103D40000E080E080E0E0E0E0E0E080040F4F8407F
:103D500046F4F843C4E9070392F8891FC80707D55A
:103D6000E16947F6084041F008012843C4E906012B
:103D700023F00803236292F8B01FC90702D543F06D
:103D800008032362154B93F8E034013B012B0BD859
:103D9000236AD4E9060143F4800340F4800041F42F
:103DA00080012362C4E9060192F8643ADB0712D568
:103DB0000B49D4E90623086842F4807243F4807307
:103DC000C4E9062338B1192160F05AFE18B1236AFC
:103DD00043F48073236270BDB07C0030B0AC00301F
:103DE00068B7003070B54FF450700D46164616F0A7
:103DF000FDFF044628B13246294673F0AFFD024B61
:103E00002360204670BD00BF08171608704700BF2A
:103E1000F0B500238FB00446009300F5E04393F91A
:103E2000483C002B40F0948000F5A0479FED4D7A70
:103E300007F67423D3ED007A67EE877ACDED007A2A
:103E40003322002101A804F5C04538F115FBA32356
:103E500004F5DC468DF8043095238DF80530C4F068
:103E600049F905F6D413CDF8070045F6F870CDF8FA
:103E70000B10D3F8B820D3F8BC302044CDF80F2075
:103E8000CDF813306FF064FAB7EE001A90ED000A27
:103E9000DFED350A9E202EF021FC10EE103AB6EE32
:103EA000061A95ED3B0AF4EE000A3020CDF81730E3
:103EB0002EF014FCDFED2D6A10EE103A46F6FC00F1
:103EC000CDF81B30204496EDD87BB7EEC77BC7EE0C
:103ED000267A17EE903ACDF81F30BBF0F9FD9FED32
:103EE000217A01A9B7F8663A20EE070AB5F8AC289E
:103EF000ADF82D304C2504F5D363D6EDDF7A10EE06
:103F0000100AADF83520FDEEE77A3322CDF8230014
:103F100048F28470204490ED0F7ABDEEC77A17EE18
:103F2000100AADF82B0094F8A90605FB00330098A1
:103F300017EE905ACDF82F0045F63010DB6A20447A
:103F4000ADF83350CDF827306BF03EF90FB0F0BD2F
:103F500047F648400122694604F5A047204469F02D
:103F6000D9F86DE70AD7233C000000000000C842E2
:103F700030B5044646F61C208BB09FED130A204452
:103F800033F064FA0AAACDED080A01AD8DED091AE5
:103F900004AB8DED070A12E9070085E807009DEDE7
:103FA000030A83E807002EF031FB42F62800294679
:103FB0008DED030A204409F04BFE0CF029FA0CF0B9
:103FC000B7F90BB030BD00BF9F0CB34570B50D46BF
:103FD00084B04FF6FF710646144608F0ADFB08B9F1
:103FE00004B070BD0023CDE90033CDE90233A32333
:103FF0008DF8003095238DF8013004238DF80230C0
:10400000C4F078F8CDF8030045F630100B461022C6
:10401000304469468DF80B50CDF8073003946BF0AF
:1040200069F904B070BD00BFF0B58BB01546064607
:104030000F462422002101A81C4638F11DFAA323B3
:104040008DF8043095238DF8053006238DF8063061
:10405000C4F050F82B682422CDF8070045F6301044
:1040600004936B683044CDF80B1001A90593AB683D
:104070006568069323688DF80F700793A368089509
:1040800009936BF0A1F80BB0F0BD00BF10B504466A
:1040900045F6301004F5A04304F58042204492F820
:1040A000182193F88C1F6BF06BFA42F6280020441D
:1040B0000CF0CCFB04F54470BDE810401DF0A2B933
:1040C000034645F63010A222014918446BF0D6BDD4
:1040D0006443160800207047704700BF00207047F7
:1040E0000020704700207047002070470020704774
:1040F0000020704700207047002070470020704764
:10410000704700BF704700BF002070470020704715
:104110000020704700207047002070470020704743
:104120000020704700207047002070470020704733
:10413000704700BF00207047002070470020704784
:104140000020704700207047002070470020704713
:1041500000207047704700BF0120704700F5A04065
:1041600090F88C0F704700BF494B00212DE9F043B8
:104170001F68054644F288348FB0F86A2C440368FF
:104180001B68984720465DF011F828B105F580437B
:10419000B3F98833012B78D0B86902AE3D49036882
:1041A0001B6898477DF09EFA5BF0EEFE01233146D6
:1041B0002046ADF808305FF05FFAB869364A036808
:1041C00036491B6898474FF0010831462046ADF844
:1041D00008805FF023FAC3F079FF04465EF06AFAC4
:1041E000BF693B68D3F80090C3F070FF2C49021BF5
:1041F00038462C4CC847002205212B485DF05EFF55
:104200005EF026FE294AB446138843F00803138063
:104210000FCCACE80F000FCCACE80F0094E80F0017
:104220008CE80F000022032130465DF047FF7CF050
:10423000C7FF17211E485EF05BFEB6EE000A1D4860
:104240005EF070FE44F24040314628445CF0CEFE01
:10425000C0B1002440F6D37243F628311323BDF8D1
:1042600008002944CDE90024134A5DF041FF44F2DF
:104270000401234639202944104ACDF804800094D3
:104280005DF036FF0FB0BDE8F08302AE9BE700BFE4
:10429000AC2C00304C581608705816087858160880
:1042A00080581608D8051608545A160830B700303A
:1042B0009C59160894581608FC731608D40B190854
:1042C000F8B50746A5F046FC164E07F1580007F66C
:1042D000D82496F0C9FA07F1740095F0FDFA07F6B4
:1042E0004C207AF0F5FB07F698550F4BC7F84C3A7F
:1042F00020467AF0EDFD44F82C6BAC42F8D1204614
:104300007CF072FF07F59E50C3F060FF41F28C40D5
:10431000384400F013FE384604495DF0DBF83846B7
:10432000F8BD00BF9059160894661608A45A1608DE
:104330002DE9F047B82786B0DFF88C8009260DF10B
:10434000030138461F4DDFF88490DFF884A07CF02D
:1043500095FD20B9701EC0B27CF0DAFA90B1093533
:1043600001360C2E2AD038F9027B0DF103013846B4
:104370007CF084FD0028F2D1701EC0B27CF0C8FA37
:104380000028ECD12C46093501E0AC42E8D014F805
:10439000011B484602F0C0FB0028F6D033465246C7
:1043A000142101A8C2F0D4FF07EE907A013601A8CB
:1043B000B8EEE70A5EF032FE0C2ED4D106B0BDE8AE
:1043C000F08700BFD4641608F2641608B02C0030E1
:1043D000A45816082DE9F04F89B0B526B6213B2226
:1043E00002AF3C230DF10608204CB946DFF880A04F
:1043F000DFF880B0ADF80460ADF80610ADF8082025
:10440000ADF80A300DF1030130467CF037FD30B9CC
:104410000DF10301B7F900007CF030FD50B9033411
:10442000C84507F1020702D109B0BDE8F08F38F99D
:10443000026BE7E72546033415F8011B504602F0EE
:104440006BFB10B9A542F7D1EAE79DF803305A4655
:10445000142103A80133DBB2C2F07AFF07EE906AA1
:1044600003A8B8EEE70A5EF0D9FDD9E7CC641608D8
:10447000B02C0030A45816082DE9F04345F65B2512
:1044800089B00124DFF8A4800646254F0544DFF8F3
:10449000A09015F9011B002906DDD8F80030D86975
:1044A0000368DB69BB4205D10134042CF1D109B0AA
:1044B000BDE8F083C9B20DF10B0298470028F3D094
:1044C0009DF80B007DF082F80028EDD19DF80B00DF
:1044D0007CF01EFA9DF80B3001330093B0B945F61D
:1044E000745023460F4A062130446FF063FD9DF857
:1044F0000B300D4A1421013303A8DBB2C2F028FFB0
:10450000BFEE000A03A85EF089FDCDE745F67450C2
:1045100023464A46042130446FF04CFDC4E700BFF7
:10452000D5400208B8581608A4581608AC2C00301C
:10453000EC5816082DE9F04F42F2867689B0012436
:1045400000250746DFF8BC900644DFF8BC80DFF8A2
:10455000BCA016F91520631E36F91510002A5FFA63
:1045600083FB06DDD9F80030D8690368DB69434571
:1045700006D101340335072CEBD109B0BDE8F08F2B
:10458000C9B20DF10B0298470028F2D042F28470B4
:10459000594638448BF04CF90028EAD09DF80B00BE
:1045A0007DF014F80028E4D19DF80B007CF0B0F900
:1045B0009DF80B3001330093B0B945F67450234693
:1045C0000E4A062138446FF0F5FC9DF80B300C4A7A
:1045D0001421013303A8DBB2C2F0BAFEBFEE000A19
:1045E00003A85EF01BFDC4E745F67450234652460F
:1045F000042138446FF0DEFCBBE700BF28591608E1
:10460000A4581608AC2C0030D5400208545916089E
:1046100000207047002070470069C0F340107047C9
:104620000F2904D82C2303FB01008C307047002095
:10463000704700BF002070470120704701F0E6B8C6
:1046400001F064BB00F038BE01F006BEF8B5444985
:1046500000F5A043434A06460160D3F81C0FC3F897
:10466000742D08B116F0D2FB3F4B43F684703360D3
:10467000304415F097FC06F5405393F82C2A42B9C4
:10468000D3F8284A2CB1204628F0A6FC204616F084
:10469000B3FB42F2F86042F2842442F26C253044CB
:1046A00034443544B3F0C2FE14F8043C083C3BB932
:1046B0002768384627B128F08FFC384616F09CFB57
:1046C000AC42F1D141F6707041F65C4441F6FC35E4
:1046D0003044344435447EF03BF82046183C28F002
:1046E0002DF8A542F9D141F27C4441F204471F4B19
:1046F00034443744C6F8803B14F8043C083C3BB9CA
:104700002568284625B128F067FC284616F074FB7A
:10471000A742F1D106F5756406F69C65243C204657
:104720006EF0ECFAA542F9D106F6046406F555657B
:10473000243C20466EF0E2FAA542F9D10C4A96F8E4
:10474000D431C6F8EC2043B9D6F8D0412CB120467C
:1047500028F042FC204616F04FFB3046F8BD00BF63
:104760001C641608545B17086C36170800DC160822
:10477000D88F1608F8B5684B0546002744F2281470
:1047800040F8043B44F2283689F096FA05F110000F
:1047900010F0ACFA05F1B00013F0FCFE05F518704E
:1047A00066F07AFB05F544701BF03AFF05F5D3601F
:1047B0000DF0E8FF05F63C0019F0AAFA05F538609F
:1047C0002AF00AFA41F6F0302C442E44284489F0AD
:1047D000CFF905F5E6505FF007FB41F6707028440D
:1047E0007DF09EFF41F6AC70284412F0C1FF42F20A
:1047F00068002844A5F0BAFB42F2F8602844B3F000
:1048000001FE42F21470284466F042FF42F28470C6
:1048100028448AF0AFFE05F5005342F2D8703F4AB3
:1048200083F8C87742F2C87328442B44136055F0CC
:104830004FF842F628003946284409F043FD42F675
:1048400050702844A3F03AFF42F65C70284491F07F
:1048500067F942F688702844A4F0A6FC43F61400D9
:104860002844ACF019FF43F62C102844ABF0ECFBC5
:1048700043F654102844AFF095F943F6D410284479
:10488000B2F0CEFD43F638202844B3F045FB05F5E1
:104890006A50A2F01DF843F62830284408F0AAF91F
:1048A00043F690402844B5F051F943F6E4701C49B2
:1048B00028445CF00FFE43F6FC7028442DF070F89D
:1048C00044F20400284496F051FD44F2C00028440C
:1048D000B4F0E8FE05F5804383F8187120461034E3
:1048E0006EF086FCA642F9D144F234300D4C2844D7
:1048F000B5F036F844F2583028446DF0FBFF2368D9
:1049000033B9284608495CF0E5FD28462560F8BD26
:104910000648C3F0B3FB00BF6C36170810C3003065
:10492000B8101908B0B7003034351708B06616084B
:104930002DE9F04F044644F2883544F284360027CE
:1049400025444FF6FF782DED028B87B0FFF712FF5D
:10495000EB4BA21905F15600236045F6EC260392B5
:10496000BBF0C2F805F158002644BBF0BDF805F1D4
:104970005A00BBF0B9F805F15C00BBF0B5F805F1E1
:104980005E00BBF0B1F805F16000BBF0ADF805F1D9
:104990006200BBF0A9F805F16400BBF0A5F805F1D1
:1049A0006600BBF0A1F805F16800BBF09DF805F1C9
:1049B0006A00BBF099F805F16C00BBF095F805F1C1
:1049C0006E00BBF091F805F17000BBF08DF805F1B9
:1049D0007200BBF089F805F17400BBF085F805F1B1
:1049E0007600BBF081F804F58840BBF07DF805F156
:1049F0007A00BBF079F805F17C00BBF075F805F1A1
:104A00007E00BBF071F805F18000BBF06DF805F198
:104A10008200BBF069F805F18400BBF065F805F190
:104A20008600BBF061F805F18800BBF05DF805F188
:104A30008A00BBF059F805F18C00BBF055F805F180
:104A40008E00BBF051F805F19000BBF04DF805F178
:104A50009200BBF049F805F19400BBF045F844F230
:104A6000404004F5A0452044FFF72AFC44F2B83149
:104A700045F63010214420446AF07EFA45F6402085
:104A80002044BBF055F895F8643A05F52762A5F87F
:104A9000667A23F00303C5F8687AC5F86C7A45F6A0
:104AA000782085F8643A00232044136005F67422C8
:104AB00013606EF09DFB45F6882020447DF028F9B8
:104AC000904B45F62C30C5F8044BC5F8083B8E4B8F
:104AD0002044C5F80C4BC5F8103B8C4BC5F8144B63
:104AE000C5F8183B15F01AFB45F64830204415F080
:104AF00015FB45F66430204415F010FB844B04F59B
:104B0000B740A5F87C8BC5F8783B15F007FB814BC7
:104B1000304681491E605CF0DDFC45F63050A5F85A
:104B2000248BA5F8408B45F69856204459F020F97F
:104B3000C5F8707D45F6FC57784B26442744C5F8E8
:104B4000743D3046143675F073FBB742F9D11E221E
:104B5000002340F2CC60C5F8202FA5F8243F16F0C2
:104B60004FF9034645F62870C5F81C3F2044C2F0B3
:104B70001BFB45F66C702044C2F016FB684B1A68AC
:104B8000002A00F08C81674B45F6B4794FF4C87168
:104B900004F5C047C5F8743DA1441323484685F881
:104BA0008C3FBDF067FE604B604AC5F8B43F604B78
:104BB000C7E9A2221A680292002A40F07B819FED89
:104BC0005D8A4FF07E525C494846C3F8009005F676
:104BD000B473C5F8B41F46F6D41BC3F84C2346F68D
:104BE00018185649A34483EDD48A46F6FC0A5CF0B3
:104BF00071FC534B46F220304FF40071059304F5DD
:104C00000046504B20440494009306AB13E90C007B
:104C10000EF0ACFE46F64C002044BEF0D9FC029BE0
:104C200046F6C00087F8BD38474B2044C7F84C38DB
:104C300015F074FA42F628014FF0010C07F608133C
:104C400007F6D40007F6FC02214487F8D0C8B0EE7E
:104C5000480A80ED008A80ED018A80ED028A08EB27
:104C6000040082ED008A82ED018A82ED028A83EDE2
:104C7000008A83ED018A83ED028A029AC7F814192B
:104C800004F5DC4709F06AFA039A4B4608EB040185
:104C90005846B5F0B1F84B460AEB040208EB0401A4
:104CA0003846CDF800B0B7F0E3FD47F2C8103B46F8
:104CB00008EB04020AEB04012044CDF800B0B9F07F
:104CC000FFFC3B4608EB04020AEB040104F5F54047
:104CD000CDF800B0BAF06AFC47F6D0203B4608EBAE
:104CE00004020AEB04012044B9F024F947F63830F5
:104CF0004FF40041204410F043F947F6B83025E066
:104D00001C6416083D460208414602084546020852
:104D10000000FFFF40B60030A0EC1608545B1708F7
:104D2000ACBB00300418160870491908100D16089D
:104D3000F0C9003000000000C4471908CC4619082B
:104D400049460208CC141608140E160820447DF0BB
:104D500003FE47F6344020445EF03EFD47F64840EF
:104D6000204468F035F8029F2C2206F2E4403946D0
:104D700037F182FB5149524B48F2105019602044E0
:104D80000B7C4BB13B4601339BB203EB830201EB3F
:104D90008202127C002AF6D14A494B4A0B801768DE
:104DA0004A490B80002F40F08280106048F22C505E
:104DB000C6F820752044C6F82475C6F8280502F008
:104DC00033FE434B48F26850C6F82C35204402F0BD
:104DD0002BFE404B48F2A450C6F86835204402F040
:104DE00023FE3D4B48F2E050C6F8A435204402F0C3
:104DF0001BFE3A4B48F21C60C6F8E035204402F036
:104E000013FE374B48F25860C6F81C36204402F0B7
:104E10000BFE344B48F29460C6F85836204402F03A
:104E200003FE314B48F2D060C6F89436204402F0BD
:104E3000FBFD2E4B48F20C70C6F8D036204402F031
:104E4000F3FD2B4B48F24870C6F80C37204402F0B3
:104E5000EBFD284B48F28470C6F84837204406F032
:104E600017FB48F2CE7348F2D672A6F8CC772344EB
:104E700022441F70023303F8017C9342F9D195F864
:104E8000AC3F1D4A43F00103116885F8AC3F59B9A6
:104E90002046146007B0BDEC028BBDE8F08F45F6EC
:104EA000745222441A606EE61448C3F0E7F81448BE
:104EB000C3F0E4F81348C3F0E1F800BF545B1608F0
:104EC00058B7003054B70030F4B6003024B7003083
:104ED000786D1608386F16081C6B1608706B16086C
:104EE000886C1608286D1608E46E1608D86C16082B
:104EF000886F1608946E1608A82C003004671608F0
:104F0000E8661608C466160810B5084CC2F0A4FC82
:104F1000074B024620461A60FFF70AFD2046054A65
:104F20000549BDE8104033F105BB00BFB02C00308F
:104F3000AC2C0030406001304D46020810B50446EC
:104F400002495CF0C7FA204610BD00BFD4671608BE
:104F500070B5B82482B01A4D00F130060DF107018A
:104F600020B27BF08BFF08B39DF807301F2B24D8AD
:104F700003EB83032968D6ED006A002201EB83006E
:104F800031F82310438807EE901A5B1AB8EEE77ADF
:104F90009BB207EE903AF8EEE77AA7EEA67AFCEE1F
:104FA000C77A17EE903A99B27BF032FA01340436A0
:104FB000A4B2BE2CD2D102B070BD00231B88FFDE8C
:104FC00048BC0030F0B5B82483B01A4E054600F155
:104FD00030070DF1070120B27BF050FFD8B19DF8EA
:104FE00007301F2B22D8316803EB830301EB8302C8
:104FF00031F82310538892885B1A521A9BB207EE3D
:10500000902AB8EEE77A07EE903AF8EE677AC7EEA4
:10501000276AC7ED006A01340437A4B2BE2CD8D188
:10502000284603B0BDE8F040FFF792BF00231B887D
:10503000FFDE00BF48BC0030052900D9704710B51D
:1050400000EB8104B7EE001A6020DFED060A94ED54
:105050000C0AD4ED007A30EE270A2DF03FFB84EDE8
:105060000C0A10BD00000000052900D9704710B5DA
:1050700000EB8104B7EE001A6720DFED060A94ED1D
:105080000C0AD4ED007A30EE670A2DF027FB84ED90
:105090000C0A10BD00000000052903D800EB8100B8
:1050A00000230363704700BF052904D84FF07E53E7
:1050B00000EB810003637047052910D800EB8100E5
:1050C000DFED077A90ED0C7AB4EEE77AF1EE10FAA4
:1050D00003D54FF07C53036370470023036370478D
:1050E000CDCCCC3E052911D800EB8100DFED087A4C
:1050F00090ED0C7AB4EEE77AF1EE10FA03DB4FF0A4
:105100007C53036370474FF07E530363704700BFC7
:105110009A99193F052904D84FF07C5300EB810080
:105120000363704730B505468DB042F628046846E3
:105130002C4414F0F3FF04A814F0F0FF6946204655
:105140000BF022F908B90DB030BD04A920460BF0D0
:1051500049F90028F7D0059B08A8019314F0DEFF59
:1051600008A920460BF03EF90028ECD069462046FD
:105170000AF03CFDE7E700BF70B5044642F628059B
:1051800088B00E462544684614F0C8FF6946284694
:105190000BF0FAF808B908B070BD4C2194F8A926B4
:1051A00004F5D363DDED017A9FED157A04A801FBC8
:1051B0000233F8EEE77AD3ED0B6AE6EEC77AFDEE3E
:1051C000E77ACDED017A14F0A9FF04A928460BF087
:1051D00009F910B9002008B070BD694628460AF0E8
:1051E00005FD0028F6D0002ED5D004F50054304639
:1051F00094F89C3A43F0020384F89C3ACBE700BF52
:105200000000C84200F5005292F89C2AD20708D448
:1052100000F5C04393F8911009B1FFF783BFFFF782
:10522000ABBF7047F0B5044642F6280585B00E4680
:1052300025441746684614F071FF694628460BF06E
:10524000D1F810B9002005B0F0BD314628460AF06B
:10525000CDFC0028F6D0002FF5D004F500543846D8
:1052600094F89C3A43F0020384F89C3A05B0F0BDF0
:1052700030B585B004460D46684614F04FFF42F63F
:105280002800694620440BF0ADF808B905B030BDE0
:105290006846294615F018F99FED057BB4EEC70B5B
:1052A000F1EE10FACCBF0120002005B030BD00BFE8
:1052B00000000000006AE8400A4A10B5137804466E
:1052C00048F21C6043F080032044137003F072FD29
:1052D00000B110BD204608220221BDE8104002F0B6
:1052E0003DBC00BF98B600302DE9F04101F1080344
:1052F00088B005460E4604AC05F5C0470FCB84E8E0
:105300000F00134305D1D7F8C8380693D7F8CC3827
:105310000793059B73B1002348F21C602146C7F830
:1053200014332844B388A7F8123303F0A5F908B062
:10533000BDE8F08146F6C008204614F045FF03AAF8
:10534000A8440146404614F04BFF58B9D7F8C4189A
:105350004046019114F038FF01990246204614F0AE
:1053600015FFD8E7039920460191F3E770B58CB09B
:105370000C46064604AD284614F0D0FE23690BB94E
:10538000636963B31F4B002204F108011A700FC94F
:1053900085E80F0046F6C00003AA0321304414F04C
:1053A0001FFF78B906F5C04301222846D3F8C41878
:1053B00014F0ECFE48F21C602946304403F05CF91E
:1053C0000CB070BD08AA0321284614F009FF00287C
:1053D000E8D003220399284614F0D8FEEAE7012218
:1053E00006F5C041074808AC027020460092D1F88B
:1053F000CC28D1F8C81814F0A9FE94E80F0085E86D
:105400000F00D7E788B4003070B508318EB005467C
:1054100006AC0FC984E80F00134327D0079B3BB1AC
:1054200048F21C602146284403F026F90EB070BDF6
:1054300046F6C006204614F0C7FE0AAA2E440146CE
:10544000304614F0CDFE68B905F5C0433046D3F8B8
:10545000C418019114F0B8FE01990246204614F0D8
:1054600095FEDDE70A9920460191F3E747F2C8105F
:10547000002303A92844039304930593B9F0B2F9D8
:10548000022203A90AA815F07FFADDE90C23CDE971
:105490000823C3E7F0B501F1080389B00C460646BE
:1054A00004AD0FCB85E80F00134307D106F5C043C9
:1054B000D3F8C828D3F8CC38CDE90623059BBBB177
:1054C000227EA388D2074FEA132302D503EB83037E
:1054D0005B0007EE903A227A48F21C602946B8EE4B
:1054E000670AC2F34002304403F0F4F809B0F0BD9B
:1054F00046F6C007284614F067FE03AA3744014663
:10550000384614F06DFE50B103992846019114F00D
:105510005BFE01990246284614F038FED0E706F5F6
:10552000C0433846D3F8C418019114F04DFE0199D8
:105530000246284614F02AFE6AF064FF0222152172
:105540006AF082FCBCE700BF70B504460D4682B02D
:1055500004F5C046C2F0C6FDC6F81C03D5ED027ABC
:10556000F5EEC07AF1EE10FA17DD9FED147A67EED2
:10557000877AFCEEE77A17EE903AC6EDC67A1049C4
:1055800045F674500F4AA1FB0313204406219B09E2
:1055900002B0BDE870406EF00DBD95F009FE00232D
:1055A000009395F90E3095F90D2095F90C1095F0B2
:1055B000F7FC0346C6F81803E1E700BF00007A4491
:1055C000D34D621044681608F8B500F5E04393F82F
:1055D000CC3113F0010418D0154A00F5C047054638
:1055E0000E46537843F001035370D7F814337BB160
:1055F000C2F078FDD7F81433B7F81223C31A0D4858
:10560000A0FB0313B2EB931F07D900242046F8BD7B
:10561000C2F068FDC7F81403EAE745F67450338812
:10562000054A062128446EF0C5FC2046F8BD00BF9F
:1056300098B60030D34D621054681608F0B5154E78
:1056400087B00446357865B1012D07D100F5E040FB
:1056500090F8CC0100F0010007B0F0BD012007B0C8
:10566000F0BD00F5E04393F8CC2112F00100F3D037
:1056700001272B4602A80097D1E9041214F066FD19
:1056800048F21C6002A9204402F0F6FF2846377059
:1056900007B0F0BD88B4003000F5004370B593F852
:1056A000CC3784B00C46012B1ED00B7907EE903A14
:1056B0000B7E9B07F8EE677A11D4274BDFED276A44
:1056C00093ED006A86EE267AB0EEC77AB4EEE77AFA
:1056D000F1EE10FAACBF0120002004B070BD9FEDC8
:1056E000207A67EE877AE8E700F5E043054693F80D
:1056F000CC3113F00100F0D001AE002304F108001A
:10570000314601930293039314F0C2FEDDED037A58
:105710009FED147AF0EEE77AF4EEC77AF1EE10FA24
:1057200012D423694BB963693BB946F6FC0028449F
:10573000BAF0CCF903C886E8030048F21C6028449C
:1057400003F0A0F80020C8E746F6FC002844BAF0B1
:10575000BFF98DED030AE4E7C8A70030DB0FC940AD
:105760000000803B0000003400F5A04208B592F82C
:105770008C2F0B46042A09D0032A01D0002008BD33
:1057800000F5004090F8CC27032AF7D15A88102A58
:105790000DD0732AF2D15A7C93F91010D3ED030A7D
:1057A00093ED020A054803F0C3F8012008BD03F198
:1057B00008010348BDE8084004F062BECCB20030E6
:1057C00008B3003010B58B8882B00446012B05D099
:1057D0000B6953B94B6943B9CB6833B900212046F3
:1057E00002B0BDE81040FFF7C7BC08312046019168
:1057F000FFF73EFD019908B102B010BD02462046F8
:1058000002B0BDE81040FFF70DBD00BF70B50C46FB
:105810004FF48071054606F08FFF002877D104F120
:105820000806304614F0D0FC012864D0032813D1B8
:10583000E368002B75DB6388732B28D85B2B14D8A7
:10584000A3F1100291B2052974D8052A72D8DFE8B5
:1058500002F07A80868C9AA445F674508D4A042111
:1058600028446EF0A7FB002070BDA3F15C02172A4C
:1058700060D8DFE802F0C9CD5F5F5F5F5F5F5F5FA9
:105880005F5F5F5F5F5F5F5F5F5F985FADBDCD2B09
:1058900015D8B12B4ED9A3F1B2021B2A4AD8DFE8A2
:1058A00002F0C3BD4949494949494949494949491A
:1058B000494949494949494949D7494949DDDE2BBF
:1058C00038D1DFED757A4FF47A7194ED041A48F20D
:1058D0005860D4ED030A94ED020A2844A38821EE0F
:1058E000271A60EEA70A20EE270A03FB01F104F055
:1058F000C5FC012070BDE368002B9CDD45F67450AB
:10590000664A042128446EF055FB002070BD45F620
:10591000EC2145F6301022462944284469F06CFEFB
:105920007DE745F674505E4A042128446EF042FB40
:10593000002070BD45F674505A4A042128446EF088
:1059400039FB002070BD28462146FFF7CDFC012021
:1059500070BD28462146FFF757FD012070BD28463F
:105960002146FFF797FD012070BD28462146FFF72D
:105970004BFD05F5C04500230120C5F81433A3886D
:10598000A5F8123370BD42F68C2148F21C60294400
:10599000284402F071FE012070BD28462146FFF721
:1059A000E5FC012070BDC2F09DFB05F5C045034636
:1059B0009FED3D7A0120C5F8F838D4ED027A67EE04
:1059C000877AFDEEE77A17EE903AC5F8F43870BDA5
:1059D000D4ED027A05F5C0459FED2F7A012067EEE0
:1059E000877AFDEEE77A17EE903AC5F8F43870BD85
:1059F000627C94F91010D4ED030A94ED020A2B484E
:105A000002F096FF012070BDA388CBBB012070BDC2
:105A100028462146FFF798FD012070BD2846214603
:105A2000FFF7D0FE012070BDD4F8093007EE903AA0
:105A3000F5EEC07AF1EE10FAE8DD9FED170A47F2B5
:105A4000C81027EE800A2844B8F0AAFF012070BDD4
:105A50003146164802F0E6FF012070BD05F5E0432F
:105A600047F6B830002294ED041A2844D4ED020A17
:105A700094ED030A93F8291C7CF0E8FF012070BD27
:105A800048F21C64601904F005FC601903F00EFB79
:105A9000012070BDAC6816080000C842686816088E
:105AA00088681608BC68160800007A44CCB200303A
:105AB00038B54B880446152B15D9732B27D85B2B8B
:105AC00013D9A3F15C02172A0FD8DFE802F0858A08
:105AD0000E0E0E0E0E0E0E0E0E0E0E0E0E0E0E0EE6
:105AE0000E0ED70EE9C00F2B08D845F67450844A25
:105AF000042120446EF05EFA012038BD113B042BD6
:105B000000F2F980DFE803F0769F78989400A3F123
:105B1000B20291B22C29E8D82C2AE6D801A151F87A
:105B200022F000BFDF5B0208DF5B0208EB5A0208CD
:105B3000EB5A0208EB5A0208EB5A0208EB5A020829
:105B4000EB5A0208EB5A0208EB5A0208EB5A020819
:105B5000EB5A0208EB5A0208EB5A0208EB5A020809
:105B6000EB5A0208EB5A0208EB5A0208EB5A0208F9
:105B7000EB5A0208EB5A0208EB5A0208EB5A0208E9
:105B8000DF5B0208EB5A0208EB5A0208EB5A0208E4
:105B9000DF5B0208DF5B0208EB5A0208EB5A0208DF
:105BA000EB5A0208EB5A0208EB5A0208EB5A0208B9
:105BB000EB5A0208EB5A0208EB5A0208EB5A0208A9
:105BC000EB5A0208EB5A0208EB5A0208EB5A020899
:105BD000EB5A0208DF5B02088B88002B75D101208D
:105BE00038BD04F5C044C2F07DFAD4E9C632801A4B
:105BF000984276D8002038BD00F5E04393F8CC31C8
:105C0000DB07F7D500F5C045D5F81433002B6DD070
:105C1000C2F068FAD5F814133A4B401AB5F81223BB
:105C2000A3FB0013B2EB931F94BF0120002038BDEB
:105C3000BDE83840FFF702BD00F5E04090F8CC0128
:105C400000F0010038BDBDE83840FFF725BD04F580
:105C5000C04595F8D038032B3ED104F50050D5F857
:105C6000E838D0F8200AC01A2CF06EFC0028B8BF23
:105C70004042C828CCBF0020012038BD04F5C045F3
:105C8000C2F030FAD5F8F828D5F8F438801A23EAAB
:105C9000E3739842AED900230120C5F8F43838BD2B
:105CA00047F2C81004F5C0452044B8F0E7FCD5F829
:105CB000F43823EAE37307EE903AF8EEE77AB4EEAD
:105CC000E70AF1EE10FA95D5E5E748F21C602044AA
:105CD000BDE8384004F0F0BA03210B4803F03AFF66
:105CE000BBE700230120C4F8183338BDC2F0FAF92D
:105CF000C5F814038CE7BDE83840FFF765BC00BF6A
:105D0000D0681608D34D6210CCB2003000F5A04325
:105D100070B593F88C3F032B02D00026304670BD3F
:105D200004460D46FFF7C4FE06460028F5D045F6AA
:105D300074502988204474F047FAEFE708B501222F
:105D4000034B1A70C2F0C2F9024B186008BD00BFC5
:105D50008AB4003090B40030014B00221A707047B2
:105D60008AB4003038B500F5804595F99E3303B903
:105D700038BD0446C2F0B6F9D5EDE87A034604F51D
:105D8000D362F8EEE77A92ED097AF4EEC77AF1EE93
:105D900010FA22DC174A126802F5FA62824204F510
:105DA000A04205D292F8AC1F41F0200182F8AC1F4E
:105DB00092F8AC2F9206DBD50F4947F230520868B3
:105DC00002449A42D4D245F674500B600B4A042127
:105DD0002044BDE838406EF0EDB804F5A044054815
:105DE000054994F8AC2F03606FF345120B6084F8FB
:105DF000AC2F38BD9CB40030A0B40030EC6816085D
:105E000038B500F5804595F99F3303B938BD044690
:105E1000C2F068F995F9A43304F5D36207EE903A1D
:105E2000034692ED0A7AF8EEE77AF4EEC77AF1EEDD
:105E300010FA22DC174A126802F5FA62824204F56F
:105E4000A04205D292F8AC1F41F0400182F8AC1F8D
:105E500092F8AC2F5206D9D50F4947F23052086854
:105E600002449A42D2D245F674500B600B4A042188
:105E70002044BDE838406EF09DB804F5A0440548C4
:105E8000054994F8AC2F03606FF386120B6084F819
:105E9000AC2F38BDA4B40030A8B40030086916088F
:105EA00070B500F5A04494F8523A2BB100F5804645
:105EB000054696F99C336BB994F8AC3FD90638D4B3
:105EC000002294F8AC3F234962F30413CA7484F8A7
:105ED000AC3F70BD1F4B0122DA74C2F003F9D4F855
:105EE000902F44F620631344834229D394F8AC3FA7
:105EF000DA06EED443F0100384F8AC3F6AF082FA7D
:105F000001221B2169F0A0FF94F8AC3FDB06E0D52D
:105F100096F99C33022BDCD105F5C04393F8913000
:105F2000002BD6D028461D220921BDE8704001F083
:105F300015BE6AF067FA00221B2169F085FFBFE7F2
:105F4000C4F8900F45F67450034A022128446EF0BD
:105F500031F8CBE778B600302869160838B5044622
:105F60000D46C2F0BFF804F5A0443DB9D4F89C3FFB
:105F7000C4F8A00F0BB9C4F89C0F38BDD4F8A03FEB
:105F8000C01A6428F9D90023C4F8A03FC4F89C3F84
:105F900038BD00BF2DE9F0410446C2F097F8314BFF
:105FA0000546B4F8B6221988914208D02E492F48E8
:105FB0001A800B780560002B43D1BDE8F0812A4E92
:105FC00033780BBBDFF8AC8098F80030002BF4D0AE
:105FD000264F274A3B68C31A9342EED904F5C043C3
:105FE000012293F891303270002B34D16AF00AFA12
:105FF0000122132169F028FF98F80030002BDCD033
:106000003378002BD9D004E01A4B1B78002BD4D066
:10601000164F3B68184AEB1A9342CED904F5C04399
:106020003D6093F89130002BC7D045F6B475002140
:1060300025442846BAF060FF2846BDE8F041BCF090
:106040007BBF00240C706AF0DDF922461321BDE805
:10605000F04169F0F9BE45F6B4702044B9F078FE1D
:10606000C4E700BF8CB4003089B4003090B4003075
:1060700080841E008AB4003040420F0038B500F51D
:10608000A04595F8893FDC072DD595F8B03F13F072
:10609000010F95F8AD3F27D1DA0724D443F001036F
:1060A000044645F674501C4A85F8AD3F0221204451
:1060B0006DF080FF6AF0A6F903221A2169F0C4FE90
:1060C00095F88C3F022B08D0092B06D0134BD3F840
:1060D000280503689B68984728B11C221321204695
:1060E00001F03CFD78B138BDD907FCD56AF08AF9DA
:1060F00000221A2169F0A8FE95F8AD3F6FF3000366
:1061000085F8AD3F38BD46F64C00012217212044EA
:10611000BDE83840FBF794BF38691608B0AC0030D2
:1061200070B500F580468AB0044696F9BC5385B335
:10613000002207AD05AB42F6280006A9079201939D
:10614000204404AB0892099203AA009509F0E0FDEF
:10615000284631F01FFED6EDF07AF4EEC07AF1EE6B
:1061600010FA06DD9DED067AF4EEC77AF1EE10FA2C
:106170004EDCC1F0B7FF354B1B6803F5FA6398425C
:1061800017D304F5A04595F8AC3F5A071ED50AB0C1
:1061900070BD04F5A044C1F0A5FF2C4A94F8AC3FB3
:1061A0002B4965F382031060CD7384F8AC3F0AB0CD
:1061B00070BD04F5A044264A002194F8AC3FD17389
:1061C0006FF3820384F8AC3F0AB070BD43F0040360
:1061D0001F4A85F8AC3F0123D3736AF013F90222FA
:1061E000102169F031FEC1F07DFFD5F8A82F44F6EB
:1061F0002063134498421BD896F9BC33022BC6D1B6
:1062000046F64C00012218212044FBF719FFBEE797
:1062100004F5A044C1F066FF00250C4A94F8AC3F99
:106220000B496FF382031060CD7384F8AC3FAEE787
:10623000C1F058FF034645F67450064A0421C5F8DC
:10624000A83F20446DF0B6FED6E700BF94B40030FE
:1062500078B600304C69160838B5144605466AF021
:10626000D1F80122062169F0EFFD022C08D0032CA1
:106270000FD1284604220921BDE8384001F06EBC48
:1062800046F64C00012207212844BDE83840FBF7C0
:10629000D7BE38BD38B500F58045044695F9A6331C
:1062A00043B900F5A04393F8AC2F6FF3000283F8D5
:1062B000AC2F38BDC1F016FF04F5A04307EE900ADD
:1062C00095EDEA6AD3F8982FB8EE677ADFED186A91
:1062D00007EE902AF8EE677AE6EE267AB4EEE77AD1
:1062E000F1EE10FADFD493F8AC2FD107E1D442F0ED
:1062F000010283F8AC2F6AF085F801221C2169F0B5
:10630000A3FD45F674500B4A022120446DF052FE65
:10631000204600F0D3FB95F9A633022BC9D146F6EF
:106320004C0001221D212044BDE83840FBF788BE07
:1063300000007A4454691608F8B500F5804797F9CB
:106340009D332BB100F5A0460446D6F8185F05B979
:10635000F8BDC1F0C7FE40F6C313451B9D4242D9AC
:10636000D6F8943F47F23052C31A93422FD896F88A
:10637000AC3F9A07ECD404F5C04595F89120002A6B
:10638000E6D043F0020386F8AC3F6AF03BF8012206
:10639000082169F059FD97F99D33022B49D0032B51
:1063A0002CD0042BD4D195F89130002BD0D00522DD
:1063B0000921204601F0D2FB0028C9D146F64C0045
:1063C000012219212044BDE8F840FBF739BEC6F888
:1063D000940F45F674501B4A0421B7F98C332044BE
:1063E0006DF0E8FDC3E796F8AC3F99071AD496F82C
:1063F000AC3F6FF3410386F8AC3FF8BD95F89130A0
:10640000002BA5D005220221204601F0A7FB002881
:106410009ED146F64C0001221A212044BDE8F840E6
:10642000FBF70EBE69F0EEFF0022082169F00CFDBB
:10643000DDE746F64C00012212212044BDE8F84079
:10644000FBF7FEBD6869160870B50446C1F04AFE48
:1064500004F5C04304F5A04593F89120002A3FD0ED
:1064600004F5804696F9BD23D2B395F88C2F012A06
:1064700036D0A2F11302B2FA82F2520982BB03F6BD
:10648000D413DFED2A6AB3EE0E7AD3ED2D7A67EEE0
:10649000A67AF4EEC77AF1EE10FA2AD9244B1B68DB
:1064A00003F5FA6383421AD8D5F8A42F44F6206383
:1064B000134483422FD395F9AC3F002B0FDB95F8A3
:1064C000AC3F43F0800385F8AC3F69F09BFF0122AD
:1064D0000C2169F0B9FC96F9BD33022B12D070BDC6
:1064E00095F8AC3F124A6FF3C713106085F8AC3FC4
:1064F00070BD95F8AC3F0E4962F3C713086085F88C
:10650000AC3F70BD46F64C0001220C212044BDE892
:106510007040FBF795BDC5F8A40F45F67450054AC9
:10652000042120446DF046FDC5E700BFE02E654222
:1065300098B400308469160800F5804310B593F9CB
:10654000A5330446012B0AD0022B13D046F64C008B
:10655000012215212044BDE81040FBF771BD0B223C
:10656000102101F0FBFA78B1094A137843F00803CF
:10657000137010BD0B22092101F0F0FA044A1378C0
:1065800043F00803137010BD0B2202212046F3E7ED
:1065900098B6003038B500F5A045044695F8AC3FF4
:1065A00043F0080385F8AC3F69F02CFF0122172166
:1065B00069F04AFC95F8643ADB0703D5044802F019
:1065C0006BFA20B92046BDE83840FFF7B5BF38BDAB
:1065D000CCB2003070B500F5A045D5F8A04FD5F885
:1065E0009C2F95F88C3FA41A033BB4F57A7F8CBF9F
:1065F00001240024012B95F8AC3F88BF0024C3F38D
:10660000C003A34229D0E4B1064645F67450164AA9
:10661000022130446DF0CEFC95F8AC3F43F0080306
:1066200085F8AC3F69F0EEFE0122172169F00CFC01
:1066300095F8643ADB0711D43046BDE87040FFF7A7
:106640007BBF69F0DFFE2246172169F0FDFB95F85C
:10665000AC3F64F3C30385F8AC3F70BD034802F060
:106660001BFA0028F9D1E7E794691608CCB200308C
:1066700038B500F5C04393F8913003B938BD00F543
:106680008043084893F8445095F096F9044608B9B9
:10669000002DF3D069F0B6FE22460921BDE838404E
:1066A00069F0D2BBB46C003070B546F6FC0586B01C
:1066B00000210446054404F5C0462846B9F0A8F96F
:1066C00002A813F02BFD42F6280002A9204409F08D
:1066D0005BFE2846DDE90423C6F8CC38C6F8C82896
:1066E000B9F0E8F9830611D52846B9F0F1F9BDEE05
:1066F000C00A284610EE103AC6F8C438B9F0F0F9CE
:10670000BDEEC00A10EE103AA6F8AC3806B070BD67
:1067100003461F2900F28D80DFE801F08B837F7B29
:1067200077736F6B67635F5B57534F4B4744403CD6
:106730003834302C2824201C1814108744F21A40B6
:106740001844704744F218401844704744F2164009
:106750001844704744F214401844704744F2124001
:106760001844704744F210401844704744F20E40F9
:106770001844704744F20C401844704744F20A40F1
:106780001844704744F208401844704744F20640E9
:106790001844704744F204401844704744F20240E1
:1067A0001844704700F58840704744F2FE301844A2
:1067B000704744F2FC301844704744F2FA301844F1
:1067C000704744F2F8301844704744F2F6301844E9
:1067D000704744F2F4301844704744F2F2301844E1
:1067E000704744F2F0301844704744F2EE301844D9
:1067F000704744F2EC301844704744F2EA301844D1
:10680000704744F2E8301844704744F2E6301844C8
:10681000704744F2E4301844704744F2E2301844C0
:10682000704744F2E0301844704744F21C4018446A
:10683000704744F2DE301844704700BF38B5144644
:106840000546FFF765FF2146B9F058F9A0F14C0362
:106850003C2B20D8DFE803F020201F1F26261F1F17
:106860002C2C1F1F1F1F1F1F1F1F1F1F1F1F1F1F1E
:106870001F1F1F1F526069444D72775B1F1F1F1F30
:106880001F32321F1F1F1F1F1F1F38381F1F1F1FC0
:106890001F1F1F3E3E0038BD00212D48BDE8384077
:1068A000FEF738BC01212A48BDE83840FEF732BC6B
:1068B00002212748BDE83840FEF72CBC03212448BC
:1068C000BDE83840FEF726BC04212148BDE8384029
:1068D000FEF720BC05211E48BDE83840FEF71ABC73
:1068E00042F28470002203212844BDE8384089F038
:1068F00027B91848BDE8384005F0BEBA002242F278
:10690000847011462844BDE8384089F019B912480E
:10691000BDE8384005F0B0BA42F28470002201218F
:106920002844BDE8384089F00BB942F28470002257
:1069300002212844BDE8384089F002B90748BDE883
:10694000384005F099BA0648BDE8384005F094BAD9
:106950007C8500307EB4003084B4003080B40030D8
:1069600082B40030F0B50F4F89B006460024EC46E3
:106970000DF101050FCFACE80F0097E80F008CE890
:106980000F00E1B23046FFF7C3FE15F8011C0DEB16
:106990004403013402355A78B9F0B6F8102CF0D11E
:1069A00009B0F0BD0806160830B5044683B0FFF7FD
:1069B000D9FF012204F580451321204601F0CEF8CD
:1069C00095F9D433002B5EDD012B6AD095EDF31AD7
:1069D000DFED377A95EDF20A31EE277AD5EDF40A3C
:1069E000B4EEC70AF1EE10FA3CD4002B1A4631EE91
:1069F000607A04F5C044B8BF5A1C013B521007EE40
:106A0000903A04F6B803013AF8EEE77A52B201EE92
:106A1000102AB8EEC11A21EE071A81EE270A30EECD
:106A2000200A83ED000AB7EE001ADFED220A2920C2
:106A300004F6B8042BF052FEF0EE407AB5209FED3C
:106A40001E0AC4ED007A7AF07BFA9FED1B0AB6208D
:106A50007AF076FA9FED180AB72003B0BDE830400F
:106A60007AF06EBA70EEE77AB4EEE70AF1EE10FA59
:106A7000BBDD04F5C04423202BF030FE04F6B80340
:106A800083ED000ACFE744F2D43001230DF1070172
:106A900020448DF807305CF093FD95F9D433012B39
:106AA00094D195EDF20A95EDF31AD5EDF40AE0E7ED
:106AB0000AD7233CCDCCCC3D0000000038B5C1F056
:106AC00011FB00240546E0B201342A4640F2DC51B5
:106AD00078F0B6F8062CF6D100230249024A0B8062
:106AE000138038BDC6B40030C4B400300023074959
:106AF000074A00F5C04010B4064C0B80138080F8A4
:106B0000BC3823805DF8044B704700BFB2B400303E
:106B1000B4B40030B0B400302DE9F843002581460C
:106B20000F46A8462E460FE0B8F0E8FF01210346C5
:106B300020468B4208BF0E46B8F0E0FFB84208BFBF
:106B40004FF00108202D12D0E9B24846FFF7E0FDD2
:106B50000135002104460028F4D0B8F0CFFF0346E9
:106B600000212046BB42DFD10120BDE8F88306EAC0
:106B70000800C0B2BDE8F88344F2E6330B4400EBF2
:106B8000430005F07DB900BF44F2E6330B4400EB4F
:106B9000430005F077B900BF70B5144684B01E46B7
:106BA0000546FFF7B5FD2146B8F0A8FF821E882AEA
:106BB00000F2A080DFE812F0F000E101DB01D80173
:106BC000D501D201CF01CC01C901C601C201BA0170
:106BD0009E009E009E009E009E009E009E00A001C2
:106BE0009C0198019E008401D204CD049E009E0069
:106BF0009E00980472044C041204EE038C039E0061
:106C00009E009E009E0067030F03A8029D0299024A
:106C1000560289000E0233019E00D50052014B013D
:106C2000CE002E015D01C2007F0178019E00760139
:106C30007401BE00BC00590157015B01BA00B800E5
:106C4000720166016401B600B4007502BE00BC00AA
:106C500070026B02BA00B80066026102B600B400AE
:106C6000E700EB019E009E009E009E009E009E009D
:106C70009E009E009E009E009E009E009E00DC00E6
:106C80002A011E01D300CC00C000DA001C011A0149
:106C9000E1009702B200B0000C0105011301B2003F
:106CA000B00001016801AE00A700950291028F02B9
:106CB000AE00A7008A028502A0009E009302830214
:106CC0008102A0009E007C027702B34C40F24F107C
:106CD000B4F900309FEDB11ADFEDB10A0A3B00EEC6
:106CE000103AB8EEC00A2BF0F9FCBDEEC00A10EE67
:106CF000103A238004B070BD0521AA4804B0BDE855
:106D00007040FEF7C9B90421A64804B0BDE8704040
:106D1000FEF7CAB90421F0E70321F5E70321ECE708
:106D20000221F1E70221E8E70121EDE70121E4E793
:106D30000021E9E70021E0E7002EDBD142F2847078
:106D400001220221284404B0BDE8704088F0F8BE5A
:106D5000002ECFD1012242F284701146F2E7002EBC
:106D6000C8D142F2847001220021EBE7002EC1D18C
:106D700042F2847001220321E4E78B4804B0BDE8AD
:106D8000704005F06FB8002EB4D10221854804B0E0
:106D9000BDE87040FEF790B905F5C043012246F604
:106DA0004C0093F8913011462844002B00F0EA8003
:106DB00004B0BDE87040FBF743B9002E9AD103211F
:106DC000E4E70321774804B0BDE87040FEF734B92A
:106DD0000321744804B0BDE87040FEF79BB903215D
:106DE000704804B0BDE87040FEF73EB96F48C5E793
:106DF0006F48C3E7002E7FF47DAF42F28470032119
:106E0000284404B0BDE8704088F068BE42F2847047
:106E10000022B0E742F284700022012192E7002EA6
:106E20007FF468AF05F5C04245F6745092F8BD385E
:106E300083F0010382F8BD38002B00F0B7835D4A70
:106E40000621284404B0BDE870406DF0B3B8002EB0
:106E50007FF450AF42F284703146D1E7002242F213
:106E6000847011466EE70121ACE70021B1E70121F2
:106E7000B6E7002E7FF43EAF42F284700121BFE7F7
:106E80000221ADE702219DE7002E7FF433AF0321FD
:106E9000444804B0BDE87040FEF724B9012198E7EA
:106EA00000219DE700218DE7002E7FF423AF42F201
:106EB00084700221A4E742F284700022022141E79B
:106EC000002E7FF417AF3C4AB720137883F00103FC
:106ED0001370002B00F06C839FED380A7AF030F8C5
:106EE00045F67450364AABE7364B374A1A6001E72D
:106EF000344B364A1A60FDE647F6B8349FED341A33
:106F000005F5E04600222C44F0EE410A96F8291CD3
:106F1000B0EE410A20467BF099FD032296F8291C29
:106F2000204604B0BDE870407BF07EBD01221521F3
:106F3000284604B0BDE8704000F010BE012228468B
:106F40001146F6E701220421F2E701220721EFE7CB
:106F500001220321ECE701221021E9E701220221AD
:106F6000E6E701220021E3E701221321E0E7012205
:106F700046F64C00114628441AE7012246F64C001A
:106F80001146284404B0BDE87040FAF7CBBF002E8C
:106F90007FF4B0AE02217BE7C6B400300000484366
:106FA000000048C37C85003082B4003080B40030DB
:106FB0007EB400302C6A1608C8B4003000007A4451
:106FC000B0691608DC240030008089440080ED445C
:106FD0000000000005F5C04494F89130012B7FF4C7
:106FE00089AE002E7FF486AED54BD649B3F900307A
:106FF000A3F5FA7383EAE372A2EBE372322AD24A70
:10700000D4BF33461BB2B2F900200B80CF49D04E1B
:10701000B1F9000082EAE271A1EBE27189B2322992
:1070200080EAE071A1EBE07198BF002289B2328062
:10703000322900F2C582C74900201343088000F0BE
:10704000C782012345F67450C34A062184F8BC3830
:1070500028446CF0AFFF94F8BC3883F00103BF4ABA
:10706000137047E6BE4C4FF4A6709FEDBE1AB4F9FC
:107070000030DFEDBD0A0A3331E6002E7FF43AAE70
:10708000012105E7002E7FF435AE01217EE6002EBA
:107090007FF430AE3146FBE6002E7FF42BAE314656
:1070A00074E6022195E6002E7FF424AE0521EFE67A
:1070B000002E7FF41FAE052168E6052190E605212C
:1070C00080E6002E7FF416AE0421E1E6002E7FF468
:1070D00011AE04215AE6042182E6042172E605215C
:1070E00077E6042175E6A14848E6A14C40F2491034
:1070F000EEE59F4C4FF4A3709FED9A1AB4F900305F
:10710000DFED990A0A33EAE5002E7FF4F3AD05F5C9
:1071100080449FED981ADFED980A4FF49C7094ED2F
:10712000F40A2BF0DBFA44F2D03003A98DED030A08
:1071300028445CF0EBF9B7EE001AD4EDF40A40F203
:10714000391094EDF30A2BF0C9FA44F2CC3003A9BC
:107150008DED030A28445CF0D9F90A22012194F943
:10716000D4032BF027FB034644F2D43003A98DF857
:107170000C3028445CF024FA94F9D433012B00F04D
:107180002F82013B94EDF31AD4EDF40A46F6B804CD
:1071900007EE903A40F23F1071EE606A2C44F8EE30
:1071A000E77A94ED000A86EEA77A30EE470A2BF0D4
:1071B00095FA84ED000AB7EEC07A45F674506F4A2E
:1071C000062128449FED5A6B27EE067B8DED007B50
:1071D0006CF0F0FE8EE5002E7FF48CAD05F580445A
:1071E0009FED641ADFED640A4FF4947094EDF40A95
:1071F0002BF074FA44F2D03003A98DED030A284431
:107200005CF084F9B7EE001AD4EDF40A40F22910CC
:1072100094EDF30A2BF062FA44F2CC3003A98DED21
:10722000030A28445CF072F90A22012194F9D4037C
:107230002BF0C0FA034644F2D43003A98DF80C3089
:1072400028445CF0BDF994F9D433012B00F0D881C7
:10725000013B94EDF31AD4EDF40A46F6B80407EEB8
:10726000903A40F22F1071EE606A2C44F8EEE77A03
:1072700094ED007A86EEA70A30EE070A2BF02EFA7C
:1072800084ED000A97E7002E7FF434AD3C4946F6C2
:10729000B804B7EE006A45F674500B78F6EE006A53
:1072A0002C44384A83F0010328449FED215B9FED75
:1072B000227B002B0B704FF0060105FE077B46FE7C
:1072C000266AC4ED006A8DED007B6CF073FE11E55B
:1072D000002E7FF40FAD05F58045DFED2D6A2A4CB9
:1072E00040F21510B5F9DC33B0EE661A94ED000AE1
:1072F00007EE103ADFED250AB8EEC77AC6EE877AB8
:10730000FCEEE77A17EE903A9BB207EE903AF8EE71
:10731000E77A30EE670A2BF0E1F9B62084ED000A37
:1073200004B0BDE8704079F00BBE00BFAFF3008041
:10733000000000000000594000000000000049402B
:10734000BAB40030B4B40030B6B40030B8B40030D1
:10735000B0B40030B2B40030046A1608D42400304F
:10736000C6B4003000004843000048C384B4003075
:10737000C4B40030CDCC4C3FCDCCCC3DF069160828
:10738000C9B40030E0691608C0B400300000000045
:1073900000007A44002E7FF4ADAC05F580455FED2A
:1073A000046A9F4C4FF48770B5F9DC33B0EE661A6F
:1073B00094ED000A07EE103ADFED9A0AB8EEC77AAC
:1073C000C6EE877AFCEEE77A17EE903A9BB207EEAC
:1073D000903AF8EEE77A37EE800A9CE7002E7FF4C9
:1073E00089AC05F580409FED901A904CB0F9DC33E4
:1073F000227807EE103A8A4DB8EEC77AC1EE077AC6
:10740000FCEEE77A17EE903A9BB207EE903AF8EE70
:10741000E77A002A00F0BD8095ED000A40F20110E5
:10742000DFED800A37EE800A2BF058F985ED000A6F
:10743000DFED7D7AB4EEE70AF1EE10FA80F2988083
:10744000B5EEC00AF1EE10FA40F29280B62067E77E
:10745000002E7FF44FAC05F58045DFED736A744C68
:10746000F820B5F9DC33B0EE661A94ED000A07EEA9
:10747000103ADFED6C0AB8EEC77AC6EE877AFCEEFA
:10748000E77A17EE903A9BB207EE903AF8EEE77A79
:1074900030EE670A2BF022F9B5203FE7002E7FF48B
:1074A00029AC05F58045DFED606A614CF120B5F946
:1074B000DC33B0EE661A94ED000A07EE103ADFED09
:1074C000590AB8EEC77AC6EE877AFCEEE77A17EE6D
:1074D000903A9BB207EE903AF8EEE77A37EE800AE0
:1074E0002BF0FCF8B52019E7002E7FF403AC05F56E
:1074F00080409FED4D1A4F4CB0F9DC33227807EEF7
:10750000103A4B4DB8EEC77AC1EE077AFCEEE77A37
:1075100017EE903A9BB207EE903AF8EEE77A62B334
:1075200095ED000AE420DFED3F0A37EE800A2BF0EC
:10753000D5F885ED000ADFED3C7AB4EEE70AF1EE0E
:1075400010FA10DAB5EEC00AF1EE10FA0BD9B52038
:10755000E6E6394B394A1A60FFF7CCBB364B384A5E
:107560001A60FFF7C7BB237883F001032370EEE7AF
:10757000237883F00103237068E795ED000AE62085
:10758000DFED280A30EE670A2BF0A8F885ED000A37
:10759000D1E795ED000A40F20310DFED220A30EE4C
:1075A000670A2BF09BF885ED000A41E7254A47E47E
:1075B0009FED1C0A79F0C4FC45F67450224A3FE462
:1075C00003431343214A1BB21080002B7FF439ADD3
:1075D00094F8BC38002284F8BC28A3B901233EE506
:1075E00040F23D1094EDF31AD4EDF40A94EDF20A52
:1075F0002BF074F846F6B8032B4483ED000ADAE565
:1076000040F22D10EEE745F67450114A0621284449
:107610006CF0D0FC94F8BC3883F001031FE500BF88
:10762000C0B400300000000000007A44E1240030C3
:10763000BCB40030E0240030D824003000808944FD
:107640000080ED44406A1608C8691608B2B40030DC
:10765000146A16082DE9F04F2DED088B85B007460A
:107660009FEDCDAA00F58040019307F5C04ABDF912
:1076700058300024BDF85C5089460AEE903ABDF8B7
:107680006030DFEDC67AA34645EA03450AF6B80343
:10769000D0EDF66AB0EE678AD3ED009A01269FED31
:1076A000C07A29EE8AAABF4B9FEDBF6AC3ED007A6C
:1076B0002AEE26AABD4B69EE869A0092C3ED007AA7
:1076C000AAEE478ABDF968300293BDF96C30039386
:1076D000BDEEC88A18EE103A1BB208EE103A01E06F
:1076E000202C11D006FA04F3E1B201342B42F7D07A
:1076F0003846FFF70DF80021B8F000FA012808BF5E
:107700004FF0010B202CEDD10024A94E4FF00108C1
:1077100008EE907A06E03268134240F0E7800134C8
:10772000202C11D008FA04F3E1B22B42F3D03768D1
:1077300001345A4618EE900A3B4214BF012300233D
:10774000FFF72AFA202CEDD19AF8BD383560002BCE
:1077500040F0E680DFF87C82964EC0F0C3FC964A8B
:1077600004461378002B40F0C78094496FF4E17011
:10777000934D0988934F01F5FA7109B209EE101A79
:1077800001990144B5F9000089B28346B7F90000B8
:1077900062290BEE100A40F21F811370B8F8000046
:1077A00040F26C72029B40F24C4100F2DC50DFED83
:1077B0007B8A184400B22AF0FDFF224601460020D1
:1077C00077F03EFA3088039B40F26C7200F2DC5096
:1077D00040F24C41184400B22AF0ECFF2246014628
:1077E000012077F02DFAB8EEC99AB8EEC88A40F2B7
:1077F0006C7240F24C41A9EE0A8AFDEEC87A17EE8F
:10780000903A18B22AF0D6FF22460146022077F0BD
:1078100017FAF8EEEAAAF0EE687A40F26C7240F2DB
:107820004C41EAEEA97AFDEEE77A17EE903A18B2EB
:107830002AF0C0FF22460146032077F001FA9AF8A9
:10784000BD38002B40F08980F8EECB7A40F26C72A4
:10785000B0EE687A40F24C41A7EEA97AFDEEC77A05
:1078600017EE903A18B22AF0A5FF224601460420EE
:1078700077F0E6F907EE90BAF8EEE77A40F26C722C
:1078800040F24C41E7EEA98AFDEEE87A17EE903A15
:1078900018B22AF08FFF22460146052077F0D0F972
:1078A000424B22460620D3ED007AFDEEE77A17EE32
:1078B000903A19B277F0C4F93A4B22460720D3ED3B
:1078C000007AFDEEE77A17EE903A19B277F0B8F940
:1078D0003D4B3E4A0099A3F8009011803C4B019A21
:1078E0001A8005B0BDEC088BBDE8F08F5A4618EE43
:1078F000900AFEF7A3FF12E7304B019A1B88304D28
:107900001344009A2F4F1BB209EE103A2B881344F0
:107910001BB29B463B884B441BB20BEE103A3DE733
:10792000DDED007AC9F10003224EB8EEE77A07EEEA
:10793000903ADFF8A080F8EEE77A27EE297A67EE32
:10794000A97ABDEEC77AFDEEE77A17EE103A3380DA
:1079500017EE903AA8F80030FFE6B7F90030F0EEE5
:10796000687A40F26C7240F24C4107EE103AB8EE81
:10797000C77AE7EE297AFDEEE77A17EE903A18B269
:107980002AF018FF22460146042077F059F9B5F98C
:10799000003007EE903A6FE7CDCC4C3F0080BB44FF
:1079A0000000FA43DC240030CDCCCC3ED82400309B
:1079B000ACB40030C4B40030D4240030B4B40030CF
:1079C000B2B40030B0B40030B6B40030B8B4003057
:1079D000BAB40030C6B400300099084681EAE171BB
:1079E000A1EBE07189B231293FF6D7AE89EAE9739C
:1079F000A3EBE9739BB2312B8CBF00230123CCE6B0
:107A00000120704700207047002070470020704719
:107A100000207047002070479FED010A704700BFAB
:107A200000000000704700BF134A144930B4144DE1
:107A300002F1B804C0E90012C0E90245A5F64811F8
:107A4000A2F5DB54C0E90441A5F57E610D4CC0E907
:107A5000064108340831C0E9084102F5AD54083147
:107A6000A2F58142C0E90A41074C08498263C0E996
:107A70000C4130BC704700BF38700030D46A160823
:107A8000AC950030C8850030B09A00308496003044
:107A9000034615290CD8DFE801F01115191D210B3B
:107AA0000B250B290B0B0B0B0B0B2D0B0B31350D7A
:107AB0000020704748F284701844704748F26850BC
:107AC0001844704748F2A4501844704748F2E050F8
:107AD0001844704748F21C601844704748F25860D8
:107AE0001844704748F2D0601844704748F20C7050
:107AF0001844704748F294601844704748F22C507C
:107B00001844704748F248701844704700F5004028
:107B1000D0F8280503685B68184700BF38B500F542
:107B200000450446D5F8280503685B69984704F5C5
:107B3000A041D5F82835084A91F88C1F10741846D2
:107B4000D1701A68136A9847014642F2D8702044EF
:107B5000BDE8384052F042BA78B600302DE9F8431B
:107B600000F5A0490446904699F88C3F8B426ED0B0
:107B7000FFF78EFF0546002878D003680F469B6804
:107B8000984728B13C4804F0C3FD0646002866D05B
:107B90003948FAF7E5FBA0B904F50043D3F8280506
:107BA0000368DB68984760B12B682846DB68984714
:107BB000064630B92B682846DB6998472F4A0346AA
:107BC0000CE02B68002128461B6898470646A0B9A0
:107BD0002B682846DB699847294A034645F67450C6
:107BE000042120446CF0E6F968F00CFC3A460A21C6
:107BF00068F02AF93046BDE8F88304F5E04347F61B
:107C0000B83093F8291C20447AF0FEFE99F88C3F96
:107C100045F63010424689F88D3F04F50043394659
:107C20002044C3F8285504F5804389F88C7F83F8F5
:107C3000188167F0A5FC45F674500021204472F0CD
:107C4000ABFA2046FFF76AFF3046BDE8F88300F53F
:107C50008044012684F818213046BDE8F8832B685B
:107C60002846DB699847074A0346B7E720462E4671
:107C700065F03EFFBEE700BFB02C0030806A1608FA
:107C8000AC6A1608546A16080148FFF767BF00BFC0
:107C9000B02C003070B52DED068B09EE901A09EE70
:107CA000102A92B04FF0000CB8EEE90B0446B8EE83
:107CB000C97BCDF80CC0CDF810C020EE000BCDF87C
:107CC00014C0CDF818C0CDF81CC0CDF820C0019369
:107CD000A7EE070BB5EE400BF1EE10FA00F1A48110
:107CE000B1EEC07BB7EEC77BDFEDD27AB4EEE77AB8
:107CF000F1EE10FA17DDC7EE876AF8EEE99AB8EEF2
:107D0000C99A69EEA69A29EE269AFDEEE99ABDEE89
:107D1000C99A19EE903A1BB209EE903A19EE103A50
:107D20001BB209EE103A636893ED2B7AB5EEC07A78
:107D3000F1EE10FA4DD9F7EE007AB4EEE77AF1EEF3
:107D400010FA04DDC3ED2B7A636893ED2B7AB8EE5D
:107D5000E96A9FEDB80AF8EEC96A93ED264AF7EE94
:107D6000007AC6EE005A86EE806A77EEC77A65EE34
:107D7000A54A67EEA56A64EEA55A27EE868A26EE26
:107D8000065AE5EE876AF0EE487A25EE066AE6EED8
:107D9000077A26EE807A27EE04AA27EE808A28EE5C
:107DA000048A9DED017AD3ED277AF8EEC78A93F91C
:107DB000A83068EEA78ABBB91C9B83ED00AA1D9B67
:107DC00083ED008A1E9BC3ED008A12B0BDEC068BCA
:107DD00070BDB8EEE97A93ED260AB8EEC98A27EEAF
:107DE00000AA28EE008ADCE72369D3F8F0012AF024
:107DF000ABFB40F6B832904905462AF0CBFC434233
:107E000007EE903A6368F8EEE77A93ED287A2369F3
:107E100067EE877AD3F8F401CDED037A2AF094FB6C
:107E200040F6B832844906462AF0B4FC43420022A8
:107E300007EE903A63680592F8EEE77AD3ED296A87
:107E400093F9A82067EEA67A022ACDED047A00F015
:107E5000A180666B0CAD9FED790A06F148002FF00A
:107E6000F5FA12AA09AB8DED0F0ACDED100A8DEDD2
:107E7000111A9FED730A12E9070083E8070085E8ED
:107E8000070018462FF0E2FA06AB2946304603AA4F
:107E90008DED0C0ACDED0D0A8DED0E1AB2F066FFD8
:107EA000636893F9A830022B00F0928019EE103A23
:107EB00019EE902A9FED5F7AB7EE001A002BDFEDE6
:107EC000610A4FF48270B8BF5B42002AB8BF5242C9
:107ED0009BB292B29342B8BF1346019A002AB8BF30
:107EE000524292B29342B8BF134607EE903AF8EE70
:107EF000E77A87EE870A31EE400A2AF0EFFB236922
:107F000006A8D3ED917A20EE270A2FF09FFAF0EE23
:107F1000CA7A8DED081A4FF48670F0EEC06ACDED86
:107F2000070AB0EE407A30EE0A0A37EEE61A8DED17
:107F3000067AB0EEC11AF1EE410A2AF0CFFBDDED70
:107F4000077AB0EEC81A40F21110B0EEE77AB0EE40
:107F500040AA37EE880A31EE471AB0EEC11AF1EEA8
:107F6000410A2AF0BBFBDDED087AB0EEE81A4FF4C7
:107F70008B70B0EEE77AB0EE408A38EEA70A31EEA9
:107F8000471AB0EEC11AF1EE410A2AF0A7FBF0EE53
:107F9000408A11E72C4AB2F98423AA4233DAAD1A97
:107FA000D3ED285A07EE105AB8EEC76A9DED037A52
:107FB000A5EEC67A8DED037AB24216DAB21A07EE52
:107FC000102AB8EEC77AE6EEC77ACDED047A40E71C
:107FD000DDED066A9DED077ADDED087A3AEE26AA18
:107FE00038EE078A78EEA78AE6E65342B3427FF777
:107FF00030AF324407EE102AB8EEC77AE6EEC77A01
:10800000CDED047A25E75142A942D5DD15449DED19
:10801000036AD3ED285A07EE105AB8EEC77AA5EED8
:10802000C76A8DED036AC7E731F190FAB0EE407B85
:1080300058E600BF00A08C4548F4FFFF9F0CB345F5
:10804000D302373900000000B06C00300148FFF760
:1080500085BD00BFB02C003000487047248A003036
:1080600000207047012070470120704700207047B2
:10807000004870470C6B1608004870470C6B1608D8
:1080800008B5034606489FED047B1B6B83EDD87B48
:10809000FEF714FD012008BD0000000000000000F4
:1080A000B02C003070B50446406988B090F8DD30DF
:1080B000002B3ED00221B8F033FF636A07A81B688B
:1080C000D4E90612B3F9083012680968B2F9082039
:1080D000B1F90810029006A8019005A8009020466A
:1080E000FFF7D8FD606B9DED071A0368DDED060A0A
:1080F0009DED050A9B6B9847656B226A2B6810689B
:108100009E6D76F091FF636800212846D3ED020A48
:10811000B047A36A6569186876F086FF85ED0E0A98
:10812000E36A6469186876F07FFF84ED0F0A08B08F
:1081300070BD0121B8F0F4FE606B62680121036834
:10814000D2ED020A9FED040A9B6D9847606B08B060
:10815000BDE87040B2F022BF000000000020704770
:10816000002070470120704700207047004870478A
:10817000546B160800487047606B16080346B6EE4D
:10818000061AF4EE000A302093ED4E0A2AF0A6BA41
:1081900070B504462248FAF7E3F8054600283CD0BB
:1081A0001F48266BFAF7AEFC0346626830465B4216
:1081B00000EE103AB2F92C3001EE103AB2F9283044
:1081C000B8EEC00A00EE903AB8EEC11AF8EEE00A36
:1081D000B4F026FD1248266BFAF794FC0346626859
:1081E00030465B4200EE103AB2F92C3001EE103A04
:1081F000B2F92830B8EEC00A00EE903AB8EEC11AD3
:10820000F8EEE00AB4F08AFD206BB4F093FD226929
:10821000044BD2F8F821C3F81425284670BD00BFDE
:10822000B02C0030B0AC003070B504462DED028BA0
:108230008AB0BFF057FF06468C48256BFAF762FC00
:108240000346626828465B4200EE103AB2F92C30D1
:1082500001EE103AB2F92830B8EEC00A00EE903ABA
:10826000B8EEC11AF8EEE00AB4F0DAFC606990F8F2
:10827000DD30002B7CD07E4D0221B8F051FE41F262
:108280008732D5F8E434F31A934240F2B080606B41
:10829000D4E906231B681268B3F90830B2F9082044
:1082A00000EE903A036808EE102AF8EEE00ADB6D63
:1082B000B8EEC88ACDED010A9847DDED010AB0EEAF
:1082C000401AA5F50040B0EE480A04AA03A9FAF73F
:1082D00071FA636A1868438A828907EE903A654B9F
:1082E000F8EEE77A93ED007A67EE877AFCEEE77AAC
:1082F00017EE903A99B276F02DFE0146A5F50040B2
:10830000FAF7D2FAB0EEC07ADFED5B7AB4EEE77A34
:10831000F1EE10FA14D4606BB0EE401ADDED040AF1
:1083200003689DED030A9B6A98472369D3F8F831E7
:10833000C5F81865C5F814350AB0BDEC028B70BDE0
:10834000D5F81835606BFA33B3423ED903689FED18
:108350004B1ADDED040A9DED030A9B6A98472369D9
:10836000D3F8F831C5F814350AB0BDEC028B70BDF6
:108370000121B8F0D5FD606B626801210368B6EE9B
:10838000000AD2ED020A9B6D9847606BB2F006FEC0
:1083900063693B491A68256BD2688A4262D1B6EE9E
:1083A000061A3020F4EE000A93ED4E0A2AF096F9F0
:1083B0002846B4F043FD22692D4BD2F8F821C3F8CA
:1083C00014250AB0BDEC028B70BD05F214530121D7
:1083D000DDED040A93ED001A0368B8EE411A9DED35
:1083E000030ADB6A98470AB0BDEC028B70BD05F248
:1083F000F44205F2EC4105F59E6305F59F651668AC
:1084000006A82A6809681B68069103A9079305ABAB
:10841000099204AA08962DF0DBFF9FED1A7A01213C
:10842000DDED037ADDED040A9DED051A67EE877A2E
:1084300060EE870A606B21EE071A9FED130ACDEDFF
:10844000037ACDED040A60EE800A8DED051A21EE67
:10845000001A036827EE800ADB6A98470AB0BDEC71
:10846000028B70BD18469047A2E700BFB02C0030C9
:10847000B0AC00306895003000000034000000000F
:108480007D810208E02E65420000C84238B5836A4B
:1084900004464569186876F0C7FD85ED0E0AE36A63
:1084A0006469186876F0C0FD84ED0F0A38BD00BF1E
:1084B00030B504463A482DED028B236A83B01B6821
:1084C000B3F9083000EE103AB8EEC00AFAF774FAC1
:1084D00033488DED010AFAF715FB626803469DEDFE
:1084E000010A6C20B2F928205B4201EE102A00EE4E
:1084F000903AB8EEC11AF8EEE00A2AF0EFF8B0EEC2
